:020000040000FA
:1000000000EFF6F08FEF00F0E9CF11F1EACF12F137
:10001000D9CF13F154EF22F0D8CF31F0E8CF32F03E
:10002000E0CF33F0E9CF34F0EACF35F0E1CF36F06E
:10003000E2CF37F0D9CF38F0DACF39F0F3CF3AF05A
:10004000F4CF3BF0F6CF3CF0F7CF3DF0F8CF3EF0E9
:10005000F5CF3FF09DA001D001D00AD09EA001D0E5
:1000600001D006D09FB001D001D002D031ECACF06D
:10007000A0A201D001D00AD0A1A201D001D006D007
:10008000A2B201D001D002D0B1EC0FF09DA401D0FA
:1000900001D00AD09EA401D001D006D09FB401D0D7
:1000A00001D002D023EC42F09DAA01D001D00AD0A9
:1000B0009EAA01D001D006D09FBA01D001D002D0B3
:1000C000FCECF2F0A3AA01D001D00AD0A4AA01D07E
:1000D00001D006D0A5BA01D001D002D0DEEC3BF0B1
:1000E0003FC0F5FF3EC0F8FF3DC0F7FF3CC0F6FF44
:1000F0003BC0F4FF3AC0F3FF39C0DAFF38C0D9FF84
:1001000037C0E2FF36C0E1FF35C0EAFF34C0E9FF87
:1001100033C0E0FF32C0E8FF31C0D8FF100028EF45
:100120001FF0FFFFFFFFFFFFFFFFFFFFFFFFFFFFCE
:10013000FFFFFFFFFFFFFFFFFFFFFFFFFFFFFFFFCF
:10014000FFFFFFFFFFFFFFFFFFFFFFFFFFFFFFFFBF
:10015000FFFFFFFFFFFFFFFFFFFFFFFFFFFFFFFFAF
:10016000FFFFFFFFFFFFFFFFFFFFFFFFFFFFFFFF9F
:100400001F1F1F1B1B1B1B1B13131313131319116C
:10041000130919191919191919191B1D1919190075
:100420000005310791073207920733079307340716
:1004300094073505950599073907360537053805B9
:1004400098050000960544070A0314000101020004
:100450000000EFFF009091A5FE123400000303009E
:1004600034CB123403010104000A0206010000002B
:100470000F02033C02020800000000000000000020
:10048000090909090911780585054005410588050F
:100490008907900770007105696E7465726E6574E6
:1004A0002E6C6D742E6C76000000000000000000C1
:1004B00000000031313131313131310000000000B4
:1004C00000000000000000003932330000323133F8
:1004D0002E32312E3139362E363800000047736DFA
:1004E00054736300000000000000000000000000E2
:1004F00000000000000000000000000000000000FC
:1005000000000000000000000000000000000000EB
:1005100000000000000000000000000000000000DB
:1005200000000000000000000000000000000000CB
:1005300000000000000000000000000000000000BB
:1005400000000000000000000000000000000000AB
:10055000000000000000000000000000000000009B
:10056000000000000000000000000000000000008B
:10057000000000000000000000000000000000007B
:10058000000000000000000000000000000000006B
:10059000000000000000000000000000000000005B
:1005A000000000000000000000000000000000004B
:1005B000000000000000000000000000000000003B
:1005C000000000000000000000000000000000002B
:1005D000000000000000000000000000000000001B
:1005E000000000000000000000000000000000000B
:1005F00000000000000000000000000000000000FB
:1006000000000000000000000000000000000000EA
:1006100000000000000000000000000000000000DA
:1006200000000000000000000000000000000000CA
:1006300000000000000000000000000000000000BA
:1006400000000000000000000000000000000000AA
:10065000000000000000000000000000000000009A
:10066000000000000000000000000000000000008A
:10067000000000000000000000000000000000007A
:10068000000000000000000000000000000000006A
:10069000000000000000000000000000000000005A
:1006A000000000000000000000000000000000004A
:1006B00000000000460545054205430501A0A1A232
:1006C000A3A4A5A6A7A8A9AAABACADAEAF01B0B133
:1006D000B2B3B4B5B6B7B8B9BABBBCBDBEBF01C042
:1006E000C1C2C3C4C5C6C7C8C9CACBCCCDCECFD082
:1006F000D1D2D3D4D5D6D7D8D9DADBDCDDDEDFE072
:10070000E1E2E3E4E5E6E7E8E9EAEBECEDEEEF0051
:1007100000000000000000000000000000000000D9
:10072000696E7465726E6574000000000000000060
:1007300000000000000000000000000000000000B9
:1007400000000000000000000000000000000000A9
:10075000033E033E033E033E033E00000000000054
:100760000000000000000000000000000000000089
:100770000000000000000000000000000000000079
:100780000000000000000000000000000000000069
:100790000000000000000000000000000000000059
:1007A0000000000000000000000000000000000049
:1007B0000000000000000000000000000000000039
:1007C0000000000000000000000000000000000029
:1007D0000000000000000000000000000000000019
:1007E0000000000000000000000000000000000009
:1007F00000000000000000000000000000000000F9
:100800000401CD6713D0656A0F015C6B02D0658669
:10081000040065A6FCD7010E0401CD6F140E0F0174
:100820005F6F65BAFED7626AA8D8A0880401CD05BB
:10083000D8B465BA02D0626AA0D862A409D00F0108
:100840005CA506D065925C9501D0629462B4FDD738
:1008500065B2120062A012D00F015CA10FD03DEC76
:1008600047F0040E0401CD6F040E0401036F200E47
:10087000026F080E016F8C0E006F629062A807D0A5
:100880000F015CA904D05C8562986582629862ACB5
:1008900003D00F015CBD629C62AA11D00F015CAB5A
:1008A0000ED04CA10BD004010051800A05E1045187
:1008B000840A02E18C0E006F0F014C91629A636A08
:1008C000040E0401CD6101D0040C0F015CA708D017
:1008D00062B604D005D007EC12F0629662B6FBD780
:1008E00004011CBF12000401B151030A01E1B16B04
:1008F0000401B16701D012000401B151020A09E1FB
:1009000004011E6B1F6B1D6B26EC4EF0030E0401E1
:10091000B16F0401B105D8A41200B2C4CBF4400EEB
:100920000401B26502D00401CB6F0401CB51040174
:10093000B25FB2670AD0030E0401B16F0401CB515C
:10094000400A03E1020E0401B16FCBC41DF4040E92
:1009500004011F6F700E1E6F040E0401CA6F700E2B
:10096000C96FB3C4C7F4B4C4C8F41CEC45F0C7C421
:10097000B3F4C8C4B4F426EF4EF00F015C6B5C8195
:100980005C89020E0401CD6F020CE8CF3BF1900EA2
:10099000F66EEB0EF76E000EF86E21EE35F0060ED9
:1009A0000900F5CFDEFFE82EFBD70101010E1D6F18
:1009B000350E1C6F010E13EC3CF03D0E00EC4CF0BC
:1009C00001013BC11BF11C6BDDEC2DF01BC13CF1A7
:1009D0001CC13DF120EE03F03C51D9263D51DA22F5
:1009E000DF505BEC4CF000EC4CF0010120EE04F029
:1009F0003C51D9263D51DA22DF505BEC4CF000EC43
:100A00004CF00D0E00EC4CF042EC4EF00101406B4E
:100A10003E6B77D018EC4EF074E33EEC4EF00101E3
:100A20003F6F61D0350E4025D96EDA6A010EDA22A9
:100A3000DF50336F346B33BF34073F5133193411F8
:100A400002E0406B5ED0402B01014051050A59E1A4
:100A50003E2BF7D73F512C0A54E101013E2B51D0D8
:100A60003F51220AF9D73F51220A04E13E2B40C1EF
:100A700030F5E7D7200E01014025D96EDA6A050E60
:100A8000DA223FC1DFFF402B4051800A700F39E36B
:100A9000070E306FD00E2F6F77EC40F0D890120019
:100AA0003F518FEC4AF0D9E22CD03F510D0A04E1BE
:100AB0003E2B40C1E5F5C5D7310E01014025D96E69
:100AC000DA6A050EDA223FC1DFFF402B4051800A6F
:100AD000580FDDD7070E306FD00E2F6F77EC40F038
:100AE000DDE3D88012003E519DE0010AB3E0030A25
:100AF000B7E0010AB8E0070AD3E0010AD6E0030A2A
:100B0000E9E01FEC4EF0D10E01012F5D070E3059C8
:100B1000C5E280D754C11EF155C11FF1F6EC37F084
:100B20005C6F9F0E5C650AD0B00E5C6107D0020E50
:100B30001F6FBC0E1E6FF6EC37F02FD0AF0E5C654A
:100B40000AD0C00E5C6107D0020E1F6FCD0E1E6F63
:100B5000F6EC37F022D0CF0E5C6504D0E00E5C617D
:100B600001D0E5D7DF0E5C6504D0F00E5C6101D0EA
:100B7000EBD7BF0E5C650AD0D00E5C6107D0020EC9
:100B80001F6FDE0E1E6FF6EC37F007D054291E6F74
:100B9000000E55211F6FF6EC37F0576F5CC146F120
:100BA000000E10EC07F0010146C15AF147C15BF19C
:100BB0005AC11EF15BC11FF1010E206F90EC21F0B4
:100BC0005AC11EF15BC11FF1020E206F90EC21F0A3
:100BD0005AC11EF15BC11FF1030E206F90EC21F092
:100BE0005AC11EF15BC11FF1040E206F90EC21F081
:100BF0005AC11EF15BC11FF1050E206F90EC21F070
:100C0000010E596F000114A82AD085EC46F00101AD
:100C1000566F5AC13FF15BC140F1010E416F56C1A1
:100C200042F1030E436F16EC3DF002E2D890120041
:100C3000020E596FD8905733586B57A107D05951AE
:100C400085EC46F01FD816EC3DF0F0E3D890573312
:100C5000592B582B020E5865F0D7D880120001018D
:100C6000586B57A107D0595185EC46F00BD816ECBC
:100C70003DF0DCE3D8905733592B582B030E5865C1
:100C8000F0D7EBD70101566F5AC13FF15BC140F17C
:100C900059C141F156C142F1030E436F030CE8CF35
:100CA00028F1310E01012825D96EDA6A050EDA2203
:100CB0003A0EDF6E282BC441E8423F0B1F0B1B6F1F
:100CC0001C6BDDEC2DF070D85BEC4CF080D85BEC4D
:100CD0004CF0DF6E282BC545E846030BC4C124F158
:100CE00097D824130F0E24151B6F000E1C6BDDEC20
:100CF0002DF05AD85BEC4CF06AD85BEC4CF0DF6E10
:100D0000282BC645010BC5C124F1256BD89024378B
:100D1000253724137F0E24151B6F000E1C6BDDEC92
:100D20002DF042D85BEC4CF052D85BEC4CF0DF6E0F
:100D30005FD8050EDA222D0EDF6E282BC239E84669
:100D40001F0B1B6F1C6BDDEC2DF02ED85BEC4CF0F9
:100D50003ED85BEC4CF0DF6E282BC339E842070B22
:100D6000C2C124F155D84BD8DDEC2DF01DD85BEC79
:100D70004CF02DD85BEC4CF0DF6E282BC445010BFA
:100D8000C3C124F1256B3BD8DDEC2DF00DD85BEC15
:100D90004CF01DD85BEC4CF0DF6E2AD80501050E37
:100DA000DA22000EDF6E000C1BC126F11CC127F1F8
:100DB000310E01012825D96EDA6A050EDA2210EE0D
:100DC00003F02651E1262751E222E7501200DF6EA0
:100DD000282B310E01012825D96EDA6A050EDA2298
:100DE00010EE04F02651E1262751E222E7501200CE
:100DF000282B310E01012825D96EDA6A1200D8900D
:100E00002437253724133F0E24151B6F1C6B000C51
:100E1000256BD89024372537D890243725371200F2
:100E2000E8CF48F10101496B040E1F6F020E1E6FDF
:100E3000F6EC37F0516F040E1F6F030E1E6FF6ECC9
:100E400037F0506F5151536F5051526FFF0E525D3A
:100E5000000E535917E2524B532B5351516F52C14D
:100E600050F1040E1E6F020E1D6F51C11FF1E2EC16
:100E70003DF0040E01011E6F030E1D6F50C11FF1E6
:100E8000E2EC3DF0040E01011F6F000E1E6BF6EC4C
:100E900037F0516F040E1F6F010E1E6FF6EC37F026
:100EA000506F5151536F5051526FFC0E52254E6F7F
:100EB000FB0E53214F6F4EC123F14FC124F1266B1E
:100EC0000E0E256F1FEC44F023C14AF124C14BF1F3
:100ED00025C14CF126C14DF14B514A1109E0500E8C
:100EE000266FD40E256FA3EC40F0E7EC45F0FF0031
:100EF0004CC14EF14DC14FF101014651D4ECEEF021
:100F0000F4EC09F00101485134EC4EF00D0EA7EC61
:100F100041F052C11DF153C11EF1E90E01014925F5
:100F2000D96EDA6A000EDA22DF501F6FE2EC3DF074
:100F30000101524B532B492B4951800A720FE9E3AF
:100F4000E80E525D110E535911E3040E506F1E6FDF
:100F50001D6B1F6FE2EC3DF0040E01011E6F010ED0
:100F60001D6F040E1F6FE2EC3DF015D05351516F11
:100F700052C150F1040E1E6F000E1D6B51C11FF1C6
:100F8000E2EC3DF0040E01011E6F010E1D6F50C119
:100F90001FF1E2EC3DF04EC146F14FC147F11200A6
:100FA000E8CF24F10CB002D006AA66D011A605D075
:100FB000000111B802D0D89012000B980B960C903B
:100FC00009900201CA6B08BE8A9C06AA51D04084CF
:100FD00024C1CCF21AA610D0FE0E96D815EC23F040
:100FE00001011E6B540E1D6F0201CC052009010189
:100FF0001F6FE2EC3DF00ED0CD0E86D815EC23F03D
:1010000001011E6B540E1D6F0201CC0501011F6F03
:10101000E2EC3DF01DA007D01D9001011C6B240ED9
:101020001B6F15EC23F01DA607D01D9601011C6B4C
:10103000280E1B6F15EC23F01DAA07D01D9A010185
:101040001C6B2C0E1B6F15EC23F01EA007D01E90FE
:1010500001011C6B300E1B6F15EC23F01EA607D090
:101060001E9601011C6B380E1B6F15EC23F040948B
:10107000069A000107989FD711A603D0000111B866
:101080009AD709A007D009900201CA6B000108BED7
:101090008A9C91D716A818D00C800401D8C2E0F41D
:1010A000E16BE03BE13BF00EE117E0510F0BE11388
:1010B000F00EE017000111A604D0010E0001FA6F36
:1010C0007AD724C1FAF077D70101E1A102D0010E4D
:1010D0000FD0E1A302D0020E0BD0E1A502D0030E87
:1010E00007D0E1A702D0040E03D0E1A903D0050E7A
:1010F0000201DF6F020E0201DF03F350DF6F0D828A
:1011000000011A9AD8801200010124251B6F1C6B64
:10111000020E1C23020C01013B6B9C9EA8847C8662
:101120007D6A670EAB6E9C8E9C88A88AA49AA59A4D
:10113000A38A0301CC6B000104908E9C8D9842EC35
:101140004EF01FEC4EF0590E01012F5D020E30598A
:10115000F8E38D8842EC4EF01FEC4EF0650E010175
:101160002F5D000E3059F8E38E8C42EC4EF005D026
:1011700085AE03D0010E3B6F08D01FEC4EF0C50EBC
:1011800001012F5D090E3059F3E33B6702D0D8907F
:101190001200030E306FE80E2F6F77EC40F0F50E63
:1011A00001011D6F4E0E1C6F010E13EC3CF0030E7F
:1011B0000101306FE80E2F6F77EC40F0A8947C9619
:1011C000260EAB6E0401E86BE96BF80E01011D6F92
:1011D000EA0E1C6F010E13EC3CF0130E0101306F90
:1011E000880E2F6F77EC40F0D2E342EC4EF01FEC0C
:1011F0004EF0B90E01012F5D0B0E3059F8E3FF0ED2
:101200001D6FA10E1C6F010E13EC3CF0130E0101BB
:10121000306F880E2F6F77EC40F0B9E3FB0E0101C1
:101220001D6F5E0E1C6F010E13EC3CF0130E0101DE
:10123000306F880E2F6F77EC40F0A9E3000113B8F0
:1012400023D0300EADEC13F03B6F3B510C0A06E09F
:101250003B51360A03E03B512C0A04E1300EADEC61
:1012600013F03B6F3B512C0A03E1000113888FD729
:10127000C2EC39F001013B51DDEC1AF005E240B05F
:101280001388000140A083D7D8801200FB0E1D6F89
:101290002E0E1C6F010E13EC3CF04C0E0101306F52
:1012A000080E2F6F77EC40F00701A6511FE0F40EF7
:1012B00001011D6F3C0E1C6F010E13EC3CF0070E7C
:1012C00001011D6FA60E1C6F000E13EC3CF0F50E15
:1012D00001011D6F340E1C6F000E13EC3CF04C0E20
:1012E0000101306F080E2F6F77EC40F0EE0E010118
:1012F0001D6FD40E1C6F010E13EC3CF00801D2518F
:1013000009E0080E01011D6FD20E1C6F000E13ECD8
:101310003CF008D0060E01011D6FC50E1C6F000EBB
:1013200013EC3CF0FF0E01011D6FEE0E1C6F000E62
:1013300013EC3CF0050E01011D6FF70E1C6F000E43
:1013400013EC3CF0ED0E01011D6F2F0E1C6F000E13
:1013500013EC3CF0080E01012F6F4C0E306F010EA4
:10136000316F000E326B336B7CECA0F00101366FF5
:101370003651080A01E0040C080E4FECE9F07CEC51
:10138000A0F00101366F3651020A0CE03651030A13
:1013900001E1000C36512F0A01E1020C36510C0A12
:1013A000EAE0EAD7080E4FECE9F07CECA0F001018E
:1013B000366F3651390A07E036512F0AEEE03651C2
:1013C0000C0AD9E0EFD7080E4FECE9F07CECA0F066
:1013D0000101366F3651030ADCE036512F0ADDE099
:1013E00036510C0AC8E0EFD70101216B226B0601D0
:1013F000315138EC4CF0236F0601325138EC4CF08F
:10140000246F000E74EC3BF021510001F06F0101DC
:10141000216B226B0601345138EC4CF0236F06012E
:10142000355138EC4CF0246F000E74EC3BF0215138
:101430000001F16F0101216B226B0601375138EC7D
:101440004CF0236F0601385138EC4CF0246F000E3D
:1014500074EC3BF021510001F26FF1C02EF101015B
:10146000D8902E33D8902E33D8902E330001F039F7
:10147000E842F80B01012E110001F06FF2C02EF1CD
:101480000101D8902E330001F139E846E00B01014B
:101490002E110001F16FF241800BF26F0101216BFF
:1014A000226B06012E5138EC4CF0236F06012F51B0
:1014B00038EC4CF0246F000E74EC3BF021512F6F90
:1014C0002F45E846FC0B0001F2130101216B226B52
:1014D00006012B5138EC4CF0236F06012C5138ECEF
:1014E0004CF0246F000E74EC3BF021512F6F2F4114
:1014F000E8423F0B0001F213F36B01012F41E84278
:10150000C00B0001F3130101216B226B060128516E
:1015100038EC4CF0236F0601295138EC4CF0246F65
:10152000000E74EC3BF021512F6FD8902F31000149
:10153000F313F46B01012F41800B0001F411F46FE0
:101540001200E8CF60F1000115B002D0D89012006F
:1015500005C51BF1010160516BEC49F0F7E3050192
:10156000E551070AF3E1310EE525D96EDA6A050E79
:10157000DA22DF6A340E01015B6F050E5C6F5BC11E
:1015800021F15CC122F18EEC24F021C15DF122C178
:101590005EF15DC125F15EC126F1CEEC47F0D6E3E8
:1015A00006BA4ED0000116A82ED0068A07880990E8
:1015B0000201CA6B08BE8A9C408405013251300A80
:1015C00010E1020E01011C6FFE0E1B6F15EC23F0E3
:1015D00001011E6B540E1D6F3F0E1F6FE2EC3DF0BC
:1015E0000FD0020E01011C6FCC0E1B6F15EC23F007
:1015F00001011E6B540E1D6F1F0E1F6FE2EC3DF0BC
:101600000001409410D045EC16F001016039F00B58
:101610005F6F480E466F5F5110EC07F005010551F2
:10162000B6EC4DF002E2D8801200605185EC46F035
:1016300001015F6F5FC154F1605123ECEDF0F3D70E
:101640000B980B960C9009900201CA6B08BE8A9CFD
:10165000069A40841AA610D0020E01011C6FDD0EFE
:101660001B6F15EC23F001011E6B540E1D6F2F0E26
:101670001F6FE2EC3DF00FD0020E01011C6FDD0E7A
:101680001B6F15EC23F001011E6B540E1D6F0F0E26
:101690001F6FE2EC3DF00798B3D71FA463D0000E94
:1016A0000001FE25D96EDA6A0C0EDA22F8C0DFFFDF
:1016B000FE2BFE510201A619A711D8A41200A66B99
:1016C000A76B11D0000E0201A625D96EDA6A0C0EA6
:1016D000DA22000EA625E16EE26A0A0EE222DFCFD0
:1016E000E7FFA64BA72BFEC020F0216A2050020185
:1016F000A65D2150A759E6E30E880001FE6B0001AC
:101700001F941200F851490AD8A412000001FE2BC0
:101710001200F851500AFAE0FE6B1200F851440A28
:10172000FBE10201FF6BC46BC56BF0D7F8513A0ABD
:10173000F3E0F851D00F0201FF6FE8D7F8513A0AF1
:1017400022E0F851D00F0201C46FE0D7F8513A0AF5
:101750001AE0F851D00F0201C56FD8D7F8513A0AF4
:10176000DBE111D00001FE51CDE0010AD2E0030A15
:10177000D5E0010ADBE0070AE1E0010AE7E0030A3D
:10178000D8A41200EBD7FE6B0201A66BA76BC4674F
:1017900006D0C56704D0FFC2A6F2A76B1ED0C567EE
:1017A00008D0FF510A0DC451F324A66F000EF42097
:1017B00013D0FF51640DF3CF20F0F4CF21F0C451CA
:1017C0000A0DF3502024226EF4502120236EC551BF
:1017D0002224A66F000E2320A76FA10EA65D000E87
:1017E000A759D8B0120000011F841200E60EC4EC05
:1017F00029F0010100C10FF101C110F1D451050A16
:1018000008E10F510F0B020A02E1030ED46FF292AE
:101810001200E50EC4EC29F0010100510E6FD45105
:10182000060A22E10C8E0986030E0201B56FE80E4E
:10183000B46F7CD80F510F0BDF6EDA2BDA51100A20
:1018400013E166EC46F008010F1904E1070E0101EF
:10185000D46F04D0070E0101D46F128A0201B56B58
:10186000640EB46F0101DA6BD451090AD8B40FB712
:10187000CED70FA90FBBCBD710A307D0DA6B030EBF
:101880000201B56FE80EB46FC2D70FADC0D7030E1B
:101890000201B56FE80EB46F0C8E48D80EC1DFFFA1
:1018A000DA670FD00EC107F13F0E0717075DAFE2F1
:1018B0000EC1E1F30E513F0B0201ED6F0101DA2B76
:1018C000A6D7EDC207F10101086B020E0727000E33
:1018D0000823DA5107190811F1E10C690D6B0AD0E0
:1018E000000E01010D25D96EDA6A080EDA22DF50EA
:1018F0000C1B0D2BDAC107F1086B072B000E082318
:101900000DC109F10A6B0A51800A0B6F0751095D7D
:101910000851800A0B59E4E30C6703D00C0ED46F16
:1019200001D0128A0101DA6BF2921200000E01015D
:10193000DA25D96EDA6A080EDA22120033C139F1DB
:1019400034C13AF1345133110AE131C11BF132C1D2
:101950001CF195EC3FF01BC139F11CC13AF139C1C2
:101960001BF13AC11CF1DDEC2DF01BC13BF11CC198
:101970003CF120EE02F03B51D9263C51DA22DF50F7
:101980005BEC4CF0366F20EE03F03B51D9263C5116
:10199000DA22DF505BEC4CF0376F20EE04F03B5165
:1019A000D9263C51DA22DF505BEC4CF0386F09A4A9
:1019B00009D0FA0E01011D6F290E1C6F010E13ECE8
:1019C0003CF008D0FA0E01011D6F1E0E1C6F010EB7
:1019D00013EC3CF00101365100EC4CF001013751A1
:1019E00000EC4CF00101385100EC4CF00D0E00EC15
:1019F0004CF042EC4EF00AD018EC4EF007E33EEC0F
:101A00004EF00101356F35513E0A0DE01FEC4EF0EE
:101A1000890E01012F5D130E3059EEE31B0E00EC11
:101A20004CF0D890120031C11CF132C11DF1000EF2
:101A300013EC3CF00301AA6BAB6B02941CD056EC88
:101A4000F1F002A418D002940201CF6701D013D0A4
:101A5000080E0101226FA00E216FFD0E246F6B0E88
:101A6000236F266B070E256FEBEC2FF0225121110F
:101A700002E1D8801200310E0301AA5D750EAB5948
:101A8000DEE31B0E00EC4CF0CCD701014D6B03AA3A
:101A900096D0039A880E01012F6F130E306F316BB1
:101AA000326B010E336F7CECA0F00101516F51518C
:101AB000370A03E051510C0AEDE15151370A70E148
:101AC00006017B51220A6CE10501306B0101516B6B
:101AD0007C0E01015125D96EDA6A0601060EDA2262
:101AE000220EDF6201D016D07C0E01015125D96E85
:101AF000DA6A060EDA22200E5125E16EE26A05014D
:101B0000050EE222DFCFE7FF302B0101512B0F0E34
:101B10005165DED772ECE7F0506F505141E0050E91
:101B200050613ED0500504E1020E4F6F520E11D0AD
:101B30005051020A04E1020E4F6F630E0AD0505159
:101B4000030A04E1020E4F6F740E03D0020E4F6FB2
:101B5000850E4E6F0501E56B0101516B310E0101E0
:101B60005125D96EDA6A050EDA2251514E251E6FC3
:101B7000000E4F211F6FF6EC37F0DF6E310E0101C2
:101B80005125D96EDA6A0501050EDA22DF5006E02A
:101B9000E52B0101512B100E5165E0D750C14DF1DD
:101BA000FF0E01011D6FE50E1C6F010E13EC3CF0E2
:101BB000130E0101306F880E2F6F77EC40F001019A
:101BC0004D51120020EE04F02451D9262551DA227D
:101BD00010EE06F02451E1262551E222DFCFE7FF87
:101BE00020EE03F02451D9262551DA2210EE05F01B
:101BF0002451E1262551E222DFCFE7FF20EE02F05B
:101C00002451D9262551DA2210EE04F069D810EEBD
:101C100003F066D8CA51DF6E20EE02F02451D926B7
:101C20002551DA22C9C1DFFF20EE05F02451D92663
:101C30002551DA22DF50276F266B286B0F0E2715F0
:101C4000296F20EE06F02451D9262551DA22DF50E3
:101C500028112A6F29512B6F2AC11BF12BC11CF1AE
:101C6000DDEC2DF01BC12CF11CC12DF120EE06F096
:101C70002451D9262551DA22DF6A20EE06F02451BC
:101C8000D9262551DA2210EE04F02C51E1262D51EF
:101C9000E222E750266F10EE03F02C51E1262D5181
:101CA000E222E750276F2739F00B2611DF6E20EE76
:101CB00005F02451D9262551DA22F00EDF1620EE48
:101CC00002F02C51D9262D51DA22DF50266F20EE5A
:101CD00005F02451D9262551DA222651DF121200AF
:101CE0002451E1262551E222DFCFE7FF20EE01F06B
:101CF0002451D9262551DA221200010E60ECE0F0C1
:101D000004E2010E60ECE0F014E3486B0AD0436B90
:101D10006AD8200E0101482583D8E2EC3DF001018C
:101D2000482B6CD8F4E3436B5ED8000E1F6BE2ECDB
:101D30003DF0020E60ECE0F004E2020E60ECE0F038
:101D400016E3486B0BD0110E436F4DD8200E0101E6
:101D5000482566D8E2EC3DF00101482B4FD8F3E36B
:101D6000110E436F40D8000E1F6BE2EC3DF0030EE6
:101D700060ECE0F004E2030E60ECE0F016E3486B88
:101D80000BD0220E436F2FD8200E0101482548D8D2
:101D9000E2EC3DF00101482B31D8F3E3220E436F12
:101DA00022D8000E1F6BE2EC3DF0040E60ECE0F078
:101DB00005E2040E60ECE0F0D8A01200486B0BD0F6
:101DC000330E436F10D8200E0101482529D8E2ECCC
:101DD0003DF00101482B12D8F3E3330E436F03D8D3
:101DE0001F6BE2EF3DF0010E446F435148251D6F1C
:101DF000000E48BFFF0E44211E6F120030C543F194
:101E00000101446B48C145F1466B45BF4607465149
:101E1000800A476F4351455D4451800A475912007B
:101E2000D96EDA6A050EDA22DF501F6F1200E8CF92
:101E30003DF1000111AC000C11AC1200130E0101B8
:101E40001F6F6A0E1E6FF6EC37F03E6F3E51800A30
:101E5000500F04E33E51800A460F03E33D5167EC07
:101E60003AF019EC29F004E319EC29F001E3020C33
:101E700001013E6B280E01013E25D96EDA6A06018A
:101E8000060EDA22DF506CE001013D6733D0370ED9
:101E90003E25D96EDA6A060EDA226A0E396F130E03
:101EA0003A6F39513E251E6F000E3EBFFF0E3A219C
:101EB0001F6FF6EC37F0DF6E280E01013E25D96E5C
:101EC000DA6A060EDA22DF50396F3A6B39BF3A0709
:101ED0006A0E3B6F130E3C6F3B513E251E6F000E8A
:101EE0003EBFFF0E3C211F6FF6EC37F039193A1157
:101EF000BEE131D0370E01013E25D96EDA6A060EF9
:101F0000DA22790E396F130E3A6F39513E251E6F62
:101F1000000E3EBFFF0E3A211F6FF6EC37F0DF6E6A
:101F2000280E01013E25D96EDA6A060EDA22DF504C
:101F3000396F3A6B39BF3A07790E3B6F130E3C6F1E
:101F40003B513E251E6F000E3EBFFF0E3C211F6F12
:101F5000F6EC37F0CBD73E2B3E51800A710F8AE367
:101F6000010CA192F60E7B6E3C0E7A260101D3671E
:101F700001D03C0C010ED307D8A4010C000110AA1B
:101F8000010C10B60AD011A011800101D06B10987D
:101F9000109E00011194F19C120011A075D011A4A3
:101FA00002D0119471D00101D02B81A402D0D8901D
:101FB00001D0D8800301EA370301EB370301EC3786
:101FC0000301ED370301EE370301EF370301F0376B
:101FD0000301F1370301F2370301F3370101D05157
:101FE000070B04E10301EA510101CE2710A827D015
:101FF00010AC04D00101D051500A06E010BC44D00E
:102000000101D051400A40E111840301EA5101016C
:10201000CE5F0301EA510101CE630ED009B20CD0AC
:102020000301030E226EEA0E216EECEC24F0010196
:10203000D06B8F80148628D00101D06B09D010AEF0
:1020400009D00101D0512A0A03E0D0512B0A1CE12A
:10205000F18C1AD00101D051080A16E1EAC3CEF181
:1020600011840301EA51110A02E1108E1B8410ACA5
:1020700004D00301EA51EB0A06E010BC05D00301CD
:10208000EA51A50A01E11088140E0101D36F000185
:102090001096140C960EF66EEB0EF76E000EF86EA0
:1020A00021EE32F0060E0900F5CFDEFFE82EFBD759
:1020B000070E3C6F3CC12EF1F90E2E27320E2E2555
:1020C000D96EDA6A010EDA22DF502F6F73D82F191A
:1020D00002E0D89012003C2B0B0E3C65EBD7030EB0
:1020E0002A252E6F000E2B212F6F2EC121F12FC11B
:1020F00022F18EEC24F021C13AF122C13BF1386B80
:10210000396B070E3C6F0DD038C11BF139C11CF182
:1021100051D81D6F3CEC48F01BC138F11CC139F19E
:102120003C2B070E3A252E6F000E3B212F6F3CC132
:1021300030F1316B2E51305D2F513159E5E320EEF6
:1021400002F02A51D9262B51DA22DF502E6F2F6B45
:102150002EBF2F0720EE01F02A51D9262B51DA226B
:10216000DF50316F306B2E5130113A6F2F513111DA
:102170003B6F3B51391902E13A513819AAE10C0E73
:102180002A252E6F000E2B212F6F2EC121F12FC17A
:1021900022F1C8EC20F021C13AF122C13BF13B51C0
:1021A0000401E71904E101013A510401E61991E142
:1021B000D88012003C512A25D96E000E2B21DA6EF0
:1021C000DF501200E8CF44F1456B466B050120510A
:1021D0002B0A15E1010E0101466F11D0200E0101FD
:1021E0004625D96EDA6A050EDA222E0E4525E16EF5
:1021F000E26A010EE222DFCFE7FF462B452B050105
:1022000030510101465DEAE32E0E4525D96EDA6AAA
:10221000010EDA22DF6A1C6F2E0E1B6F95EC3FF069
:102220001B51456F45C123F1246B266B020E256FB0
:102230001FEC44F023C140F124C141F125C142F11A
:1022400026C143F14151800A800F010ED8B4405D90
:102250000AE3010E1C6F2E0E1B6FFB0E1E6FEC0EA1
:102260001D6F87EC43F0466B2CD046C12BF12B2B16
:102270002E0E2B25D96EDA6A010EDA22310E2C6F62
:10228000050E2D6F46512C27000E2D2344512C2571
:10229000E16E000E2D21E26EDFCFE7FF2E0E462508
:1022A000D96EDA6A010EDA2218D82B27000E2C23F9
:1022B0002B29E16E000E2C21E26EDFCFE7FF020E2C
:1022C00046274551465DD1E308D82B25D96E000E2F
:1022D0002C21DA6E000EDF6E000C310E2B6F050E16
:1022E0002C6F46512B27000E2C23445112006450B2
:1022F0002FE104010031E8320F0B0D0A0FE104BF9A
:10230000046B0401BF6B0401C06B0401C56BC46B9B
:10231000A1EC2FF077EC2EF090EF2DF00401C051DE
:10232000020A44E1070E0401CB6F040EC86F280EA9
:10233000C76F040ECA6FCE0EC96F3EEC45F0010E9A
:102340000401D56F040E0401036F200E026F12000A
:102350006450040AD8A412000401CD51080A0AE10D
:1023600022C45EFF040ECD6F0F015E5103E0100E1C
:102370000401CD6F0401C00519E1040E0401076FCB
:10238000280E066FC0EC2AF00401BF51020A04E1D6
:10239000840E0401046F840C040104BD03D0C80E34
:1023A000046FC80C880E0401046F880C0401C16B13
:1023B0000401C051020AD8B465A81CD0040101511F
:1023C000080A18E10031E8320F0B0D0A13E100BFD3
:1023D00011D0040E036F200E026F040E0401C86FAB
:1023E000280EC76F040ECA6F200EC96F080ECB6F80
:1023F0005AEF45F00401C06B080E0401016F040E92
:10240000036F200E026F8C0E006F046B120064507D
:102410002FE104010031E8320F0B0D0A0FE104BF78
:10242000046B0401BF6B0401C06B0401C56BC46B7A
:102430000DEC2FF0C2EC2EF043EF2DF00401C05153
:10244000020A44E1070E0401CB6F040EC86F280E88
:10245000C76F040ECA6FCE0EC96F1CEC45F0010E9B
:102460000401D56F040E0401036F200E026F1200E9
:102470006450040AD8A412000401CD51080A0AE1EC
:1024800022C45EFF040ECD6F0F015E5103E0100EFB
:102490000401CD6F0401C00519E1040E0401076FAA
:1024A000280E066F64EC2BF00401BF51020A04E110
:1024B000840E0401046F840C040104BD03D0C80E13
:1024C000046FC80C880E0401046F880C0401C16BF2
:1024D0000401C051020AD8B465A81CD004010151FE
:1024E000080A18E10031E8320F0B0D0A13E100BFB2
:1024F00011D0040E036F200E026F040E0401C86F8A
:10250000280EC76F040ECA6F200EC96F080ECB6F5E
:1025100038EF45F00401C06B080E0401016F040E92
:10252000036F200E026F8C0E006F046B120035C11A
:102530007CF136C17DF1510E816F806B37051CE156
:102540001F6B750E1E6FF6EC37F07E6F7E51080B19
:102550007B6F7B5167E0510E1F6F750E1E6FF6EC9F
:1025600037F07E6F7E87510E1E6F750E1D6F7EC118
:102570001FF1E2EC3DF056D01F6B750E1E6FF6ECAE
:1025800037F0E3D7C00E7C25386FFF0E7D21396F01
:102590003951800A800F010ED8B4385D20E37F6B7B
:1025A00047D8F6EC37F0DF6E804B812B7F2B3F0E48
:1025B0007F65F6D733C12CF134C12DF1010E2F6F99
:1025C0003B0E2E6F400E306FA4EC45F0400E3327CB
:1025D000000E3423C00E7C27FF0E7D2323D07F6B9B
:1025E00007D026D8F6EC37F0DF6E804B812B7F2B9F
:1025F0007FC138F1396B3951800A3A6F7C51385DAF
:102600007D51800A3A59EDE333C12CF134C12DF1EB
:10261000010E2F6F3B0E2E6F7CC130F1A4EC45F004
:102620007C6B7D6B01017D517C11D8B41200AAD75F
:102630003B0E7F25D96EDA6A010EDA2280C11EF1C7
:1026400081C11FF11200E8CF29F1C239E8461F0B02
:102650001B6F1C6BDDEC2DF01BC127F11CC128F199
:102660005BD862D85BEC4CF0DF6E292B55D864D870
:102670005BEC4CF0DF6E292B4FD83A0EDF6E292B26
:10268000C339E842070BC2C125F1266BD890253724
:102690002637D8902537263757D8DDEC2DF01BC1CB
:1026A00027F11CC128F138D83FD85BEC4CF0DF6E25
:1026B000292B32D841D85BEC4CF0DF6E292B2CD87B
:1026C0003A0EDF6E292BC445010BC3C125F1266BE1
:1026D0003BD8DDEC2DF01BC127F11CC128F11CD823
:1026E00023D85BEC4CF0DF6E292B16D825D85BEC99
:1026F0004CF0DF6E292B245104E00ED8200EDF6E43
:10270000292B310E01012925D96EDA6A0501050E42
:10271000DA22000EDF6E000C310E01012925D96E80
:10272000DA6A050EDA22120010EE03F02751E126D4
:102730002851E222E750120010EE04F02751E12662
:102740002851E222E7501200D8902537263725136A
:102750003F0E25151B6F1C6B000CE8CF36F10101F5
:10276000386BFD0E1D6F530E1C6F010E13EC3CF009
:10277000880E01012F6F130E306F000E316B326B1C
:10278000336B7CECA0F001013A6F3A51080A02E188
:10279000010E386F3A51360A17E03A51280A14E010
:1027A0003A51290A11E03A510C0A0EE03A512C0A2A
:1027B0000BE0880E2F6F130E306F316B326B010EF2
:1027C000336F7CECA0F0DFD73A510C0A08E03805F3
:1027D00006E0130E306F880E2F6F77EC40F001018A
:1027E000396BFD0E1D6F5B0E1C6F010E13EC3CF080
:1027F000880E01012F6F130E306F000E316B326B9C
:10280000336B7CECA0F00101376F130E306F880E34
:102810002F6F77EC40F001013751380A0EE042EC9F
:102820004EF01FEC4EF0D10E01012F5D070E305916
:10283000F8E3392B020E3965D4D73951030A02E186
:102840000C0E3A6F42EC4EF01FEC4EF0B90E010147
:102850002F5D0B0E3059F8E319963651310A01E11C
:10286000198601013A511200E8CF5AF100010DB862
:1028700002D0D890120057C61BF101015A516BECDF
:1028800049F0F7E3050125EEE5F0020EDF64F1D72C
:1028900025EEE5F0050EDF6401D0EBD700010DA8B1
:1028A000E8D7020E0101596F0ED0310E01015925F2
:1028B0005AD8500FDEE3310E0101592554D8460F86
:1028C000D8E20101592B0501E5510101595DEDE304
:1028D0000501310EE525D96EDA6A050EDA22DF6AC6
:1028E000330E0101546F050E556F54C121F155C1CE
:1028F00022F1C8EC20F021C157F122C158F1000E9D
:10290000575D010E5859B5E28A8E57C1F2F458C18D
:10291000F3F40001148C45EC16F001015A39F00B68
:10292000566F080E466F565110EC07F046C157F12E
:1029300047C158F106015751B6EC4DF002E2D8807C
:1029400012005A5185EC46F00101566F57C13FF114
:1029500058C140F15AC141F156C142F1030E436FD3
:1029600016EC3DF0ECD7D96EDA6A0501050EDA22D5
:10297000DF50800A120000010E9842EC4EF059D050
:1029800045EC0DF00301E66F00010EA852D00A01DC
:102990000051300A01E1010C0051310A03E00051FD
:1029A000320A47E1010E0101556F546B0AD060D81D
:1029B0003A0EDF6204D0550755C154F105D001012C
:1029C000552B56D8DF50F3E10101546701D0020CBA
:1029D000556B13D0B60E01015525D96EDA6A070E74
:1029E000DA22DF50526F010E5525D96EDA6A0A0ECF
:1029F000DA22DF50521904E1552B5451555DEAE3B8
:102A000055515419E4E1556B06D023D8310E01011C
:102A1000552518D8552B1DD8DF50F7E155C1E5F5E0
:102A20000A010051310A01E1030C0051320A01E1AF
:102A3000040C1FEC4EF0E90E01012F5DFD0E305924
:102A40009FE3000CE16EE26A050EE222DFCFE7FFB2
:102A50001200020E526F0A0E536F54515227000E8D
:102A6000532355515225D96E000E5321DA6E1200B0
:102A7000000E01015525D96EDA6A0A0EDA2212001B
:102A8000E8CF60F1000115B002D0D890120005C562
:102A90001BF1010160516BEC49F0F7E30501E551D1
:102AA000070AF3E1310EE525D96EDA6A050EDA225E
:102AB000DF6A340E01015B6F050E5C6F5BC121F1B3
:102AC0005CC122F18EEC24F021C15DF122C15EF1E6
:102AD0005DC125F15EC126F1CEEC47F0D6E30001E1
:102AE00016A835D0068A1A9605013251300A02E13D
:102AF0001A8601D0078809900201CA6B08BE8A9C19
:102B0000408405013251300A10E1020E01011C6FB0
:102B1000FE0E1B6F15EC23F001011E6B540E1D6F92
:102B20003F0E1F6FE2EC3DF00FD0020E01011C6F53
:102B3000CC0E1B6F15EC23F001011E6B540E1D6FA4
:102B40001F0E1F6FE2EC3DF00001409410D045ECE9
:102B500016F001016039F00B5F6F480E466F5F5150
:102B600010EC07F005010551B6EC4DF002E2D880FB
:102B70001200605185EC46F001015F6F5FC154F1B6
:102B8000605123ECEDF0F3D7E8CF5AF100010DB618
:102B900002D0D890120054C61BF101015A516BECBF
:102BA00049F0F7E300010DA6F4D7050125EEE5F0A5
:102BB000020EDF64EED725EEE5F0050EDF6401D0EE
:102BC000E8D7020E0101596F10D0310E01015925CD
:102BD000B3EC14F0500FDDE3310E01015925B3ECD5
:102BE00014F0460FD6E20101592B0501E551010110
:102BF000595DEBE30501310EE525D96EDA6A050E64
:102C0000DA22DF6A330E0101546F050E556F54C18D
:102C100021F155C122F1C8EC20F021C157F122C1A8
:102C200058F1000E575D010E5859B3E28A8C57C116
:102C3000D8F458C1D9F40001068645EC16F001011C
:102C40005A39F00B566F050E466F565110EC07F0CF
:102C500046C157F147C158F106015451B6EC4DF049
:102C600002E2D88012005A5185EC46F00101566FFD
:102C700057C13FF158C140F15AC141F156C142F12B
:102C8000030E436F16EC3DF0ECD7CA0EF66EEA0E5B
:102C9000F76E000EF86E21EE36F0120E0900F5CF39
:102CA000DEFFE82EFBD7030E0101496F39D0FC0E81
:102CB0001D6FEB0E1C6F010E13EC3CF0D00E0101EA
:102CC0002F6F070E306F000E316B326B336B7CEC65
:102CD000A0F00101486F4851270A22E1070E496F11
:102CE000750E01014925D96EDA6A060EDA22210E27
:102CF0004925E16EE26A060EE222DFCFE7FF492BAB
:102D00004951800A680FECE3210E4925D96EDA6A31
:102D1000060EDA22DF6AD00E26D87CECA0F004D0B2
:102D2000490701014929C3E1010149671200486BC4
:102D30000BD021D8280E01014825E16EE26A060E6B
:102D4000E222DFCFE7FF482B16D8DF50F2E1482B15
:102D5000280E01014825D96EDA6A0601060EDA222C
:102D6000000EDF6E000C2F6F070E306F316B326B71
:102D7000010E336F010C360E4825D96EDA6A010E4A
:102D8000DA221200040122050EE120511F0B0BE193
:102D90000401C48F0401C66B04012151030A03E13D
:102DA000010E0401C66F04012267120020511F0B9F
:102DB000020AD8A4120024510F0BD8B41200040147
:102DC000C48FB3EC4BF0C7C4F6FFC8C4F7FF000EC6
:102DD000F86E0F0EF76404D0840EF56E0C0006D06A
:102DE000F6CFE9FFF7CFEAFF840EEF6E0401215121
:102DF000030AD8B4120024510F0B0101006F4C0ECE
:102E0000016F0F0E026F00510127E86A00BFE868EA
:102E1000022301C1D9FF02C1DAFFFE0EDE16000E49
:102E2000DD16C7C4F6FFC8C4F7FF000EF86E0F0E1C
:102E3000F76404D0C80EF56E0C0006D0F6CFE9FF9B
:102E4000F7CFEAFFC80EEF6E040124AF1200C7C42B
:102E5000F6FF0401C8C4F7FF000EF86E0F0EF7640A
:102E600004D0400EF56E0C0006D0F6CFE9FFF7CF88
:102E7000EAFF400EEF6E12000301C22BFC0E0101AF
:102E80001D6FB30E1C6F010E13EC3CF0880E010198
:102E90002F6F130E306F000E316B326B336B7CEC87
:102EA000A0F00101366F3651160A03E03651170AB9
:102EB00011E119B607D018AA0BD0189A13AA188CCA
:102EC0000E9E06D019A204D0199213A81984F8D71F
:102ED000048027D03651180A09E03651190A06E055
:102EE00036511A0A03E036511B0A0DE10001049025
:102EF00042EC4EF01FEC4EF0210E01012F5D4E0E04
:102F000030590FE2F7D736510C0A0BE0880E2F6FBD
:102F1000130E306F316B326B010E336F7CECA0F00F
:102F2000C0D7010136510C0A06E0130E306F880E2F
:102F30002F6F77EC40F0010136511B0A0CE036513F
:102F40001A0A09E03651190A06E03651180A03E058
:102F50000301C26B07D0020E0301C26503D0C26B2E
:102F6000D8901200D8801200216B000E06EC48F0B9
:102F7000226F1FC11BF120C11CF122C11DF118ECF1
:102F800033F002E301012181040E06EC48F0226FC8
:102F90001FC11BF120C11CF122C11DF1D7EC32F081
:102FA00002E301012183080E06EC48F0226F1FC1E5
:102FB0001BF120C11CF122C11DF19AEC33F002E398
:102FC000010121850C0E06EC48F0226F1FC11BF198
:102FD00020C11CF122C11DF155EC32F002E30101C8
:102FE0002187100E06EC48F0226F1FC11BF120C193
:102FF0001CF122C11DF196EC32F002E3010121899E
:103000001C0E06EC48F0226F22C1D9F12B0E226172
:1030100003D01F9C1F8E14D06E0E226504D0A00E0C
:10302000226101D0F6D72A0E226505D06F0E2261EB
:1030300002D01F8C04D09F0E226502D01F9C1F9EC1
:103040001FAC02D00101218F1FAE02D00101218DE2
:103050000101215112002E0E01011C6FE00E1B6FA9
:1030600001D0040068D8D8B41C29FBE19B8CEA0E7F
:103070001C6F600E1B6F01D004005DD8D8B41C29F2
:10308000FBE1F26AF06A9D6AA06ABB6AB66AC66A28
:10309000AC6AC26A060EC16EC088C16AF80EC26E02
:1030A000C098896A8C6A2F0E926E4F0E956E868E2E
:1030B0008A6A8D6A050E936E020E966EF19E8B6A79
:1030C0008E6AD40E946EBC0E976E8B828F6A656A80
:1030D000140E986ED56A810ECD6ED10ECF6E200E75
:1030E000CE6E9E909F909D80810E796EF60E7B6EC7
:1030F0003C0E7A6EA192A292A082C088020ECE6E81
:10310000C098D0B805D0A80E0301AD6FC00E04D092
:10311000020E0301AD6FD00EAC6F0C98750E01015D
:103120001C6F300E1B6F01D0040005D8D8B41C29C9
:10313000D8B41200F9D701011B07D8A01C071B291E
:1031400012000001F8510A0A10E016BC0ED0000E61
:10315000FE25D96EDA6A0C0EDA22F8C0DFFFFE2BEC
:10316000A00EFE65A00CFE6B12000001F8510A0AC9
:103170002FE116BC2DD0000EFE25D96EDA6A0C0E9A
:10318000DA22DF6AFE6B0C010C0E216E000E206E3F
:10319000EE0E236EFB0E226E256A110E246EC4EC19
:1031A00030F02150201014E10001168C110E2F6E0A
:1031B0000C0E306E2FC026F030C027F0F2EC21F05C
:1031C000FF0E262405010E6FFF0E27200F6F120041
:1031D000000116AC120005010F510E1104E00E079C
:1031E000D8A00F0701D0169C0001F8510A0A0FE180
:1031F0000201DB07000EDB25D96EDA6A0A0EDA223D
:10320000000EDF6A0E88DBC2E3F2DB6B1200F851BE
:103210000A0AD8B41200000E0201DB25D96EDA6A60
:103220000A0EDA22F8C0DFFFDB2B1200049230C551
:1032300049F1050120512B0A03E1010149070482EC
:10324000050E0101286F310E276FFE0E2A6F4C0EFE
:10325000296F66ECD5F027514A6F4AC14BF151D81E
:1032600049390F0B5BEC4CF0DF6E4B2B4AD84951C0
:103270000F0B5BEC4CF0DF6E4B2B04A209D0310E30
:1032800039D8FF0E2A6FF10E296F66ECD5F008D001
:10329000310E30D8FF0E2A6FF40E296F66ECD5F090
:1032A00027514A6F4A514B274B51E2EC10F0310E37
:1032B000476F050E486F47C11BF148C11CF195ECE3
:1032C0003FF01B514B6F310E15D8FF0E2A6F980E31
:1032D000296F66ECD5F027514A6F4A514B27310EC2
:1032E00001014B25D96EDA6A0501050EDA22000EBE
:1032F000DF6E000C01014B25276F286B050E28237C
:103300001200310E01014B25D96EDA6A050EDA2260
:1033100012004D0E0201006FA36B5ED8DF501BE15F
:10332000A3C23DF101013D2B5FD80D0EDF6EA3C29C
:103330003DF1020E3D2758D80A0EDF6EA3C23DF1C3
:10334000030E3D27000E3D25D96EDA6A0201020EFA
:10335000DA22DF6A12D040D8A3C23DF101013D2B31
:10336000000E3D25E16EE26A0201020EE222DFCF8D
:10337000E7FFA32B9F0EA365D0D79F0EA36505D0B3
:103380000D0EA06F0A0EA16FA26B020E0101326F2B
:10339000000E316F000E346B336B9EEC0CF002E2CA
:1033A000D89012001A9C00010E9842EC4EF00BD0FF
:1033B00000010EA808D00A010051300A02E1D880AD
:1033C000120000010E981FEC4EF0E90E01012F5D76
:1033D000FD0E3059E5E2ECD7310E0201A325D96E7E
:1033E000DA6A050EDA221200000E3D25D96EDA6A7D
:1033F000020EDA221200190E256E280EC26EC2804D
:1034000025062528FDE1C282320E256E25062528D7
:1034100002E0C2B2FBD7C4CF26F0630E26600CD008
:103420000301BB6BBA2B3B0EBA6506D0BA6BB9670A
:1034300003D0010EB96F1A80EC0E0201D125206E67
:10344000216AFF0E212226C022F0236A2350800A1F
:10345000246E2050225C2150800A24580BE3030183
:10346000BA6BBB2B3B0EBB6505D0BB6B1AB0FF0024
:10347000B96B1A90C26A280E266007D00301B52BDB
:10348000020EB565020CFF00020C0301B851265C68
:103490000FE3B66BB56BB72B770EB765770CB76BD1
:1034A000079C079A000108A21200088008921200E7
:1034B00026500201D15DD8A012000301B76BB56B95
:1034C000B62B3B0EB6653B0CB66B078C0882000131
:1034D00007BA1200078E078A1200E8CF9FF2010E8A
:1034E0000201A16F9F5102E0030EA16F0101216B48
:1034F000226B060E0201A125D96EDA6A0501050EBE
:10350000DA22DF5038EC4CF0236F050E0201A125C2
:10351000D96EDA6A0501050EDA22DF5038EC4CF07C
:10352000246F000E74EC3BF021510201A06F9F67E5
:1035300002D0039003D09F0501E1039202019E6B2C
:10354000A051C5EC04F011E300011C9672ECE7F009
:103550000201A16FA151800A7A0F07E2A151FFEC8D
:10356000CCF003E3010E02019E6F02019E6721D0A1
:10357000FB0E01011D6F8B0E1C6F010E13EC3CF056
:10358000130E0101306F880E2F6F77EC40F00201AF
:10359000A051C5EC04F00DE300011C9672ECE7F0BD
:1035A0000201A16FA151800A7A0F03E2A151FFEC41
:1035B000CCF00201A05167EF27F0E8CF36F1365189
:1035C000360A06E036512C0A03E036510C0A02E1B5
:1035D000D89012003651290A5EE11F6B5C0E1E6FF7
:1035E000F6EC37F0336F1F6B5B0E1E6FF6EC37F0A7
:1035F000356F3351346FFC0E1D6FCB0E1C6F010EF7
:1036000013EC3CF034C11BF135C11CF1DDEC2DF0A5
:103610001BC137F11CC138F120EE01F03751D9261A
:103620003851DA22DF505BEC4CF000EC4CF0010139
:1036300020EE02F03751D9263851DA22DF505BEC08
:103640004CF000EC4CF0010120EE03F03751D9268C
:103650003851DA22DF505BEC4CF000EC4CF0010109
:1036600020EE04F03751D9263851DA22DF505BECD6
:103670004CF000EC4CF0F10E01011D6F430E1C6F7D
:10368000000E13EC3CF0130E0101306F880E2F6F0B
:1036900077EC40F09DE3D8801200040122050EE192
:1036A00020511F0B0BE10401C48F0401C66B040100
:1036B0002151030A03E1010E0401C66F04012267D0
:1036C000120020511F0B020AD8A4120024510F0B24
:1036D000D8B412000401C48F8BEC4BF045EC31F0F0
:1036E000F76404D0840EF56E0C0006D0F6CFE9FF27
:1036F000F7CFEAFF840EEF6E04012151030AD8B41C
:10370000120024510F0B01011B6F4C0E1C6F0F0E8A
:103710001D6F1B511C27E86A1BBFE8681D231CC1D5
:10372000D9FF1DC1DAFFFE0EDE16000EDD1645ECD8
:1037300031F0F76404D0C80EF56E0C0006D0F6CF59
:10374000E9FFF7CFEAFFC80EEF6E040124AF1200C5
:10375000C7C4F6FF0401C8C4F7FF000EF86E0F0ED1
:10376000F76404D0400EF56E0C0006D0F6CFE9FFEA
:10377000F7CFEAFF400EEF6E1200E8CF1FF186860A
:103780000201CB6B3A0EDAEC4BF03A0E03EC4EF042
:1037900001011D6702D00F0E1D6F1E051DE11D5199
:1037A000F00B0CE01D390F0B5BEC4CF0206F20513F
:1037B000DAEC4BF00101205103EC4EF001011D51F8
:1037C0000F0B5BEC4CF0206F2051DAEC4BF0010159
:1037D000205103EC4EF00DD01D510F0B5BEC4CF063
:1037E0000301B26FB251DAEC4BF00301B25103ECBA
:1037F0004EF001011F51DAEC4BF001011F5103ECB7
:103800004EF001011C51DAEC4BF001011C5103ECAC
:103810004EF0CB390F0B5BEC4CF0DAEC4BF00201C5
:10382000CB510F0B5BEC4CF0DAEC4BF00D0EDAECFD
:103830004BF00A0EDAEC4BF00301A86BA96B000EFB
:10384000A76F0A0EA66F00011E9CADB203D0000147
:103850001EACFBD786961200266A000E23EC49F0B8
:10386000276E24C020F025C021F027C022F05BEC99
:1038700034F0D8B02680040E23EC49F0276E24C023
:1038800020F025C021F027C022F09AEC34F0D8B007
:103890002682080E23EC49F0276E24C020F025C0B4
:1038A00021F027C022F0D9EC34F0D8B026840C0ED9
:1038B00023EC49F0276E24C020F025C021F027C05A
:1038C00022F057EC35F0D8B02686100E23EC49F0E4
:1038D000276E24C020F025C021F027C022F018EC6C
:1038E00035F0D8B026881C0E23EC49F0276E27C08F
:1038F000D9F12B0E276003D01F9C1F8E14D06E0EA3
:10390000276404D0A00E276001D0F6D72A0E2764C2
:1039100005D06F0E276002D01F8C04D09F0E276445
:1039200002D01F9C1F9E1FBC268E00011FBE268C2E
:1039300026501200E8CF29F1DC07DC51220DF90EE8
:10394000F3242F6F3F0EF420306F2FC11EF130C1D2
:103950001FF1F6EC37F02D6F2E6BD8902D35256FBB
:103960002E35266F29512525316F000E2621326F05
:1039700031C12AF13107D8A03207D8902D35256FF3
:103980002E35266FDC51220D2551F324276F265149
:10399000F420286FF90E27252F6F3F0E2821306F56
:1039A0002ED02FC11EF130C11FF1F6EC37F0256F7C
:1039B000FF0E2F251E6FFF0E30211F6FF6EC37F024
:1039C0002C6F25512B6F300E01013125D96EDA6A2B
:1039D000050EDA222C51DF6E310E3125D96EDA6AEE
:1039E000050EDA222BC1DFFF2D07D8A02E07FE0E11
:1039F0003127FF0E3223020E2F5F000E305B2E5157
:103A0000800A800F010ED8B42D5DCBE22A5112003E
:103A10000301ED5138EC4CF01C6F0301EC5138EC14
:103A20004CF01D6F1D39F00B1C110301EA6F05AE40
:103A30001DD0EF5138EC4CF01C6F0301EE5138EC07
:103A40004CF01D6F1D39F00B1C110301EB6FF15190
:103A500038EC4CF01C6F0301F05138EC4CF01D6F4A
:103A60001D39F00B1C110301EC6F06D00101CA5186
:103A70000301EB6FC9C1ECF3F35138EC4CF01C6F50
:103A80000301F25138EC4CF01D6F1D39F00B1C1185
:103A90000301ED6FF55138EC4CF01C6F0301F4514C
:103AA00038EC4CF01D6F1D39F00B1C110301EE6F4B
:103AB000F75138EC4CF01C6F0301F65138EC4CF028
:103AC0001D6F1D39F00B1C110301EF6FF95138EC1C
:103AD0004CF01C6F0301F85138EC4CF01D6F1D3990
:103AE000F00B1C110301F06FF16B1200E8CF5AF1DB
:103AF0006EC61BF101015A516BEC49F002E2D890FD
:103B000012000501E5510B0AFAE138C556F1386B90
:103B1000340E0101546F050E556F54C121F155C18A
:103B200022F18EEC24F021C158F122C159F158C183
:103B300025F159C126F1CEEC47F0E1E356C138F545
:103B40000501310EE525D96EDA6A050EDA22DF6A43
:103B5000380E0101546F050E556F54C121F155C146
:103B600022F18EEC24F021C158F122C159F158C143
:103B700024F159C125F16CEC4CF001015A39F00BDC
:103B8000576F300E466F575110EC07F046C158F191
:103B900047C159F106016E51B6EC4DF002E2D880F2
:103BA00012005A5185EC46F00101576F58C13FF1A0
:103BB00059C140F15AC141F157C142F1030E436F5F
:103BC00016EC3DF0ECD7E8CF5AF16EC61BF10101BF
:103BD0005A516BEC49F002E2D89012000501E55110
:103BE0000B0AFAE138C556F1386B340E0101546FF7
:103BF000050E556F54C121F155C122F18EEC24F010
:103C000021C158F122C159F158C125F159C126F1FC
:103C1000CEEC47F0E1E356C138F50501310EE5255C
:103C2000D96EDA6A050EDA22DF6A380E0101546FA6
:103C3000050E556F54C121F155C122F18EEC24F0CF
:103C400021C158F122C159F158C124F159C125F1BE
:103C5000EDEC4BF001015A39F00B576F300E466F07
:103C6000575110EC07F046C158F147C159F1060110
:103C70006E51B6EC4DF002E2D88012005A5185EC3C
:103C800046F00101576F58C13FF159C140F15AC187
:103C900041F157C142F1030E436F16EC3DF0ECD7F2
:103CA0000201B66BB76BB86BB96B0101086B2AD018
:103CB00008510025D96E000E0121DA6EDF50020195
:103CC000B627000EB723B65D010EB75903E3B64B16
:103CD000B72BB76BB629B71102E1B66BB76BB6510C
:103CE000B827B751B923000EB85D010EB95903E3E7
:103CF000B84BB92BB96BB829B91102E1B86BB96BE4
:103D00000101082BFE0E0225036F046BFF0E042336
:103D100008C105F1066B0651800A076F0351055D66
:103D20000451800A0759C4E302511ED8FE0E12D86E
:103D3000B65D0101086F08670BD0025115D8FF0E60
:103D400009D8B85D0101086F086702D0D880120059
:103D5000D89012000325D96EFF0E0421DA6EDF50D1
:103D6000056F0551020112000025036FE86A02BFCA
:103D7000E8680121046F120020EE01F02451D926D9
:103D80002551DA22DF50266F26C127F1286B273B09
:103D9000283BF00E281727510F0B2813F00E27177A
:103DA000296B0F0E28152A6F20EE02F02451D92618
:103DB0002551DA22DF5029112B6F2A512C6F2BC18C
:103DC0001BF12CC11CF1DDEC2DF01BC12DF11CC130
:103DD0002EF124C1D9FF25C1DAFF10EE02F02451E3
:103DE000E1262551E222DFCFE7FF20EE04F02D513E
:103DF000D9262E51DA22DF50266F20EE03F02D5106
:103E0000D9262E51DA22DF50276F2739F00B2611E1
:103E100024C1D9FF25C1DAFFDF6E20EE01F0245165
:103E2000D9262551DA2210EE02F02D51E1262E512D
:103E3000E222E750266F10EE01F02451E1262551D1
:103E4000E222E750276F2739F00B2611DF6E1200B0
:103E500004EE00F0D60EEE6AE806FDE10EEE00F08C
:103E6000F00EEE6AE806FDE10DEE00F0FE0EEE6AE1
:103E7000E806FDE10CEE00F0A00EEE6AE806FDE1BA
:103E80000BEE00F0F00EEE6AE806FDE10AEE00F03F
:103E9000F00EEE6AE806FDE109EE00F0D40EEE6ADF
:103EA000E806FDE108EE00F0F20EEE6AE806FDE13C
:103EB00007EE00F0E60EEE6AE806FDE106EE00F021
:103EC000FE0EEE6AE806FDE105EE00F0FC0EEE6A7D
:103ED000E806FDE103EEA6F05A0EEE6AE806FDE103
:103EE00002EEA6F05A0EEE6AE806FDE101EEBBF026
:103EF0002A0EEE6AE806FDE100EEE9F0170EEE6A22
:103F0000E806FDE100EE01F01F0EEE6AE806FDE1B5
:103F100004EED6F02A0EEE6AE806FDE100019EEFFF
:103F20008EF0F50E1D6F410E1C6F010E13EC3CF070
:103F30004DD056ECF1F002A449D002940201CF67B3
:103F400001D044D0080E0101226FA00E216FFD0E9A
:103F5000246F630E236F266B070E256FEBEC2FF09B
:103F60002251211133E1080E346F10D037D8DF62AF
:103F70000DD007D033D8DF6204D034C133F1320E14
:103F8000346F01013451800A4E0FF4E301013451C2
:103F9000800A4E0FEBE3A00E2F6F080E306F3351E7
:103FA0002F27000E30232FC121F130C122F1C8ECA0
:103FB00020F021C131F122C132F13251800A750F56
:103FC000B80ED8B4315D08E2D8901200310E03016A
:103FD000AA5D750EAB59ADE3D8801200342B3405C1
:103FE0002F6FA00E01012F25D96EDA6A080EDA2292
:103FF0002C0CE8CF1FF11FC11DF1080E1E6F8C9E07
:104000008A968A92040EE82EFED711D01DAF02D0F8
:104010008A8601D08A96040EE82EFED78C8E040E76
:10402000E82EFED78C9E0101D8901D371E07010196
:104030001E67ECD7040EE82EFED701011F51E00ADF
:1040400009E01F51E10A06E01F51E20A03E01F5197
:10405000E80A18E1100E1E6F12D01CAF02D08A863B
:1040600001D08A96040EE82EFED78C8E040EE82E20
:10407000FED78C9E0101D8901B371C371E071E6788
:10408000ECD71AD01F51E30A17E1080E1E6F12D0A9
:104090001BAF02D08A8601D08A96040EE82EFED786
:1040A0008C8E040EE82EFED78C9E040EE82EFED7D2
:1040B00001011E071E67ECD7040EE82EFED78A8288
:1040C0001200E8CF27F027500A0A57E10301D16B0D
:1040D0000901090E216E500E206EFD0E236E130E87
:1040E000226E256A070E246EC4EC30F02150201099
:1040F00004E1020E0201E46F020C0901090E216EB7
:10410000500E206EFD0E236E700E226E256A020E7A
:10411000246EC4EC30F02150201004E1010E0201A5
:10412000E46F010C0901090E216E500E206EFF0E86
:10413000236E9D0E226E256A030E246EC4EC30F0B1
:104140002150201004E1030E0201E46F030C090169
:10415000090E216E500E206EFF0E236E250E226E6C
:10416000256A040E246EC4EC30F021502010D8A42F
:104170001200040E0201E46F040C500E0301D1255D
:10418000D96EDA6A090EDA2227C0DFFFD12B1200BE
:1041900003D00101214B222B21C1D9FF22C1DAFF1B
:1041A000DF50200AF6E021C1D9FF22C1DAFFDF503B
:1041B000090AEFE00101286B296B276B2D0E21C145
:1041C000D9FF22C1DAFFDF6202D0272B07D02B0EE6
:1041D00021C1D9FF22C1DAFFDF6222D0214B222B7D
:1041E0001FD021C1D9FF22C1DAFFDF50236F246B1A
:1041F00023BF240728C11BF129C11CF11E6B0A0E25
:104200001D6FBBEC4AF023511B25256F24511C2147
:10421000266FD00E2525286FFF0E2621296FDED7A9
:1042200021C1D9FF22C1DAFFDF509FEC4CF0D9E267
:1042300027510DE028C123F129C124F1231F241F98
:10424000234B242B23C121F124C122F1120028C1C8
:1042500021F129C122F11200385126EC41F01BC195
:104260003DF11CC13EF13DC1D9FF3EC1DAFFDF5037
:104270003B6F380502E1280E0AD03851020AFBE0F4
:104280003851030AF8E03851040AF5E0020E3C6F99
:104290003C513B5D2AE3F00E1D6F380E1C6F000E83
:1042A00013EC3CF0880E01012F6F130E306F000EDF
:1042B000316B326B336B7CECA0F038C11EF1000E19
:1042C0007DEC30F0385126EC41F01BC13DF11CC1B2
:1042D0003EF13DC1D9FF3EC1DAFFDF503B6F500ECA
:1042E000266FE00E256FA3EC40F03DC1D9FF3EC123
:1042F000DAFFDF2A010138517CEC41F01BC139F1B2
:104300001CC13AF13B51020DF3503925D96E000E14
:104310003A21DA6E36C1DEFF37C1DDFFD8801200E8
:10432000205126EC41F01BC125F11CC126F125C10D
:10433000D9FF26C1DAFFDF502B6F2B6701D01200A7
:1043400020517CEC41F01BC127F11CC128F1296BE5
:1043500044D02951020DF3502725D96E000E282193
:10436000DA6EDECF21F1DDCF22F12151236F030E72
:104370002215246F1F1902E11E5123192DE125C1B9
:10438000D9FF26C1DAFFDF50DF062B6F29C12AF1E2
:104390001ED0D8902A35216F21512725226FE86A37
:1043A00021BFE8682821236F020E2225D96E000E56
:1043B0002321DA6E2A51020DF3502725E16E000EFB
:1043C0002821E26EDECFE6FFDDCFE5FF2A2B2B5161
:1043D0002A5DD8B01200DDD7292B2B51295DD8B02A
:1043E0001200B7D702D0264A272A26C0D9FF27C0F5
:1043F000DAFFDF50200AF7E026C0D9FF27C0DAFF36
:10440000DF50090AF0E02D6A2E6A2C6A2D0E26C0B4
:10441000D9FF27C0DAFFDF6202D02C2A07D02B0E8B
:1044200026C0D9FF27C0DAFFDF6222D0264A272A1A
:104430001FD026C0D9FF27C0DAFFDF50286E296AB7
:1044400028BE29062DC020F02EC021F0236A0A0EB6
:10445000226EF5EC49F0285020242A6E29502120A4
:104460002B6ED00E2A242D6EFF0E2B202E6EDED743
:1044700026C0D9FF27C0DAFFDF504AEC4CF0D9E262
:104480002C500DE02DC028F02EC029F0281E291E2A
:10449000284A292A28C026F029C027F012002DC05A
:1044A00026F02EC027F01200DACF14F1F3CF15F169
:1044B000F4CF16F1F6CF17F1F7CF18F1F8CF19F1C5
:1044C000F5CF1AF1DAEC4DF0F2A801D001D006D008
:1044D000F2A201D001D002D0F6EC0BF0F0A801D08E
:1044E00001D00AD0F0A201D001D006D0F0AE01D0A8
:1044F00001D002D0BFEC4DF0A3A601D001D00AD06C
:10450000A4A601D001D006D0A5A601D001D002D02A
:10451000ADECE3F0F2AA01D001D012D0F2A401D0A8
:1045200001D00ED0F1A401D001D00AD0000111A613
:1045300001D001D003D03AEC43F002D066EC3FF05A
:104540001AC1F5FF19C1F8FF18C1F7FF17C1F6FF2F
:1045500016C1F4FF15C1F3FF14C1DAFF13C1D9FF6F
:1045600012C1EAFF11C1E9FF1100E8CF2AF12D6B5A
:104570002A072A51330D8D0EF3242E6F130EF420CB
:104580002F6F2EC11EF12FC11FF1F6EC37F02B6FEC
:104590002C6B2E4B2F2B2C51800A800F020ED8B47F
:1045A0002B5D07E32C51800A800F180ED8B42B5DC9
:1045B00020E32569266912002E291E6F000E2F2187
:1045C0001F6FF6EC37F0276F2EC11EF12FC11FF1C0
:1045D000F6EC37F0296F2751286F28513F0A29112F
:1045E000D8B42D2B2B07D8A02C07020E2E27000E97
:1045F0002F232C51800A800F010ED8B42B5DDCE2F2
:10460000020E2D6505D0F00E266F000E256F000CF2
:104610002D51020A04E12669000E256F000C2D05BC
:10462000C8E12669F00E256FF00C00011AB01200E7
:1046300015BE138415A01AD001011B51220A1C11AA
:1046400010E01B51260A1C110CE01B512A0A1C11F8
:1046500008E01B512E0A1C1104E01B51360A1C11E4
:1046600005E1098008BE8A8CD3C2CAF2130E01018B
:10467000D6652BD0D607226B17D0D89022351D6F68
:10468000020E01011D25D96EDA6A060EDA222251C8
:10469000020D000EF324E16EE26A060EE222DECF86
:1046A000E6FFDDCFE5FF222BD6C11DF11E6B22C137
:1046B0001FF1206B1FBF20072051800A216F1D5161
:1046C0001F5D1E51800A2159D8E3D651020D000EFC
:1046D000F324D96EDA6A060EDA2201011BC1DEFF6D
:1046E0001CC1DDFFD62B120000011AB0120015BE4E
:1046F000138415A019D02050220A211010E0205058
:10470000260A21100CE020502A0A211008E020502F
:104710002E0A211004E02050360A211005E10980FC
:1047200008BE8A8CD3C2CAF2130E0101D6652BD003
:10473000D607276A16D0D8902734226E020E22247C
:10474000D96EDA6A060EDA222750020D000EF32423
:10475000E16EE26A060EE222DECFE6FFDDCFE5FF84
:10476000272A0101D6C122F0236A27C024F0256A36
:1047700024BE25062550800A266E2250245C235034
:10478000800A2658D8E3D651020D000EF324D96EC4
:10479000DA6A060EDA2220C0DEFF21C0DDFF010149
:1047A000D62B1200246B22AF0AD0221F211F201FFC
:1047B0001F6D000E202321232223010E246F1EAF24
:1047C0000AD01E1F1D1F1C1F1B6D000E1C231D2346
:1047D0001E23010E241B256B266B276B286B225191
:1047E0001F112011211129E0010E236F06D0D8904E
:1047F0001F37203721372237232B22AFF8D7D89005
:1048000025372637273728371F511B5D20511C5964
:1048100021511D5922511E5909E31F511B5F20517F
:104820001C5B21511D5B22511E5B2581D8902233D8
:10483000213320331F33232FE2D7245108E0281FD0
:10484000271F261F256D000E26232723282325C179
:104850001BF126C11CF127C11DF128C11EF1120058
:10486000E8CF2DF1000115B002D0D890120005C597
:104870001BF101012D516BEC49F0F7E30501E55106
:10488000070AF3E1310EE525D96EDA6A050EDA2260
:10489000DF6A340E01012B6F050E2C6F2BC121F145
:1048A0002CC122F18EEC24F021C12EF122C12FF176
:1048B0002EC125F12FC126F1CEEC47F0D6E30B989F
:1048C0000B960C9009900201CA6B08BE8A9C069A4E
:1048D00040841AA610D0020E01011C6FDD0E1B6F62
:1048E00015EC23F001011E6B540E1D6F2F0E1F6F70
:1048F000E2EC3DF00FD0020E01011C6FDD0E1B6FCC
:1049000015EC23F001011E6B540E1D6F0F0E1F6F6F
:10491000E2EC3DF000014094D8801200256B266B3C
:10492000276B02D0214B222B21C1D9FF22C1DAFFF4
:10493000DF5077EC4BF0F6E22D0E21C1D9FF22C1FA
:10494000DAFFDF6202D0252B07D02B0E21C1D9FF61
:1049500022C1DAFFDF621FD0214B222B1CD028514D
:10496000B0EC4CF004E328514DEC4DF0286F285189
:104970009FEC4CF0D00ED8A0A90E2827263B273B51
:10498000F00E271726510F0B2713F00E261728516C
:104990002627000E272321C1D9FF22C1DAFF214B90
:1049A000222BDF50286F0101285195EC47F0D7E208
:1049B00025510DE026C123F127C124F1231F241F17
:1049C000234B242B23C121F124C122F1120026C143
:1049D00021F127C122F11200000110BC08D020EE05
:1049E00003F02150D9262250DA22030EDF1649D8CF
:1049F00003E13FD8D8B41200020E0AEC49F00001DE
:104A000010AC0AD020EE08F02150D9262250DA222C
:104A1000DF500AEC49F024D020EE05F02150D926D1
:104A20002250DA22DF3A20EE05F02150D92622501A
:104A3000DA2210EE05F02150E1262250E222E75062
:104A4000236ED8902332D8902330030BDF6E20EEF4
:104A500005F02150D9262250DA22DF500AEC49F025
:104A600010D80AEC49F005D80AEC49F000010F8093
:104A7000120020EE02F02150D9262250DA22DF5017
:104A8000120020EE03F02150D9262250DA22DF5006
:104A90001200F80E01011D6FDE0E1C6F010E13ECEB
:104AA0003CF02C0E00EC4CF007016B510FE0220E95
:104AB00000EC4CF0070E01011D6F6B0E1C6F000E19
:104AC00013EC3CF0220E00EC4CF006D0220E00EC71
:104AD0004CF0220E00EC4CF02C0E00EC4CF0220EB0
:104AE00000EC4CF00601DF5108E0060E01011D6FDD
:104AF000DF0E1C6F000E13EC3CF0220E00EC4CF0AD
:104B00002C0E00EC4CF0220E00EC4CF00601E851AB
:104B100008E0060E01011D6FE80E1C6F000E13EC7D
:104B20003CF0220E00EC4CF0EE0E01011D6F180E51
:104B30001C6F000E13EC3CF00D0E00EC4CF0130E4D
:104B40000101306F880E2F6F77EF40F0EF0E0101FB
:104B50001D6FAF0E1C6F010E13EC3CF0070E010130
:104B60001D6F6B0E1C6F000E13EC3CF0220E00EC60
:104B70004CF00D0E00EC4CF0130E0101306F880E5E
:104B80002F6F77EC40F0ED0E01011D6F4D0E1C6F85
:104B9000010E13EC3CF0130E0101306F880E2F6FE5
:104BA00077EC40F0ED0E01011D6F650E1C6F010EDC
:104BB00013EC3CF0130E0101306F880E2F6F77EC71
:104BC00040F0EE0E01011D6F5A0E1C6F010E13EC2A
:104BD0003CF0130E0101306F880E2F6F77EC40F020
:104BE000EE0E01011D6F450E1C6F010E13EC3CF023
:104BF000130E0101306F880E2F6F77EC40F049EFF4
:104C000025F00301B25138EC4CF0256F5B0E010129
:104C10004CD8246F24AF12005B0E2525D96EDA6ABA
:104C2000070EDA22DF2A5B0E40D8246F3F0E2417CE
:104C3000030E245D02E38F8014845B0E010135D8DE
:104C40003F0B050A09E1530E0301ED6F300EEE6FC5
:104C500001012551FAEC41F05B0E01012525D96EC9
:104C6000DA6A0701070EDA22DF503F0B3F0AD8A4A9
:104C70001200530E0301ED6F200EEE6F010125515E
:104C8000FAEC41F05B0E01012525D96EDA6A070EB8
:104C9000DA22DF6A960E25251D6F1E6B020E1E237B
:104CA0005B0E03D81F6FE2EF3DF02525D96EDA6A5F
:104CB000070EDA22DF501200436B50D843512825EB
:104CC0001E6F000E29211F6FF6EC37F0DF6E46D8FD
:104CD000DF5004E0432B100E4365EFD7305107E05F
:104CE0002951020A410ED8B4281901E01C8601019D
:104CF000416B30512B0A03E1010E416F4307D8513C
:104D000009E0D851435D426F4251800A7F0F02E3B0
:104D100042514127300E2C6F010E2D6F41512C272F
:104D2000000E2D232CC121F12DC122F1200E2E6F5A
:104D3000050E2F6F2A512E27000E2F232EC123F18F
:104D40002FC124F12BC125F1266BEBEC2FF0225162
:104D5000211102E1D8801200D8901200300E4325B4
:104D6000D96EDA6A010EDA221200E8CF59F102C5D3
:104D70001BF1010159516BEC49F002E2D89012008D
:104D80000501E551070AFAE1310EE525D96EDA6A27
:104D9000050EDA22DF6A340E0101546F050E556FDD
:104DA00054C121F155C122F18EEC24F021C156F1FC
:104DB00022C157F156C125F157C126F1CEEC47F07B
:104DC000DDE300011FB602D000010F8845EC16F0AC
:104DD00001015939F00B586F800E466F585110EC95
:104DE00007F046C156F147C157F105010251B6EC33
:104DF0004DF002E2D8801200595185EC46F00101D5
:104E0000586F56C13FF157C140F159C141F158C1E6
:104E100042F1030E436F16EC3DF0ECD720EE01F0AB
:104E20002451D9262551DA22DF501B6F1C6BDDEC93
:104E30002DF01BC12AF11CC12BF120EE04F02A51E8
:104E4000D9262B51DA22DF50266F20EE03F02A51AB
:104E5000D9262B51DA22DF50276F2739F00B261184
:104E6000286F20EE02F02451D9262551DA22DF5096
:104E700060EC45F0296F20EE02F02451D92625512F
:104E8000DA2229C126F1263B0F0E261724C1E1FFA5
:104E900025C1E2FFE750F00B2611DF6E20EE01F096
:104EA0002451D9262551DA2210EE02F02A51E126AA
:104EB0002B51E222E750266F2939F00B2611DF6EC5
:104EC00024C1D9FF25C1DAFF28C1DFFF1200E8CFD6
:104ED00031F1FE0E01011D6F710E1C6F010E13ECFE
:104EE0003CF03D0E00EC4CF0010131C11BF11C6B9C
:104EF000DDEC2DF01BC133F11CC134F120EE03F0C9
:104F00003351D9263451DA22DF505BEC4CF000ECFF
:104F10004CF0010120EE04F03351D9263451DA224D
:104F2000DF505BEC4CF000EC4CF00D0E00EC4CF064
:104F300042EC4EF00101326B19D018EC4EF016E342
:104F40003EEC4EF00101356F0DD0355179EC4AF051
:104F50000DE30101322B0AD035518FEC4AF0D8B065
:104F6000120004D03251F1E0010AF6E01FEC4EF0DD
:104F7000D10E01012F5D070E3059D8B01200DDD7D8
:104F800020EE01F02451D9262551DA22DF501B6F83
:104F90001C6BDDEC2DF01BC12AF11CC12BF120EEA6
:104FA00004F02A51D9262B51DA22DF50266F20EE49
:104FB00003F02A51D9262B51DA22DF50276F2739E7
:104FC000F00B2611286F20EE02F02451D92625512E
:104FD000DA22DF50296F20EE02F02451D926255124
:104FE000DA2229C126F1263B0F0E261724C1E1FF44
:104FF00025C1E2FFE750F00B2611DF6E20EE01F035
:105000002451D9262551DA2210EE02F02A51E12648
:105010002B51E222E750266F2939F00B2611DF6E63
:1050200024C1D9FF25C1DAFF28C1DFFF1200E8CF74
:1050300059F103C51BF1010159516BEC49F002E232
:10504000D89012000501E551070AFAE1310EE52575
:10505000D96EDA6A050EDA22DF6A340E0101546F66
:10506000050E556F54C121F155C122F18EEC24F08B
:1050700021C156F122C157F156C125F157C126F180
:10508000CEEC47F0DDE300010F8645EC16F00101A0
:105090005939F00B586F840E466F585110EC07F0D9
:1050A00046C156F147C157F105010351B6EC4DF029
:1050B00002E2D8801200595185EC46F00101586F88
:1050C00056C13FF157C140F159C141F158C142F1B8
:1050D000030E436F16EC3DF0ECD71DC1D9FF1EC186
:1050E000DAFFDF50D55FD551D8B4120020EE01F0C1
:1050F0001D51D9261E51DA22000EDF6E32D01DC19D
:10510000D9FF1EC1DAFFDF5034D820C1D9FF21C139
:10511000DAFF10EE02F01D51E1261E51E222DFCF30
:10512000E7FF20EE02F01D51D9261E51DA2210EEC3
:1051300001F01D51E1261E51E222E7501AD820C18C
:10514000E1FF21C1E2FFDFCFE7FF20EE01F01D51BB
:10515000D9261E51DA22DF2A1DC1D9FF1EC1DAFF6E
:10516000DF2A1DC1D9FF1EC1DAFF3F0EDF64C7D79A
:105170003F0C1F6F1F511B25206FE86A1FBFE86897
:105180001C21216F1200E8CF59F15EC61BF101010D
:1051900059516BEC49F002E2D89012000501E5513B
:1051A000070AFAE1310EE525D96EDA6A050EDA2230
:1051B000DF6A340E0101546F050E556F54C121F1A1
:1051C00055C122F18EEC24F021C156F122C157F1D4
:1051D00056C125F157C126F1CEEC47F0DDE3F1ECE5
:1051E0003FF045EC16F001015939F00B586F150EE0
:1051F000466F585110EC07F046C156F147C157F1C0
:1052000006015E51B6EC4DF002E2D8801200595111
:1052100085EC46F00101586F56C13FF157C140F18E
:1052200059C141F158C142F1030E436F16EC3DF0F4
:10523000ECD7FD0E01011D6F810E1C6F010E13ECEA
:105240003CF0880E01012F6F130E306F000E316B92
:10525000326B336B7CECA0F00101366F06017551A7
:10526000800A500F04E37551800A460F12E30101D2
:1052700036510C0A0EE03651090A0BE0880E2F6FEA
:10528000130E306F316B326B010E336F7CECA0F07C
:10529000E3D7010136510C0A03E13651090A1DE03A
:1052A000366B750E01013625D96EDA6A060EDA22E2
:1052B000280E3625E16EE26A060EE222DFCFE7FF16
:1052C000362B3651800A710FECE3130E306F880EC7
:1052D0002F6F77EC40F0D8901200D880120035C1C3
:1052E0007AF136C17BF139D0C00E7A25376FFF0EC7
:1052F0007B21386F3851800A800F010ED8B4375D9A
:1053000014E37C6B2FD87C51800A400FFBE333D829
:10531000400E306FA4EC45F0400E3327000E3423CE
:10532000C00E7A27FF0E7B2318D07C6B01D01AD8D1
:105330007CC137F1386B37BF38073851800A396F75
:105340007A51375D7B51800A3959F1E314D87AC11B
:1053500030F1A4EC45F07A6B7B6B7B517A11D8B4B9
:105360001200C2D73A0E7C25D96EDA6A010EDA2213
:10537000DF687C2B120033C12CF134C12DF1010EFA
:105380002F6F3A0E2E6F1200E8CF05F105C102F122
:10539000080E0101066F8C9E8A968A92040EE82EF2
:1053A000FED711D002AF02D08A8601D08A96040EB1
:1053B000E82EFED78C8E040EE82EFED78C9E0101BF
:1053C000D8900237060701010667ECD7040EE82ED5
:1053D000FED701010551E60A06E1100E066F01D065
:1053E00014D80667FDD70551E50A06E1080E066FD9
:1053F00001D00BD80667FDD7040EE82EFED78A82AF
:1054000003C100F104C101F11200D8900337043741
:10541000040EE82EFED78C8E040EE82EFED781A453
:1054200003D00101038102D0010103918C9E060784
:10543000120001011E6B1F6B0BD047D8240EDF62D8
:1054400003D001011F2B04D040D8DF501E1BF9D719
:105450003CD8DF50F2E1310E1F25D96EDA6A050E15
:10546000DA222A0EDF6E1FC11CF11D6B1CBF1D0747
:10547000320E1C25D96E050E1D21DA6E1E390F0B5A
:105480001EBFF0095BEC4CF0DF6E1FC11CF11D6B01
:105490001CBF1D07330E01011C25D96E050E1D21F1
:1054A000DA6E1E510F0B5BEC4CF0DF6E1FC11CF16E
:1054B0001D6B1CBF1D07340E01011C25D96E050E86
:1054C0001D21DA6E000EDF6E000C310E01011F256A
:1054D000D96EDA6A050EDA2212000A0E296FA00EC2
:1054E000286F2B6B48D02907CD6BD1EC4AF0010116
:1054F000285128EC46F00101CD672FD01E5128EC31
:1055000046F001011D5128EC46F001012A6B1DD027
:105510002A511F25D96E000E2021DA6EDF5028ECAB
:1055200046F001012B2BC00E1D15266F1E51276F53
:105530001D4B1E2BC00E1D15226F1E51236F2719E8
:1055400002E12651221904E12A2B21512A5DE0E3D0
:1055500070EC48F001012B511200070E256FD00EA0
:10556000246F01D000F001012407D8A025072429C9
:10557000D8B42529F7E12951800A7F0FEBE3B3D78F
:10558000080E0401CB6F0401C5610CD0C5C4CBF477
:105590000401BF0502E1020EBF6F0401BF6702D024
:1055A000010EBF6F040104930491CBC405F4040100
:1055B000CB510401C55DC56F040E0401CA6F280EEE
:1055C000C96F0401C4A11DD022D0C2C4F6FFC3C458
:1055D000F7FF000EF86EC9C4D9FFCAC4DAFF0F0E78
:1055E000F76403D00800F55005D0F6CFE9FFF7CFF8
:1055F000EAFFEF50DF6E0401C24BC32B0401C94B1D
:10560000CA2B0401CB07CB29D8B41200DED7C2C401
:10561000C7F4C3C4C8F43EEC45F0C7C4C2F4C8C460
:10562000C3F412000101766BCA390F0B566F576B2A
:1056300056510F0B5BEC4CF0716F3ED8CA510F0BFB
:105640005BEC4CF0DF6E38D8C9390F0B5BEC4CF0DB
:10565000DF6E32D8C9510F0B5BEC4CF0DF6E2CD8EB
:10566000DF6A010E286F580E276FFC0E2A6F900E0E
:10567000296F070E01012C6FB60E2B6F010E2E6FD6
:10568000710E2D6F66ECD5F02751766F580E76258A
:10569000D96EDA6A010EDA22DF6A326F580E316F84
:1056A000000E346B336B9EEC0CF001E2000C000139
:1056B00009B4010CBBEF14F0762B710E7625D96E70
:1056C000DA6A010EDA221200080E0401CB6F04011F
:1056D000C5610CD0C5C4CBF40401BF0502E1020EC4
:1056E000BF6F0401BF6702D0010EBF6F04010493B6
:1056F0000491CBC405F40401CB510401C55DC56F11
:10570000040E0401CA6F280EC96F0401C4A11DD084
:1057100022D0C2C4F6FFC3C4F7FF000EF86EC9C49E
:10572000D9FFCAC4DAFF0F0EF76403D00800F550A2
:1057300005D0F6CFE9FFF7CFEAFFEF50DF6E0401A7
:10574000C24BC32B0401C94BCA2B0401CB07CB2985
:10575000D8B41200DED7C2C4C7F4C3C4C8F41CEC6A
:1057600045F0C7C4C2F4C8C4C3F412000101E1513A
:105770001F0B02E0169801D016880301B02BB05120
:105780003E0A06E1B06B00014084CBECF3F040949C
:105790000101D20507E10201F06702D07DEF4CF074
:1057A000F0071200D251020A0EE10201F067F8D7A9
:1057B000EF2BEF51080AF2E1EF6B1A9A8B9C960ED1
:1057C0000201F06F960C00010CB0120006AA0BD07B
:1057D0000201F067E5D7EF2BEF51060ADFE1EF6B2F
:1057E0001A9A8B8CECD716A804D000010D928B8CE2
:1057F00012000DA208D00201DF5105E0F067D0D7FA
:10580000DF077DEF4CF000010D928B9C1200E8CF7A
:105810005FF1000105BA02D0D890120061C61BF1F9
:1058200001015F516BEC49F0F7E3040E0501E561FE
:1058300001D0F2D725EEE5F0050EDF6401D0ECD7FC
:1058400045EC16F001015F39F00B566F180E466FEC
:10585000565110EC07F0080E0101576F0501E55194
:10586000040A09E1325138EC4CF0586F33C559F154
:1058700034C55AF111D0335138EC4CF0546F050156
:10588000325138EC4CF0556F5539F00B5411586FBC
:1058900034C559F135C55AF15B6B5C6B5D6B5E6B62
:1058A000010E1D6F570E1C6F0BEC4AF0D8801200D2
:1058B000050E3B6F0401E551E41105E1B2EC44F043
:1058C0003FE3D8801200E4C439F1E5C43AF10101A4
:1058D0003751392738513A233A51800A7D0FE90E62
:1058E000D8B4395D2DE30401E46BE56B51EC36F07F
:1058F00023E3E7D791EC1FF014E2B2EC44F0E1E2CD
:1059000035C11CF136C11DF1000E13EC3CF0010154
:1059100037510401E427010138510401E523D890EF
:10592000120042EC4EF01FEC4EF0890E01012F5D8B
:10593000130E3059F8E33B0701013B67DBD7C1D7B2
:1059400035C11CF136C11DF1000E13EC3CF0DFD760
:10595000000109B21200010E21C0D9FF22C0DAFFF6
:10596000DF6204D0060E0AEC49F003D0070E0AEC01
:1059700049F020EE02F033D820EE01F0215024D877
:105980000AEC49F020EE05F02AD8233A0F0E231630
:10599000231620EE03F0215017D80AEC49F020EE30
:1059A00005F01DD82338F00B256E25500AEC49F080
:1059B00020EE04F02150D9262250DA22DF500AECE2
:1059C00049F000010F801200D9262250DA22DF5060
:1059D000246E2438F00B2310256E25501200215020
:1059E000D9262250DA22DF50236E1200E8CF57F179
:1059F0001CB609D00101575103E05751050A03E1D4
:105A0000010E576F138651C61BF1010157516BEC04
:105A100049F002E2D8901200000113A60CD01396B0
:105A20000101316B010E326F050E62ECD7F0F2E32B
:105A3000050E0101576F45EC16F001015739F00BC7
:105A4000566F8D0E466F565110EC07F046C154F15B
:105A500047C155F106015151B6EC4DF002E2D88034
:105A60001200575185EC46F00101566F54C13FF1C9
:105A700055C140F157C141F156C142F1030E436F88
:105A800016EC3DF0ECD76598080E0401016F040197
:105A9000C4BF1BD00401C1510EE0020E0401C06F4F
:105AA0000401056BC80E046F040E036F280E026F0D
:105AB000C80E006FC80C040E0401036F200E026FA5
:105AC0008C0E006F840E046F840C0401C151D8A4A5
:105AD0001200040120AFE1D70401C5510401265D85
:105AE000000E2759D8A026C4C5F464EC2BF0010E93
:105AF0000401C06F040E0401036F200E026F800EBC
:105B0000006F080E016F040E036F200E026F800EEF
:105B1000006F040E076F280E066FC80E046FC80CC6
:105B20006598080E0401016F0401C4BF1BD0040175
:105B3000C1510EE0020E0401C06F0401056BC80ED6
:105B4000046F040E036F280E026FC80E006FC80C9E
:105B5000040E0401036F200E026F8C0E006F840E82
:105B6000046F840C0401C151D8A41200040120AFB9
:105B7000E1D70401C5510401265D000E2759D8A0C4
:105B800026C4C5F4C0EC2AF0010E0401C06F040E57
:105B90000401036F200E026F800E006F080E016F6C
:105BA000040E036F200E026F800E006F040E076F4D
:105BB000280E066FC80E046FC80C0101010E1E6F7F
:105BC0001F0E1D6F1F6B206B216B226B236B100E42
:105BD0001B5D270E1C590AE31F2B100E1B5F270E9F
:105BE0001C5B100E1B5D270E1C59F6E2E80E1B5DB8
:105BF000030E1C590AE3202BE80E1B5F030E1C5BEF
:105C0000E80E1B5D030E1C59F6E2640E1B5D000ED0
:105C10001C590AE3212B640E1B5F000E1C5B640EF3
:105C20001B5D000E1C59F6E20A0E1B5D000E1C598E
:105C30000AE3222B0A0E1B5F000E1C5B0A0E1B5D83
:105C4000000E1C59F6E21BC123F11DC11BF11EC140
:105C50001CF11200E8CF28F01D9828B21D88000121
:105C60000CA008D028A2120000011AA812000001FE
:105C700007881200000106AA120000010BB81200EA
:105C800000010BA613D000F028A208D0216A260E2E
:105C9000206E74EC23F000011D861200216A280E8C
:105CA000206E74EC23F000011D96120028A2120051
:105CB0000B881AA604D00401C6C3DEF403D0040185
:105CC000C5C3DEF4DF6BDE3BDF3BF00EDF17DE51DA
:105CD0000F0BDF13F00EDE17DF51DE11D8A4120018
:105CE0000B980B86216A260E206E74EF23F00401B8
:105CF00020511F0B0101006F0005D8A41200040100
:105D00002039E832030B0101006F0005D8A412000E
:105D1000040124512AE02405D8A4120026D0040E40
:105D20000401C36FB50EC26F080EC56FC4810401B4
:105D3000C48F1200040E0401C36FB50EC26FF7D7F3
:105D4000010E0401C16F010C040E0401C36FCE0EDD
:105D5000C26F070EC56F810EC46F810C22C4CCF4D4
:105D60000401CC8F0401C48F120004012151D7E03B
:105D7000010AE0E0210AE4E0010AE6E0030AD8A40F
:105D80001200ECD7040120511F0B01011B6F1B05F2
:105D9000D8A4120004012039E832030B01011B6F63
:105DA0001B05D8A41200040124512AE02405D8A41C
:105DB000120026D0040E0401C36FB50EC26F080E88
:105DC000C56FC4810401C48F1200040E0401C36FA7
:105DD000B50EC26FF7D7010E0401C16F010C040E9E
:105DE0000401C36FCE0EC26F070EC56F810EC46F64
:105DF000810C22C4CCF40401CC8F0401C48F1200A6
:105E000004012151D7E0010AE0E0210AE4E0010A9F
:105E1000E6E0030AD8A41200ECD704012039E832E6
:105E2000030BD8A412002ED00401C48F080E040165
:105E3000CD6F080CADEF43F0D3EF3AF0040E040140
:105E4000C36FBD0EC26F0401C481010EC56FC48F44
:105E5000010C0AEF31F04DEF1BF0BE0E01011E6F79
:105E6000040E1F6F0401245101011E27000E1F2381
:105E70001EC1C2F41FC1C3F4E6D70401C48F22C4FB
:105E8000BEF4120004012151E4E0010AE4E0020A38
:105E9000E2E0060AC9E0030ACDE00E0ACFE0010AFB
:105EA000CBE0030ADAE0010AD8A41200E6D73DD01D
:105EB00028C121F129C122F12AC123F12BC124F1EA
:105EC0002AC11BF12BC11CF195EC3FF01BC125F140
:105ED0001CC126F1EBEC2FF02251211105E128C164
:105EE00028F129C129F1120028291B6F000E292150
:105EF0001C6F2AC1F6FF2BC1F7FF000EF86E0F0EC4
:105F0000F76403D00800F55005D0F6CFE9FFF7CFCE
:105F1000EAFFEF5001011D6F1E6B1DBF1E07C8EC8D
:105F200049F01BC128F11CC129F12951281106E0B3
:105F300028C1D9FF29C1DAFFDF50BAE1286B296BEC
:105F4000120004012039E832030BD8A412002ED02D
:105F50000401C48F080E0401CD6F080C61EF43F0FB
:105F600009EF3BF0040E0401C36FBD0EC26F0401C4
:105F7000C481010EC56FC48F010C59EF33F0C2EF1D
:105F800016F0BE0E0101036F040E046F04012451CC
:105F900001010327000E042303C1C2F404C1C3F4AA
:105FA000E6D70401C48F22C4BEF4120004012151BB
:105FB000E4E0010AE4E0020AE2E0060AC9E0030ABA
:105FC000CDE00E0ACFE0010ACBE0030ADAE0010AD5
:105FD000D8A41200E6D735D021C1D9FF22C1DAFFFB
:105FE000DF5013E039D8F76403D00800F55005D02E
:105FF000F6CFE9FFF7CFEAFFEF500101276F21C18C
:10600000D9FF22C1DAFFDF1818E021C1D9FF22C170
:10601000DAFFDF50276F20D8F76403D00800F5506F
:1060200005D0F6CFE9FFF7CFEAFFEF500101275D7A
:10603000216F226BD8A022071200214B222B234B69
:10604000242B2507D8A0260701012529D8B4262905
:10605000C3E1216B226B120023C1F6FF24C1F7FFBD
:10606000000EF86E0F0E12000401E86BE96BFC0ED7
:1060700001011D6FB30E1C6F010E13EC3CF0880E76
:1060800001012F6F130E306F000E316B326B336BCB
:106090007CECA0F00101366F880E2F6F130E306F6D
:1060A000316B326B010E336F7CECA0F00101365185
:1060B000180AD8B412003651160AD8B41200365154
:1060C0001A0AD8B4120036511B0AD8B4120036513D
:1060D000170AD8B4120042EC4EF01FEC4EF0D10E6D
:1060E00001012F5D070E3059F8E3780E0401E85DD9
:1060F000000EE959D8B01200BAD7E8CF22F1010159
:106100001E5126EC41F01BC123F11CC124F123C117
:10611000D9FF24C1DAFFDF50276F276701D01200B3
:106120001E517CEC41F01BC125F11CC126F123C19D
:10613000D9FF24C1DAFFDF50DF06276F22C128F123
:106140001ED0D89028351F6F1F512525206FE86A73
:106150001FBFE8682621216F020E2025D96E000E90
:106160002121DA6E2851020DF3502525E16E000E33
:106170002621E26EDECFE6FFDDCFE5FF282B27519B
:10618000285DD8B01200DDD733D020C0D9FF21C0A0
:10619000DAFFDF5012E036D8F76403D00800F5507C
:1061A00005D0F6CFE9FFF7CFEAFFEF50266E20C00B
:1061B000D9FF21C0DAFFDF1817E020C0D9FF21C0C6
:1061C000DAFFDF50266E1ED8F76403D00800F550C2
:1061D00005D0F6CFE9FFF7CFEAFFEF50265C206E3F
:1061E000216AD8A021061200204A212A224A232A05
:1061F0002406D8A025062428D8B42528C6E1206A7C
:10620000216A120022C0F6FF23C0F7FF000EF86ECD
:106210000F0E12000401286B296B24D00401C48FD7
:10622000040128810401C65125E00401288322D0FD
:106230000401C48F1FD00401C48F8BEC4BF025D810
:10624000F76403D00800F55005D0F6CFE9FFF7CF8B
:10625000EAFFEF5001011B6F1BA50CD0010E0401DA
:10626000286F08D0040120511F0BD8E0010AE0E09C
:10627000030AE1E00401C4AF1200040EC36F280E4C
:10628000C26FC481020EC56F020CC7C4F6FFC8C43A
:10629000F7FF000EF86E0F0E1200E8CF28F0020193
:1062A000FC670AD028A803D0216A360E02D0216AE2
:1062B000380E206E74EF23F0FC0522E10BA803D00A
:1062C0001E9828B81E8800010BB812001AA603D029
:1062D00000011EBA1200000106AA120028A808D068
:1062E000216A360E206E74EC23F000011E86120027
:1062F000216A380E206E74EC23F000011E96120005
:10630000FC51020AD8A412001AA603D000011EBA3A
:106310001200000106AA120028B8E2D7E9D7E8CF98
:1063200028F00201F9670AD028A003D0216A220EC2
:1063300002D0216A240E206E74EF23F0F90522E1C9
:106340000BA803D01D9228B01D8200010BB81200CB
:106350001AA603D000011DB41200000106AA120003
:1063600028A008D0216A220E206E74EC23F00001D0
:106370001D801200216A240E206E74EC23F00001AF
:106380001D901200F951020AD8A412001AA603D0D7
:1063900000011DB41200000106AA120028B0E2D7C5
:1063A000E9D7E8CF28F00201FB670AD028A603D07E
:1063B000216A2E0E02D0216A300E206E74EF23F077
:1063C000FB0522E10BA803D01E9228B61E82000115
:1063D0000BB812001AA603D000011EB4120000016F
:1063E00006AA120028A608D0216A2E0E206E74EC90
:1063F00023F000011E801200216A300E206E74EC22
:1064000023F000011E901200FB51020AD8A41200D2
:106410001AA603D000011EB41200000106AA120041
:1064200028B6E2D7E9D7E8CF28F00201FA670AD008
:1064300028A403D0216A2A0E02D0216A2C0E206ED5
:1064400074EF23F0FA0522E10BA803D01D9C28B4B9
:106450001D8C00010BB812001AA603D000011DBE4E
:106460001200000106AA120028A408D0216A2A0EF0
:10647000206E74EC23F000011D8A1200216A2C0E9C
:10648000206E74EC23F000011D9A1200FA51020AEA
:10649000D8A412001AA603D000011DBE12000001EC
:1064A00006AA120028B4E2D7E9D715B00BAA24D067
:1064B000180E01011D6503D03C0E1D6502D0018C34
:1064C00001D0019C29D824E00201AE4BAF2B010181
:1064D0001B510201AE5D01011C510201AF590AE3DB
:1064E0000001019E01BC018E01BE02D0D8901200B5
:1064F000D88012000001F8D73E0E01011D6102D0C4
:10650000019C04D04C0E1D6501D0018C05D8DCE146
:106510000201AE6BAF6BEED7010E01AC000E0101B4
:106520001E6F010E01AE000E1E1B120015B00BAA4D
:1065300024D0180E01011D6503D03C0E1D6502D04C
:10654000028001D0029029D824E00201B04BB12B87
:1065500001011B510201B05D01011C510201B15941
:106560000AE30001029202B0028202B202D0D89085
:106570001200D88012000001F8D73E0E01011D6103
:1065800002D0029004D04C0E1D6501D0028005D8C7
:10659000DCE10201B06BB16BEED7010E02A0000E80
:1065A00001011E6F010E02A2000E1E1B120015B08B
:1065B0000BAA24D0180E01011D6503D03C0E1D65E9
:1065C00002D0018401D0019429D824E00201AA4B11
:1065D000AB2B01011B510201AA5D01011C510201FB
:1065E000AB590AE30001019601B4018601B602D05D
:1065F000D8901200D88012000001F8D73E0E010199
:106600001D6102D0019404D04C0E1D6501D001849F
:1066100005D8DCE10201AA6BAB6BEED7010E01A439
:10662000000E01011E6F010E01A6000E1E1B1200BE
:1066300015B00BAA24D0180E01011D6503D03C0E25
:106640001D6502D0018001D0019029D824E002010B
:10665000A84BA92B01011B510201A85D01011C518E
:106660000201A9590AE30001019201B0018201B2BD
:1066700002D0D8901200D88012000001F8D73E0E48
:1066800001011D6102D0019004D04C0E1D6501D0A6
:10669000018005D8DCE10201A86BA96BEED7010EE1
:1066A00001A0000E01011E6F010E01A2000E1E1BB3
:1066B00012000401286B296B2AD00401C48F040145
:1066C00028810401C6512BE00401288328D004014D
:1066D000C48F25D00401C48FB3EC4BF0C7C4F6FFC0
:1066E000C8C4F7FF000EF86E0F0EF76403D0080061
:1066F000F55005D0F6CFE9FFF7CFEAFFEF500101E3
:10670000006F00A50CD0010E0401286F08D0040111
:1067100020511F0BD2E0010ADAE0030ADBE004019A
:10672000C4AF1200040EC36F280EC26FC481020EE4
:10673000C56F020C15B00BAA24D0180E01011D65FF
:1067400003D03C0E1D6502D0018801D0019829D8E4
:1067500024E00201AC4BAD2B01011B510201AC5DE9
:1067600001011C510201AD590AE30001019A01B86F
:10677000018A01BA02D0D8901200D880120000011C
:10678000F8D73E0E01011D6102D0019804D04C0ED5
:106790001D6501D0018805D8DCE10201AC6BAD6B51
:1067A000EED7010E01A8000E01011E6F010E01AA15
:1067B000000E1E1B1200F80E01011D6FC60E1C6F8D
:1067C000010E13EC3CF00301D62B42EC4EF01FEC13
:1067D0004EF0E90E01012F5D030E3059F8E3020E71
:1067E0000301D665020CD66BFB0E01011D6F240E52
:1067F0001C6F010E13EC3CF0010E0101306FF40E22
:106800002F6F77EC40F042EC4EF01FEC4EF0E90EAB
:1068100001012F5D030E3059F8E38E9C8D9842ECF8
:106820004EF01FEC4EF0E90E01012F5D030E3059C2
:10683000F8E3AEEFCAF033D02AC121F12BC122F127
:106840002CC123F12DC124F12CC11BF12DC11CF150
:1068500095EC3FF01BC125F11CC126F13FEC3BF04C
:106860002251211105E12AC12AF12BC12BF112007D
:106870002A291C6F000E2B211D6F2CC1F6FF2DC184
:10688000F7FF000EF86E0800F5501E6F1F6B1EBF5D
:106890001F07C6EC45F01CC12AF11DC12BF12B517D
:1068A0002A1106E02AC1D9FF2BC1DAFFDF50C4E16B
:1068B0002A6B2B6B120015B00BAA26D0180E22647F
:1068C00003D03C0E226402D0018001D00190010E61
:1068D00001A0000E236E010E01A2000E231A26E075
:1068E0000201A84BA92B2050A85D2150A9590AE309
:1068F0000001019201B0018201B202D0D8901200D1
:10690000D88012000001F8D73E0E226002D001901C
:1069100004D04C0E226401D00180010E01A0000EB3
:10692000236E010E01A2000E231ADAE10201A86B08
:10693000A96BE8D715B00BAA26D0180E226403D095
:106940003C0E226402D0018401D00194010E01A406
:10695000000E236E010E01A6000E231A26E002018E
:10696000AA4BAB2B2050AA5D2150AB590AE3000182
:10697000019601B4018601B602D0D8901200D880E9
:1069800012000001F8D73E0E226002D0019404D01C
:106990004C0E226401D00184010E01A4000E236E6E
:1069A000010E01A6000E231ADAE10201AA6BAB6BFD
:1069B000E8D715B00BAA26D0180E226403D03C0EDF
:1069C000226402D0018801D00198010E01A8000EB6
:1069D000236E010E01AA000E231A26E00201AC4B21
:1069E000AD2B2050AC5D2150AD590AE30001019A56
:1069F00001B8018A01BA02D0D8901200D8801200E2
:106A00000001F8D73E0E226002D0019804D04C0E4F
:106A1000226401D00188010E01A8000E236E010E30
:106A200001AA000E231ADAE10201AC6BAD6BE8D7C4
:106A300015B00BAA26D0180E226403D03C0E226497
:106A400002D0028001D00290010E02A0000E236E3F
:106A5000010E02A2000E231A26E00201B04BB12B58
:106A60002050B05D2150B1590AE30001029202B0FA
:106A7000028202B202D0D8901200D8801200000127
:106A8000F8D73E0E226002D0029004D04C0E226451
:106A900001D00280010E02A0000E236E010E02A2A0
:106AA000000E231ADAE10201B06BB16BE8D715B022
:106AB0000BAA26D0180E226403D03C0E226402D00A
:106AC000018C01D0019C010E01AC000E236E010E61
:106AD00001AE000E231A26E00201AE4BAF2B205070
:106AE000AE5D2150AF590AE30001019E01BC018E49
:106AF00001BE02D0D8901200D88012000001F8D751
:106B00003E0E226002D0019C04D04C0E226401D0C3
:106B1000018C010E01AC000E236E010E01AE000EC1
:106B2000231ADAE10201AE6BAF6BE8D7FC0E1D6FE2
:106B3000A20E1C6F010E13EC3CF0300E01012F6F02
:106B4000750E306F000E316B326B336B7CECA0F046
:106B50000101366F36510C0A03E03651090A01E192
:106B6000000C36C137F1300E2F6F750E306F316B60
:106B7000326B010E336F7CECA0F0080AF1E10101E9
:106B800037510B0A0AE142EC4EF01FEC4EF0890E31
:106B900001012F5D130E3059F8E337510A0A03E063
:106BA00037510B0ADDE137511200E8CF1DF11D51BD
:106BB000FE0F1C6F0201CB6B01011E6B0DD0EA0EA4
:106BC00001011E25D96EDA6A0301030EDA22DF50B5
:106BD00003EC4EF001011E2B1C511E5DF0E302017F
:106BE000CB390F0B5BEC4CF01E6FE80E01011D253D
:106BF000D96EDA6A030EDA22DF501E1902E0D8904D
:106C000012000201CB510F0B5BEC4CF01E6FE90E32
:106C100001011D25D96EDA6A030EDA22DF501E1932
:106C2000EEE1D8801200010E26EC41F01BC11EF1EE
:106C30001CC11FF11EC1D9FF1FC1DAFFDF6A020E9E
:106C400026EC41F01BC11EF11CC11FF11EC1D9FF72
:106C50001FC1DAFFDF6A030E26EC41F01BC11EF1F3
:106C60001CC11FF11EC1D9FF1FC1DAFFDF6A040E6C
:106C700026EC41F01BC11EF11CC11FF11EC1D9FF42
:106C80001FC1DAFFDF6A050E26EC41F01BC11EF1C1
:106C90001CC11FF11EC1D9FF1FC1DAFF000EDF6E3C
:106CA000000C1A0E00EC4CF00301AA6BAB6B0294C3
:106CB0002FD056ECF1F002A42BD002940201CF6742
:106CC00001D026D0080E0101226FA00E216FFD0E0B
:106CD000246F6B0E236F266B070E256FEBEC2FF0E6
:106CE0002251211102E1D8901200080E0101226FF9
:106CF000A00E216FFB0E246F420E236F266B090E30
:106D0000256FEBEC2FF02251211102E1D880120007
:106D1000310E0301AA5D750EAB59F8E2CAD7E8CF70
:106D200027F11F6B580E1E6FF6EC37F0286F250504
:106D300007E11E6B580E1D6F2851FE0B27110CD05A
:106D40002551020A0CE11E6B580E1D6FD890273595
:106D5000266F2851FD0B15D01F6FE2EF3DF0255136
:106D6000030A05E11E6B0FD82851FB0B0AD02551F1
:106D7000040AD8A412001E6B06D8D89026372851D2
:106D8000F70B2611E9D7580E1D6F27C126F1D890B1
:106D90002637D8902637580C206B1EAF06D01D6DB5
:106DA0001E1FD8B01E2B010E206F1CAF06D01B6D0E
:106DB0001C1FD8B01C2B010E201B216B226B1E51F7
:106DC0001D111BE0010E1F6F04D0D8901D371E3718
:106DD0001F2B1EAFFAD7D890213722371D511B5DCC
:106DE0001E511C5905E31D511B5F1E511C5B218167
:106DF000D8901E331D331F2FEED7205104E0216D94
:106E0000221FD8B0222B21C11BF122C11CF112007C
:106E1000E8CF57F152C61BF1010157516BEC49F015
:106E200002E2D890120000010DA6FBD78A8C040163
:106E3000DA6BDB6B00011B8E45EC16F00101573954
:106E4000F00B566F030E466F565110EC07F046C11B
:106E500054F147C155F106015251B6EC4DF002E232
:106E6000D8801200575185EC46F00101566F54C18D
:106E70003FF155C140F157C141F156C142F1030EF6
:106E8000436F16EC3DF0ECD71BC1D9FF1CC1DAFFF4
:106E900010EE06F028D810EE05F01B51E1261C512B
:106EA000E222DFCFE7FF20EE04F01B51D9261C5170
:106EB000DA221BC1E1FF1CC1E2FFDFCFE7FF20EEBA
:106EC00002F01B51D9261C51DA2210EE04F00BD827
:106ED000CA51DF6E20EE02F01B51D9261C51DA2276
:106EE000C9C1DFFF12001B51E1261C51E222DFCF96
:106EF000E7FF20EE01F01B51D9261C51DA221200C7
:106F0000E8CF23F0226A23C021F0010E2116205081
:106F1000010B2118D8A4228023C021F0020E2116D3
:106F20002050020B2118D8A4228223C021F0040E85
:106F300021162050040B2118D8A4228423C021F04C
:106F4000080E21162050080B2118D8A4228623C031
:106F500021F0100E21162050100B2118D8A42288E1
:106F600023C021F0200E21162050200B2118D8A478
:106F7000228A22501200E8CF57F168C61BF10101A6
:106F800057516BEC49F002E2D890120045EC16F034
:106F900001015739F00B566F010E316F326B040E41
:106FA00062ECD7F0F1E3250E0101466F565110EC6B
:106FB00007F046C154F147C155F106016851B6ECDE
:106FC0004DF002E2D8801200575185EC46F00101E5
:106FD000566F54C13FF155C140F157C141F156C1FF
:106FE00042F1030E436F16EC3DF0ECD70A0E01019F
:106FF000236FA00E246F30D02307CD6BD1EC4AF065
:107000000101245128EC46F00101CD6717D01F5132
:1070100028EC46F001011E5128EC46F0D1EC4AF074
:1070200001012481245128EC46F0000E01EC47F0C8
:10703000226F70EC48F0010122511200070E216FFF
:10704000D00E206F01D000F001012007D8A0210749
:107050002029D8B42129F7E12351800A7F0FCCE2FF
:10706000000CE8CF57F166C61BF1010157516BECDC
:1070700049F002E2D890120045EC16F001015739B0
:10708000F00B566F010E316F326B020E62ECD7F0CF
:10709000F1E3230E0101466F565110EC07F046C193
:1070A00054F147C155F106016651B6EC4DF002E2CC
:1070B000D8801200575185EC46F00101566F54C13B
:1070C0003FF155C140F157C141F156C142F1030EA4
:1070D000436F16EC3DF0ECD7E8CF57F167C61BF1D4
:1070E000010157516BEC49F002E2D890120045ECD7
:1070F00016F001015739F00B566F010E316F326BEC
:10710000030E62ECD7F0F1E3240E0101466F5651F5
:1071100010EC07F046C154F147C155F10601675123
:10712000B6EC4DF002E2D8801200575185EC46F0E3
:107130000101566F54C13FF155C140F157C141F1B2
:1071400056C142F1030E436F16EC3DF0ECD7080E2A
:10715000296F33D00E0E2B6F2525276F000E2621A9
:10716000286F12D02B07BB0E01012B25D96EDA6ACE
:10717000010EDA222707D8A0280727C11EF128C14F
:107180001FF1F6EC37F0DF6E2B67ECD72A6B2B6B19
:10719000BB0E2B25D96EDA6A010EDA22DF502A1BCC
:1071A0002B2B2B51800A730FF3E32A5121EEC8F0E9
:1071B000DF6202D0D880120029072967CBD7D89088
:1071C0001200E8CF57F153C61BF1010157516BEC88
:1071D00049F002E2D89012008A9C0401DA6BDB6B62
:1071E00000011B9E45EC16F001015739F00B566F5C
:1071F000040E466F565110EC07F046C154F147C1DA
:1072000055F106015351B6EC4DF002E2D880120060
:10721000575185EC46F00101566F54C13FF155C1FD
:1072200040F157C141F156C142F1030E436F16ECD4
:107230003DF0ECD70401E86BE96BF90E01011D6F1D
:107240000B0E1C6F010E13EC3CF0880E01012F6F2A
:10725000130E306F000E316B326B336B7CECA0F091
:107260000101366F36512D0A06E1130E306F880E7C
:107270002F6F77EF40F0130E306F880E2F6F77EC83
:1072800040F042EC4EF01FEC4EF0D10E01012F5DAC
:10729000070E3059F8E3B40E0401E85D000EE95919
:1072A000CCE3FF00CAD720EE02F01B51D9261C51B7
:1072B000DA22DF501F6F20EE02F024D8E7501D6F56
:1072C00010EE02F01B51E1261C51E222E7501E6F26
:1072D0001E390F0B1D11DF6E20EE01F013D8DFCF2A
:1072E000E7FF20EE01F01B51D9261C51DA22DF6A9C
:1072F00020EE01F01B51D9261C51DA221F39F00B68
:10730000DF6E12001B51D9261C51DA221BC1E1FF8E
:107310001CC1E2FF1200E8CF9FF2000108BA050C81
:10732000000116B2050C9EC2A0F21DD09F6704D0CA
:10733000CFEC40F00201A16FA15119E0A06701D08C
:1073400016D0A151040A03E0A151020AD8B4DBEC23
:1073500033F042EC4EF01FEC4EF0990E01012F5D20
:107360003A0E3059F8E30201A007A029DFE1A1514C
:10737000040A03E0A151020AD8B4DBEC33F00201A5
:10738000A1511200FC0E1D6FC30E1C6F010E13ECF9
:107390003CF0880E01012F6F130E306F000E316B21
:1073A000326B336B7CECA0F00101366F36513A0A38
:1073B000D8A41200070E366F750E01013625D96E5E
:1073C000DA6A060EDA22300E3625E16EE26A070E20
:1073D000E222DFCFE7FF362B3651800A660FECE35F
:1073E00007014A6B130E0101306F880E2F6F77EF84
:1073F00040F0E8CF2BF12B07DC5138EC4CF0256F37
:10740000DB5138EC4CF0266F2639F00B2511296F33
:107410002B51220DF80EF3241E6F3F0EF4201F6F28
:10742000F6EC37F02A6F2A51291902E0D8901200A1
:107430002B51220DF90EF324276F3F0EF420286FF5
:1074400027C11EF128C11FF1F6EC37F02C6F010E99
:107450002C65ECD7100E2C6501D0E8D7D88012002F
:10746000E8CF57F155C61BF1010157516BEC49F0BC
:1074700002E2D890120000010DA8FBD78A8E45ECDD
:1074800016F001015739F00B566F060E466F565134
:1074900010EC07F046C154F147C155F106015551B2
:1074A000B6EC4DF002E2D8801200575185EC46F060
:1074B0000101566F54C13FF155C140F157C141F12F
:1074C00056C142F1030E436F16EC3DF0ECD7E8CF06
:1074D00037F119EC29F0D8B019EC29F0D8B0120026
:1074E0000101386B376712D06A0E38251D6F1E6B8D
:1074F000130E1E23280E01013825D96EDA6A060EF6
:10750000DA22DF501F6FE2EC3DF011D0790E382502
:107510001D6F1E6B130E1E23280E01013825D96E18
:10752000DA6A060EDA22DF501F6FE2EC3DF001014D
:10753000382B0E0E3865D6D70E0CD06B0301EA053A
:1075400002E0D89012000101016BEA0E0101012551
:10755000D96EDA6A0301030EDA22DF50F26F0101FD
:10756000006B0301F2510101D0190301F36F030114
:10757000F33303E3180E0101D01B00F00101D033F7
:107580000301F233D8900101002B070E0065E9D703
:10759000012B060E0165D9D70301F1510101D01964
:1075A000D0E1D88012000401C48F0F014D6B4E6BE7
:1075B0000401BE6B22C4BDF40401226704D0100E86
:1075C0000401CD6F100C200E0401CD6F0401CE6BB1
:1075D0004B0ECF6FD06BD16BD26BD36B080ED46FC9
:1075E000010ED56F0401CC6BCC8F0401B16B04018B
:1075F000B06B1A0E0F014E6F0401148D149F1E0EF6
:107600000F014F6F04011C8D1C9F188D189F40EFB8
:107610004DF00401C48F0F014D6B4E6B0401BE6B26
:1076200022C4BDF40401226704D0100E0401CD6F02
:10763000100C200E0401CD6F0401CE6B4B0ECF6FEA
:10764000D06BD16BD26BD36B080ED46F010ED56F9C
:107650000401CC6BCC8F0401B16B0401B06B1A0E2A
:107660000F014E6F0401148D149F1E0E0F014F6FFA
:1076700004011C8D1C9F188D189F26EF4DF029D0FA
:1076800023C1F6FF24C1F7FF000EF86E0800F55085
:1076900033EC4DF0276F21C1D9FF22C1DAFFDF5053
:1076A00033EC4DF0286F2751285D296F01012967C0
:1076B00006D021C1D9FF22C1DAFFDF5006E12951EE
:1076C000216F226B21BF22071200214B222B234B5B
:1076D000242B2507D8A0260701012529D8B426295F
:1076E000CFE1216B226B1200E8CF2DF12DC11BF1F0
:1076F0001C6B270E1E6F100E1D6FBBEC4AF0225143
:10770000640DF3CF25F1F4CF26F123510A0DF35088
:107710002525276FF4502621286F1B512725296F17
:107720001C5128212A6F21C11BF11C6B030E1E6FF7
:10773000E80E1D6FBBEC4AF01B5129252B6F1C5125
:107740002A212C6F24512B25216F000E2C21226F12
:107750001200E8CF2DF16DC61BF101012D516BEC2C
:1077600049F002E2D89012000501E551080AFAE159
:10777000310EE525D96EDA6A050EDA22DF6A350E9A
:1077800001012B6F050E2C6F2BC121F12CC122F1B1
:107790008EEC24F021C12EF122C12FF12EC125F152
:1077A0002FC126F1CEEC47F0DDE3500E266FD20E4E
:1077B000256FA3EC40F0FF00D8801200049C9CA22F
:1077C0009CB4048CAACFF8F004AC05D09C989C889B
:1077D00000010592120005820DAA0AD0640E020172
:1077E000DD25D96EDA6A080EDA22F8C0DFFFDD2B5C
:1077F0000CA604D00001F85161EF20F000011FB683
:107800004DEC0BF0000114B802D0000118B2A1EC4D
:1078100018F005A404D00001F851C5EC42F00001B5
:10782000F85156EFD1F0E8CF1EF101011E5118E0DA
:10783000410E00EC4CF0540E00EC4CF011D0010164
:107840001FD8F76403D00800F55005D0F6CFE9FF44
:10785000F7CFEAFFEF5000EC4CF001011C4B1D2B61
:1078600001010ED8F76403D00800F55005D0F6CF1B
:10787000E9FFF7CFEAFFEF500009D8B41200DFD7D5
:107880001CC1F6FF1DC1F7FF000EF86E0F0E1200AF
:10789000E8CF57F156C61BF1010157516BEC49F087
:1078A00002E2D89012008A9E45EC16F00101573989
:1078B000F00B566F070E466F565110EC07F046C19D
:1078C00054F147C155F106015651B6EC4DF002E2B4
:1078D000D8801200575185EC46F00101566F54C113
:1078E0003FF155C140F157C141F156C142F1030E7C
:1078F000436F16EC3DF0ECD7206B1CAF06D01B6D30
:107900001C1FD8B01C2B010E206F1EAF04D01D6DA4
:107910001E1FD8B01E2B1E511D1117E0010E1F6F28
:1079200004D0D8901D371E371F2B1EAFFAD71D511C
:107930001B5D1E511C5904E31D511B5F1E511C5B36
:10794000D8901E331D331F2FF2D7205104E01B6D3A
:107950001C1FD8B01C2B1BC11BF11CC11CF1120039
:10796000E8CF5CF150C61BF101015C516BEC49F0B2
:1079700002E2D89012005C5185EC46F001015B6F89
:107980005CC125F15B51010A8FEC36F045EC16F035
:1079900001015C39F00B5B6F010E466F5B5110EC1F
:1079A00007F006015051B6EC4DF002E2D88012000B
:1079B0005C5185EC46F001015B6F5BC154F15C5199
:1079C00023ECEDF0F3D7E8CF57F165C61BF10101C9
:1079D00057516BEC49F002E2D890120045EC16F0DA
:1079E00001015739F00B566F220E466F565110ECBD
:1079F00007F046C154F147C155F106016551B6EC97
:107A00004DF002E2D8801200575185EC46F001019A
:107A1000566F54C13FF155C140F157C141F156C1B4
:107A200042F1030E436F16EC3DF0ECD73F51446F2B
:107A3000030E4015456F43C146F1476B0D0ED890BC
:107A400046374737E82EFBD741C148F1496B0A0E4C
:107A5000D89048374937E82EFBD7465148114A6F2E
:107A6000475149114B6F44514A114C6F45514B11CD
:107A70004D6F4251D8A44D8F4CC136F14DC137F1F5
:107A800041C138F12CEC21F002E3D8801200D890EB
:107A90001200E8CF57F162C61BF1010157516BECA0
:107AA00049F002E2D890120045EC16F00101573976
:107AB000F00B566F190E466F565110EC07F046C189
:107AC00054F147C155F106016251B6EC4DF002E2A6
:107AD000D8801200575185EC46F00101566F54C111
:107AE0003FF155C140F157C141F156C142F1030E7A
:107AF000436F16EC3DF0ECD7E8CF57F163C61BF1AE
:107B0000010157516BEC49F002E2D890120045ECAC
:107B100016F001015739F00B566F200E466F565183
:107B200010EC07F046C154F147C155F1060163510D
:107B3000B6EC4DF002E2D8801200575185EC46F0C9
:107B40000101566F54C13FF155C140F157C141F198
:107B500056C142F1030E436F16EC3DF0ECD7E8CF6F
:107B600057F164C61BF1010157516BEC49F002E279
:107B7000D890120045EC16F001015739F00B566F02
:107B8000210E466F565110EC07F046C154F147C123
:107B900055F106016451B6EC4DF002E2D8801200B6
:107BA000575185EC46F00101566F54C13FF155C164
:107BB00040F157C141F156C142F1030E436F16EC3B
:107BC0003DF0ECD70A0E236FA00E226F26D02307BC
:107BD000CD6BD1EC4AF00101225128EC46F00101B5
:107BE000CD670DD01E5128EC46F001011D5128EC47
:107BF00046F001011F5128EC46F070EF48F0070EE7
:107C0000216FD00E206F01D000F001012007D8A015
:107C100021072029D8B42129F7E12351800A7F0FB9
:107C2000D8A01200D4D7E8CF57F10101570502E0E0
:107C3000D890120045EC16F001015739F00B566F41
:107C4000010E316F326B62ECD7F0F2E3230E0101CB
:107C5000466F565110EC07F0010146C154F147C17F
:107C600055F1575185EC46F00101566F54C13FF173
:107C700055C140F157C141F156C142F1030E436F66
:107C800016EC3DF0D880120000010EA8000C010196
:107C9000226B15D0000E01012225D96EDA6A0A0E78
:107CA000DA2222C11DF11E6B1DBF1E071D511B25AF
:107CB000E16E1E511C21E26EDFCFE7FF222BE3C2F3
:107CC0001DF101011E6B22C11FF1206B1FBF200798
:107CD0002051800A216F1D511F5D1E51800A2159BC
:107CE000D9E30E980201E35112000101386B96ECC2
:107CF00035F00101396F39510B0A03E137EC3FF0E0
:107D000020D8395102E038511AE042EC4EF01FEC15
:107D10004EF0990E01012F5D3A0E3059F8E3386BA1
:107D200096EC35F00101396F39510B0A03E137EC5C
:107D30003FF007D8395102E0385101E0010C46EF1D
:107D400009F0010ED8A0000E386F120033C12DF1DA
:107D500034C12EF135C12FF136C130F1C3EC46F0FC
:107D60000201D05122E00401DC4BDD2BD890DC3540
:107D70000101376F280E3725D96EDA6A090EDA222B
:107D80000401FAC4DEFFFBC4DDFFD890DC3501013D
:107D9000376F000E3725D96EDA6A0901090EDA222B
:107DA000000EDE6EDD6ED880000CD8901200E8CF99
:107DB00054F145EC16F00201F139F00B0101576F57
:107DC00010D0820E466F575110EC07F005D0810E8F
:107DD000466F575110EC07F046C155F147C156F1B7
:107DE00004D05451EEE0010AF2E00201F15185ECB9
:107DF00046F00101576F55C13FF156C140F1F1C244
:107E000041F157C142F1030E436F16EF3DF025C11A
:107E1000F8F21C9A13D00101260507E123C11BF1DA
:107E200024C11CF1A4EC48F006D023C11BF124C1ED
:107E30001CF144EC3EF00201D56FF76B0201D567EF
:107E400002D0F867E8D7F86703D000011C8A000C5D
:107E5000D507F75101012325D96E000E2421DA6ED2
:107E6000DF50276F0201F72B010127511200FB0E93
:107E70001D6F380E1C6F010E13EC3CF0E80E010173
:107E80002F6FFD0E306F000E316B326B336B7CEC5D
:107E9000A0F00101366F36510C0A11E03651090A83
:107EA0000EE03651080A0BE0E80E2F6FFD0E306F22
:107EB000316B326B010E336F7CECA0F0EAD7365198
:107EC000080A02E1D8901200D8801200F294000152
:107ED000F96702D095EF4DF0F90502E17EEF4DF024
:107EE000F951020A02E1A0EF4DF0F951030A02E153
:107EF00008EF46F0F951040A02E11EEF40F0F95193
:107F0000050A02E14FEF4BF0F951060A02E1FDEFDD
:107F10004AF0F951070A02E15BEF47F0F951080A0C
:107F200002E14BEF40F0F96B12001BC11FF11CC1C5
:107F300020F101011F511D6F20511E6F1F4B202B7F
:107F40001DC1F6FF1EC1F7FF000EF86E0F0EF7649D
:107F500003D00800F55005D0F6CFE9FFF7CFEAFFD0
:107F6000EF500009E6E101011FC11DF120C11EF122
:107F70001B511D5F1C511E5BFF0E1D251B6FFF0E4D
:107F80001E211C6F12003DC131F13EC132F13FC1D3
:107F900033F140C134F19EEC0CF002E2D8901200B3
:107FA00000010E9842EC4EF013D000010EA810D044
:107FB0000A0E01012B6F000E2A6F3DC12CF13EC14C
:107FC0002DF14AEC10F002E3D880120000010E9867
:107FD0001FEC4EF0E90E01012F5DFD0E3059DEE27F
:107FE000E4D7408401011E6B520E1D6FFEC21FF1CB
:107FF000E2EC3DF001011F6B520E1E6FF6EC37F004
:108000000201FD6F0101E06BF4C41FF1F5C420F122
:10801000B4EC17F00201FE6F15B00BAA04D0FD51AD
:10802000E00BFE1903D00201FE51FD190101E06FC2
:10803000E0C1E8F3158E0001409412000101D06701
:1080400009D02F0E016F100E006FF9EC44F0000103
:10805000F96B1200D007010E016F690E006FF9EC89
:1080600044F086A6120000F086A6120000F086A654
:10807000120011AA06D0010E0401D76FF40ED66FBC
:10808000E6D7330E0301EA6F080E0101CE6F00013F
:10809000F92B4FEF4BF00101CE2F15D09DEC3AF0AC
:1080A0000EE3118A010E0401D76FF40ED66F119EF4
:1080B0001C943C0E0201CE6F010E0101DD6F000128
:1080C000F96B95EF4DF00301F1330301F033030138
:1080D000EF330301EE330301ED330301EC3303010E
:1080E000EB330301EA330001F9075BEF47F00401CA
:1080F000EC6BED6B0101316B1BD056ECF1F018EC21
:108100004EF016E33EEC4EF00101326F0DD03251CD
:1081100079EC4AF00DE30101312B0AD032518FEC9A
:108120004AF006E3D88012003151F1E0010AF6E08E
:108130000401EC5101012F5D0401ED5101013059A1
:10814000DCE2D890120025291E6F000E26211F6F39
:10815000F6EC37F0276F25C11EF126C11FF1F6ECB2
:1081600037F0296F2751286F284B292B2829D8B49D
:10817000292902E1286B296B25C11DF126C11EF1B9
:1081800029511F6FE2EC3DF0010E010125251D6F05
:10819000000E26211E6F28C11FF1E2EF3DF075ECA5
:1081A0003EF0B96FB95102E0B95112001FA608D0D4
:1081B0000301BF6B14881A8417800001039E000C12
:1081C0000001188212EC2BF00101B96F1892B90569
:1081D00003E0B951030A0EE10301BF6B14881A844E
:1081E0001780039E0101B951030AE9E1010EFFEC7A
:1081F000CCF0000C020C9AEC49F01E6F20EE03F05C
:108200001C51D9261D51DA221EC1DFFF9AEC49F01C
:108210001E6F20EE02F01C51D9261D51DA221EC11C
:10822000DFFF9AEC49F01CC1D9FF1DC1DAFFDF6EF8
:108230009AEC49F01E6F20EE01F01C51D9261D5119
:10824000DA221EC1DFFF000109921200E8CF1DF102
:1082500001011D0505E1030E1C6FFB0E1B6F1200D3
:108260001D51020A06E1030E01011C6FFC0E1B6F7B
:1082700012001D51030A06E1030E01011C6FFD0EE1
:108280001B6F12001D51040A06E1030E01011C6F51
:10829000FE0E1B6F1200030E01011C6FFF0E1B6F01
:1082A0001200040E01011F6F030E1E6FF6EC37F073
:1082B000276F040E1F6F020E1E6FF6EC37F0296F4A
:1082C0002751286FFF0E285D000E295904E2040E85
:1082D000266F256F040C040E1F6F010E1E6FF6EC47
:1082E00037F0276F040E1F6F000E1E6BF6EC37F091
:1082F000266F2751256F1200E8CF1DF11D0506E1FD
:108300000A0E01011C6FA00E1B6F12001D51020A04
:1083100006E10B0E01011C6F000E1B6F12001D51B8
:10832000030A06E10B0E01011C6F500E1B6F1200B9
:108330001D51040A06E10B0E01011C6FA00E1B6FFC
:108340001200060E01011C6FF60E1B6F1200E8CF23
:1083500021F1206B226B0AD0E90E01012225D96E92
:10836000DA6A000EDA22DF50201B222B21C11BF11A
:108370001C6B22C11DF11E6B1DBF1E071E51800A02
:108380001F6F1B511D5D1C51800A1F59E5E3E90E4B
:1083900001012125D96EDA6A000EDA2220C1DFFF41
:1083A00012005B0E010120D8DB8E19AE03D05B0EEC
:1083B0001BD8DB8C960E0101D1251D6F1E6B020EA2
:1083C0001E235B0ED125D96EDA6A070EDA22DF5042
:1083D0001F6FE2EC3DF0530E0301ED6F100EEE6FD8
:1083E0000101D151FAEF41F0D125D96EDA6A070EB9
:1083F000DA22000CE8CF20F1060E0301EA6F01013A
:10840000CA510301EB6FC9C1ECF3EF6B5B0E0101C5
:108410002025D96EDA6A070EDA22DF501F6F1FADF2
:1084200005D020510F0B0301EE1304D02039F00BBF
:108430000301EF13F06BF16B030E01011D6FEA0EE8
:108440001C6F0BEF4AF09E940301E06B000117BE16
:1084500012000301DE9182ACDE81080EDF2BDF61AA
:1084600003D0D890DE37080CDF6BF40E0201EB2549
:10847000D96EDA6A030EDA22DEC3DFFFEB2B060EBB
:10848000EB65060CEB6B829C949C829C178E178C80
:108490008F800001148412000251040A02E0D89077
:1084A000120000C1D9FF01C1DAFFDF504E0AF7E127
:1084B00020EE01F00051D9260151DA22DF50100AD6
:1084C000EEE120EE02F00051D9260151DA22DF5010
:1084D0005E0AE5E120EE03F00051D9260151DA22CF
:1084E000DF50AC0ADCE1D8801200010E0101306FD0
:1084F000F40E2F6F77EC40F0F60E01011D6F6E0E3B
:108500001C6F010E13EC3CF0030E0101306FE80EFE
:108510002F6F77EC40F0F60E01011D6F620E1C6F9D
:10852000010E13EC3CF0030E0101306FE80E2F6FCB
:1085300077EC40F000011A9E1200E8CF5CF151C6C2
:108540001BF101015C516BEC49F002E2D890120082
:1085500045EC16F001015C39F00B5B6F020E466FC3
:108560005B5110EC07F006015151B6EC4DF002E200
:10857000D88012005C5185EC46F001015B6F5BC155
:1085800054F15C5123ECEDF0F3D7E8CF20F020500C
:108590002B0A03E10201C76B12001E0E0201C72560
:1085A000D96EDA6A070EDA2220C0DFFFC72BC75167
:1085B000160AD8A4120007011E51430A0AE11F51EE
:1085C000470A07E12051530A04E121514E0AD8B469
:1085D0001200000105941200DB6BDC6BBB2903E188
:1085E000390EDB6FDC6FBB51030A0BE1C0390F0B97
:1085F0005BEC4CF0DB6FC0510F0B5BEC4CF0DC6FB5
:108600001200BB51060A04E0BB51070AD8A41200AD
:10861000BF510F0B5BEC4CF0DB6FC0390F0B5BEC09
:108620004CF0DC6F1200E8CF27F127072751330DFC
:10863000890EF324286F130EF420296F2A6BFA0E8B
:1086400001012A25D96EDA6A0601060EDA2228C14E
:108650001EF129C11FF1F6EC37F0DF6E284B292BF4
:108660002A2B030E2A65EBD7060E0101266FFA0EA0
:10867000256F1200F294EB0E0101016F500E006F96
:10868000F9EC44F011B810D086B603D00101D06BDC
:1086900012000101D02BD051330AD8A41200D06BA4
:1086A00011880001118A120086B6F0D70101D02B83
:1086B000D051330AD8A41200D06B11980001118A4E
:1086C000120004012051800AD8A41200800E040177
:1086D000C46F13D0EB0E0401C36FDF0EC26F120E16
:1086E000C56F120CEB0E0401C36F9C0EC26F430EDC
:1086F000C56F430C0401C46B120004012351010A2D
:10870000E9E0030AEFE0010AD8A41200F3D71BC185
:1087100021F11CC122F102D0214B222B21C1D9FF12
:1087200022C1DAFFDF50F8E11D511F6F1E51206F8B
:108730001D4B1E2B1FC1F6FF20C1F7FF000EF86E68
:1087400021C1D9FF22C1DAFF214B222B0800F5CF2E
:10875000DFFFDF50D8B41200E7D704012051800AB0
:10876000D8A41200800E0401C46F13D0EB0E0401D4
:10877000C36FDF0EC26F120EC56F120CEB0E040139
:10878000C36F9C0EC26F430EC56F430C0401C46BD4
:10879000120004012351010AE9E0030AEFE0010A93
:1087A000D8A41200F3D7E8CF63F104C51BF101018F
:1087B00063516BEC49F002E2D890120045EC16F0E0
:1087C00001016339F00B626F790E466F625110EC54
:1087D00007F0000112862DEC4EF0DBEC33F01C921A
:1087E00017820201E25103E0E2050301D96FD8804C
:1087F0001200C76A300EC66E01011C6B1D6B1E6B2A
:108800001F6B550E206F63EC4BF01C6B010E1D6F40
:108810001E6B1F6BAA0E206F63EC4BF0000E1C6BDF
:108820001D6B1E6B1F6B63EC4AF0550AD8A4120037
:108830001C6B010E1D6F1E6B1F6B63EF4AF023C193
:108840001BF124C11CF125C11DF126C11EF1CCEC88
:1088500036F01BC129F11CC12AF123C11BF124C12F
:108860001CF125C11DF126C11EF17CEC3CF01BC1A1
:1088700027F11CC128F127C123F128C124F129C106
:1088800025F12AC126F112005B0E0101D125D96E16
:10889000DA6A070EDA22C00EDF165B0ED12512D877
:1088A00024AFD1EF41F05B0ED1250CD824AD05D01B
:1088B000000119BE1200D1EF41F0000119AE120003
:1088C000D1EF41F0D96EDA6A070EDA22DF50246F59
:1088D0001200206B216B1E511D111BE0010E1F6F3A
:1088E00004D0D8901D371E371F2B1EAFFAD7D89053
:1088F000203721371D511B5D1E511C5905E31D51A9
:108900001B5F1E511C5B2081D8901E331D331F2F0F
:10891000EED720C11BF121C11CF112000501FD5150
:10892000D8A41200000112BC1200206A0101E1A1CA
:1089300002D00684202A0101E1A302D00684202A65
:108940000101E1A502D00684202A206601D0069408
:1089500007BC02D015AC03D000010888120000014A
:1089600008981200FA0E01011D6F080E1C6F010E0F
:1089700013EC3CF042EC4EF00CD018EC4EF009E356
:108980003EEC4EF00101316F31513E0A02E1D890C8
:1089900012001FEC4EF0890E01012F5D130E3059AD
:1089A000ECE31B0E00EC4CF0D88012000101DD67F7
:1089B00002D0C1EF4CF0DD0502E1E0EF4CF0DD51FB
:1089C000020A02E1ABEF4DF0DD51030AF6E0DD51A2
:1089D000040AF8E0DD51050AF0E0DD51060A02E183
:1089E00072EF4DF0DD51070A02E10AEF4DF0DD6B49
:1089F0001200D59E0051026F0151036F046B056B8D
:108A000002510008066F000E0355076F010E045552
:108A1000086F000E0555096F07C106F108C107F17F
:108A200009C108F1096B08BF09690651D76E0051E9
:108A30000008D66ED58E12001BD0C7C4F6FFC8C47E
:108A4000F7FF000EF86EC9C4D9FFCAC4DAFF0F0ED3
:108A5000F76403D00800F55005D0F6CFE9FFF7CF53
:108A6000EAFFEF50DF6E0401C74BC82BC94BCA2B7E
:108A70000401CB07CB29D8B41200DFD71BD0C7C461
:108A8000F6FFC8C4F7FF000EF86EC9C4D9FFCAC408
:108A9000DAFF0F0EF76403D00800F55005D0F6CFCB
:108AA000E9FFF7CFEAFFEF50DF6E0401C74BC82B99
:108AB000C94BCA2B0401CB07CB29D8B41200DFD78E
:108AC000E8CF1BF11B0501E1010C1B51020A01E17A
:108AD000020C1B51040A01E1030C1B51080A01E1BD
:108AE000040C1B51100A01E1050C1B51200A01E185
:108AF000060C1B51400A01E1070C1B51800A01E1E1
:108B0000080C000CD1EC4DF00001128C51EC41F03E
:108B10000301D86B159A0101010E286F400E276FD3
:108B2000F90E2A6FBB0E296F140E2C6F550E2B6F8A
:108B300066ECD5F02751516F010E1C6F400E1B6F74
:108B400051C11DF1EEEF4CF030C131F11CD02CC100
:108B50001DF12DC11EF12EC11FF12FC120F131C118
:108B600021F16DEC2AF0326FCD51D8A412003251B0
:108B70002C27000E2D233251010DF3502E27000E0D
:108B80002F233251315F3167E2D712001E5133EC8F
:108B90004DF01E6F1F6B1EBF1F0710D01CC1D9FFE9
:108BA0001DC1DAFFDF5033EC4DF01E1905E11CC189
:108BB0001CF11DC11DF112001C4B1D2B1CC1D9FF46
:108BC0001DC1DAFFDF50EAE11C6B1D6B1200040EC1
:108BD00001011E6F1D6B1F6FE2EC3DF0040E0101E1
:108BE0001E6F010E1D6F040E1F6FE2EC3DF0040EB0
:108BF00001011E6F020E1D6F000E1F6BE2EC3DF0B7
:108C0000040E01011E6F030E1D6F1F6BE2EF3DF09E
:108C100086B613D000F086B610D000F086B60DD020
:108C2000010E0101016F690E006FF9EC44F00001C3
:108C3000F92B050E0101D06F050C2F0E0101016FFC
:108C4000100E006FF9EC44F0010E0001F96F010CF9
:108C5000E8CF1BF11C6B1BAF03D00001038802D0CF
:108C600000010398B2EC47F00101D8901B371C2B90
:108C70001C51800A780FEFE39FEC4BF0000103A634
:108C800012000101CD671200030ECD6F030C28C145
:108C900023F129C124F12AC125F12BC126F107ECCA
:108CA0003FF001012C6F0CA604D02CC1A9FFA8A293
:108CB000FED701012C6701D0000C400E2C6503D0BB
:108CC0002C51C90F12002C51D00F1200016B026BF6
:108CD000036B000E01010325D96EDA6A080EDA2251
:108CE000DF500127032B0E0E0365F3D702D00F0EC2
:108CF00002270151025DFBE30151025D006F006735
:108D000002D00F0E006F00511200E8CF28F10101D0
:108D10001F6B580E1E6FF6EC37F0276F2851030AB1
:108D200003E100011FBA010C28C125F1FF0E01016A
:108D3000252727C126F1252B02D0D8902633252FB1
:108D4000FCD72651010B1200000109B2120021C00C
:108D5000D9FF22C0DAFFDF500AEC49F020EE01F023
:108D60002150D9262250DA22DF500AEC49F020EEB9
:108D700002F02150D9262250DA22DF500AEC49F0C5
:108D800000010F8012002DC128F12EC129F12FC141
:108D90002AF130C12BF147EC46F0316F3139F00B3D
:108DA000326F2DC128F12EC129F12FC12AF130C116
:108DB0002BF147EC46F0322732510201D027010156
:108DC000325112002551241117E0010E266F04D0F4
:108DD000D89024372537262B25AFFAD72451225D8A
:108DE0002551235904E32451225F2551235BD89058
:108DF00025332433262FF2D722C122F123C123F1B8
:108E00001200E8CF1BF101011D6B1C6B9FEC4BF0B6
:108E10000101D8901D371D9103B61D811C2B1C51DB
:108E2000800A780FF3E31B5107E000010398B2ECCE
:108E300047F001011D51120000010388F8D7254BAE
:108E4000262B286BEB0E01012825D96EDA6A030E5A
:108E5000DA22DF50276F25511E6F26511F6F254BD9
:108E6000262BF6EC37F0271902E0D8901200282BB9
:108E7000050E2865E7D7D880050C636A626A9F0EE5
:108E80000F015D6F5E6B4D6B4E6BFB0E5C6F658C07
:108E90000401C46B0401C16B0401BD6B0401CD6B03
:108EA000659C160E0F014C6F02D06296040062B6EC
:108EB000FCD76598120086969896080E0101D06F2F
:108EC000D02FFED79886280ED06FD02FFED786A63B
:108ED00003D00301F18F02D00301F19F010E0101C4
:108EE000016FA50E006FF9EC44F00001F92B1200A0
:108EF000636A626A9F0E5D6F5E6B4D6B4E6BFB0E1D
:108F00005C6F658C0401C46B0401C16B0401BD6B13
:108F10000401CD6B659C160E0F014C6F02D062965A
:108F2000040062B6FCD765981200E8CF20F1010E6C
:108F30001F6F2051800A190F04E22051800A1F0F71
:108F40000DE22051800A390F04E22051800A3F0FC0
:108F500005E220519FEC4CF0D8A01F6B1FC11EF101
:108F60001E31120096929690000103A809D08482C7
:108F700084B209D00101CD6706D0020ECD6F03D0B7
:108F8000000103A884928D8000F08DB005D001010E
:108F9000CD6702D0010ECD6F8D9012004F0E1F6F66
:108FA000D40E1E6FF6EC37F0276F4F0E1F6FD50EE5
:108FB0001E6FF6EC37F0286F27512A6F2851296F62
:108FC00026512A1902E12551291902E1D8801200FF
:108FD000D8901200216B9AEC49F01E6F21511C258C
:108FE0001F6FE86A21BFE8681D21206F1FC1D9FFEC
:108FF00020C1DAFF1EC1DFFF212B2151800A790F2A
:10900000EAE39AEC49F0000109921200E8CF1BF163
:109010001BC1C2FFC280190E01011C6F1C07010198
:109020001C29FCE1C282320E1C6FC2A204D01C07B4
:1090300001011C29FAE1C450FC0B1C6FC26A1C51CF
:10904000120000C1D9FF01C1DAFFDF50060A02E0B9
:10905000D890120020EE01F00051D9260151DA22F9
:10906000180EDF6205D002510C0A02E1D88012000E
:1090700002510A0AFBE0ECD71DC11EF11F6B1B5108
:10908000010B1E1BD8901C331B331EA104D0010EF4
:109090001B1BA00E1C1BD8901E331F2B070E1F6519
:1090A000EED71BC11BF11CC11CF1070C216B9AEC04
:1090B00049F01E6F21511C251F6FE86A21BFE86827
:1090C0001D21206F1FC1D9FF20C1DAFF1EC1DFFFA4
:1090D000212B2151800A7D0FEAE300010992120041
:1090E000849296928D80969000F000F08DB005D01D
:1090F0000101CD6702D0010ECD6F848200F000F037
:1091000084B205D00101CD6702D0040ECD6F8D90E1
:1091100000F01200216B9AEC49F01E6F21511C25C2
:109120001F6FE86A21BFE8681D21206F1FC1D9FFAA
:1091300020C1DAFF1EC1DFFF212B2151800A7B0FE6
:10914000EAE3000109921200C7EC4BF001011D6F28
:109150001D5111E0A098040E0401C86F300EC76FB6
:109160001BC1C9F41CC1CAF41DC1CBF41CEC45F0F1
:10917000A08840EC4DF001011D511200216B9AECCA
:1091800049F01E6F21511C251F6FE86A21BFE86856
:109190001D21206F1FC1D9FF20C1DAFF1EC1DFFFD3
:1091A000212B2151800A7E0FEAE30001099212006F
:1091B0000101266B24C11DF125C11EF1EA0E01013A
:1091C0002625D96EDA6A030EDA22DF501F6FE2EC31
:1091D0003DF00101244B252B262B060E2665EAD7F0
:1091E000060CE8CF1BF1000E0001FB25D96EDA6AF0
:1091F0000E0EDA221BC1DFFFFB2BFB51F00AD8B4A5
:10920000FB6B0201D22BD251F00AD8A4120000014C
:1092100009821200E8CF20F0000E0001FB25D96E74
:10922000DA6A0E0EDA2220C0DFFFFB2BFB51F00AB8
:10923000D8B4FB6B0201D22BD251F00AD8A4120091
:10924000000109821200E8CF20F020C0C2FFC280D6
:10925000190E216E21062128FDE1C282320E216EF7
:10926000C2A203D021062128FBE1C450FC0B216ED1
:10927000C26A21501200010E0101256F5B0E01012F
:109280002525D96EDA6A070EDA22960E25251E6F7D
:109290001F6B020E1F23F6EC37F0DF6E252B0F0E2F
:1092A0002565ECD70F0C02510E0A02E0D89012008F
:1092B00000C1D9FF01C1DAFF070EDF6401D0F6D784
:1092C00020EE01F00051D9260151DA22010EDF62B1
:1092D000EDD7D880010CE8CF1EF101011E5103E04B
:1092E0001E51050A02E1D89012001EC11CF1FF0EAA
:1092F0001C271BC11DF11C2B02D0D8901D331C2F25
:10930000FCD71D31120002510B0A02E0D890120066
:1093100000C1D9FF01C1DAFFDF504E0AF7E120EEAC
:1093200001F00051D9260151DA22DF50610AEEE145
:10933000D8801200000E0201D425D96EDA6A0E0E12
:10934000DA22DF5001011B6F0201D42BD451F00A45
:10935000D8B4D46BD207D26701D00F9001011B5152
:10936000120002510D0A02E0D890120000C1D9FF8C
:1093700001C1DAFFDF504E0AF7E120EE01F00051A3
:10938000D9260151DA22DF50620AEEE1D8801200BC
:109390001D511BC1D9FF1CC1DAFFDF6205D01BC103
:1093A0001BF11CC11CF112001BC1D9FF1CC1DAFF4B
:1093B0001B4B1C2BDF50ECE11B6B1C6B12000001E4
:1093C00009B2120021C0D9FF22C0DAFFDF500AEC37
:1093D00049F020EE01F02150D9262250DA22DF5048
:1093E0000AEC49F000010F801200246A256A20A0CF
:1093F00004D02250242623502522D890223623360A
:10940000D8902132203221502010F1E124C020F0E8
:1094100025C021F01200000109B2120001011E6BEB
:109420001E511C25D96E000E1D21DA6EDF50F1ECA5
:1094300048F001011E2B070E1E65F2D700010F80B8
:10944000070CE8CF20F11E517CEC41F01BC121F14B
:109450001CC122F12051020DF3502125D96E000EBE
:109460002221DA6EDECF1EF1DDCF1FF11200E8CF30
:109470003DF101013D0508E1FA0E1C6FC00E1B6FA6
:10948000090E1D6FEEEF4CF0FA0E326FC00E316F09
:10949000346B090E336F9EEF0CF0E8CF3DF1010104
:1094A0003D0508E1F90E1C6FA50E1B6F0A0E1D6F1E
:1094B000EEEF4CF0F90E326FA50E316F346B0A0EE1
:1094C000336F9EEF0CF08B92030EF3EC4DF0010125
:1094D0001E51F3EC4DF001011D51F3EC4DF01C5108
:1094E000F3EC4DF0000EF3EC4DF0206F8B82205129
:1094F0001200E8CF1BF11B514F0A04E11BC1AFF36F
:10950000D89012001B514B0A07E10301AF514F0ADB
:1095100003E1AF6BD88012000301AF6BF1D7E8CF46
:109520001BF11B510D0A04E11BC1AEF3D8901200D0
:109530001B510A0A07E10301AE510D0A03E1AE6BAC
:10954000D88012000301AE6BF1D7E8CF3DF10101E5
:109550003D0508E1FB0E1C6FC10E1B6F080E1D6F51
:10956000EEEF4CF0FB0E326FC10E316F346B080E14
:10957000336F9EEF0CF01F6B206B1BA104D01D51AD
:109580001F271E512023D8901D371E37D8901C331B
:109590001B331C511B11F1E11FC11BF120C11CF138
:1095A00012008D9096908482969200F08D8000F04B
:1095B00000F08DB005D00101CD6702D0010ECD6F56
:1095C000849200F000F000F08D9000F01200E8CFDF
:1095D0003DF101013D0508E1F90E1C6FB00E1B6F56
:1095E0000A0E1D6FEEEF4CF0F90E326FB00E316FB8
:1095F000346B0A0E336F9EEF0CF09886080E010153
:10960000D06FD02FFED7CE2F06D0400ECE6F0001E8
:10961000F92B5BEF47F00301D890EA330001F9071B
:109620004FEF4BF00101D26706D0010ED26F0B84D1
:109630000201F06B1200D20506E1020ED26F0201A8
:10964000F06BEF6B1200D26B00010C821200000174
:1096500008BA050C000116B2050CFF0E0101326FAD
:10966000E10E316F000E346B336B9EEC0CF001E2B7
:10967000000CBBEF14F000010CA00CD00201D9517A
:10968000D8A4D907D9671200C8EC4DF0320ED96FB3
:10969000D72B320C46EC4EF00201D76B12008696A7
:1096A0009896080E0101D06FD02FFED70301EAB1C2
:1096B0009886010E0101016F870E006FF9EC44F0EE
:1096C0000001F92B12008B92020EF3EC4DF0010118
:1096D0001E51F3EC4DF001011D51F3EC4DF01C5106
:1096E000F3EC4DF02051F3EC4DF08B821200E8CFFB
:1096F0001DF1010E1C6F1D51200A09E01D51800A49
:10970000720F04E21D51800A770FD8A01C6B1CC198
:109710001BF11B311200040124510F0B080D000E28
:10972000F3240401C76FC86B040EC823040124AFDF
:109730001200040E0401C727000EC823000C9682F5
:109740009690000103968D8000F08DB005D0010148
:10975000CD6702D0010ECD6F00F084A202D00001CF
:1097600003868D901200040124510F0B080D000E8A
:10977000F3240401C76FC86B040EC823040124AF8F
:109780001200040E0401C727000EC823000C0401B8
:1097900018BF000C200E0401CD6101D0000CA0A860
:1097A000000C0401196703D040EC4DF0000C0401DB
:1097B00019511200E8CF1BF10301A86BA96B000E31
:1097C000A76F0A0EA66F00011E9C9EB803D0000171
:1097D0001EACFBD71BC1AEFF120024C1C9F125C1CD
:1097E000CAF11E6B590E1D6F25511F6FE2EC3DF043
:1097F00001011E6B5A0E1D6F24C11FF1E2EF3DF0F7
:10980000E8CF1BF10301A86BA96B000EA76F0A0E2E
:10981000A66F00011E9CA4B803D000011EACFBD7AC
:109820001BC1A9FF1200E8CF22F0216A090E2264B1
:1098300005D0212A0A0E225E2260FBD722C020F02A
:109840000F0E20162138F00B20101200040118BF53
:109850001200200E0401CD6101D0200CA0A812003E
:109860000401196702D026EF4DF0040119511200CE
:10987000E8CF1BF1600E01011B6503D01B51A90F3E
:109880001200400E1B6503D01B51C90F12001B5163
:10989000D00F1200E8CF22F0216A2250800A460F32
:1098A00006E22250800A500F02E3010E216E21C011
:1098B00020F020301200E8CF1BF10F0E01011B1722
:1098C0000A0E1B6104D0300E1B271B511200370EED
:1098D0001B2701011B5112004F0E1E6FD40E1D6F6E
:1098E00025511F6FE2EC3DF04F0E01011E6FD50EAA
:1098F0001D6F24C11FF1E2EF3DF01AAA0CD01A9A95
:109900008B9C0DA204D0320E0201F06F320C0F0EB0
:109910000201F06F0F0C1A8A8B8CF3D7D92F12002B
:1099200046EC4EF0230E0401E05D000EE159320ECC
:10993000D8B0FA0E0201D96F010ED76F010CE8CF33
:109940001DF11C6B1D51800A460F06E21D51800A55
:10995000500F02E3010E1C6F1CC11BF11B311200E2
:10996000E8CF1DF11C6B1D51800A250F06E21D5129
:10997000800A3F0F02E3010E1C6F1CC11BF11B315B
:1099800012000201D76702D0FBEF4DF0D70502E1CC
:109990003BEF4BF0D751020A02E18EEF4CF0D76B50
:1099A0001200FB0E01011D6F8B0E1C6F010E13ECDC
:1099B0003CF0130E0101306F880E2F6F77EF40F0EF
:1099C0000001FF51D8A4FF07FF671200C8EC4DF05B
:1099D0000101DD2B120E0001FF6F120C39EC4EF06D
:1099E0000009FCE11BC1B3F41CC1B4F41DC1B2F405
:1099F000010E0401B16F010C2DEC4EF0DBEC33F0E5
:109A000064ECB1F049EC25F05BECE6F01782000164
:109A10001C8212000001FF51D8A4FF07FF6712004B
:109A2000C8EC4DF00101DD07640E0001FF6F640C0E
:109A3000E8CF62F1000114A807D00101620504E13A
:109A4000FCEC4CF0D8801200D8901200400E0401BB
:109A5000181B040E1B6F300E1A6F400E196F18176B
:109A6000880E1813880CE8CF1BF11B51800A050FD4
:109A700005E21B51800A1F0FD8B01B9B1B5112001F
:109A8000400E0401181B040E1B6F300E1A6F400E9F
:109A9000196F1817880E1813880CE8CF1BF11B518B
:109AA000800A250F05E21B51800A3F0FD8B01B8B9F
:109AB0001B5112001BC1EAF41CC1EBF401D00400DD
:109AC0000401EB51EA11D8B41200F9D7E8CF28F01D
:109AD00028AA03D0216A900E02D0216A920E206E2D
:109AE00074EF23F00001FF2FC1EF4CF046EC4EF075
:109AF0000101DD6B0201D66BC1EF4CF086969896A2
:109B00000B0E0101016FC40E006FF9EC44F000016F
:109B1000F92B12000201D66702D0E3EF4DF0D60513
:109B200002E1EBEF4DF0D66B120098862F0E01018B
:109B3000016F100E006FF9EC44F00001F92B1200D8
:109B40009886010E0101016F870E006FF9EC44F059
:109B50000001F92B12000001FF2F120046EC4EF01D
:109B60000101DD2B090E0001FF6F090CE8CF1BF18D
:109B700001011BA902D0D8801200D8901200F092E7
:109B80005E0E776E786AA496A38600011784120091
:109B9000AA0ECB6E550EBC6ECC6ACA843F0EBB6E4D
:109BA0003F0C0401D56B0401CC9FA2883DEC47F02B
:109BB00000EF04F0A0B8A1A8120095ECF4F026EC98
:109BC0004CF0A198120000010BA81200C8EC4DF057
:109BD0000201D62B120000010BB8120046EC4EF029
:109BE0000201D66B1200E8CF1BF11BC1C9FFC7A051
:109BF000FED7C95012000CA08AEF4DF0320E0201C0
:109C0000D96FD72B320CE8CF1BF101011B51020198
:109C1000CB1B1200400E04011C1B1C17880E1C13CA
:109C2000880C1DC1F8FF1CC1F7FF1BC1F6FF120015
:109C3000000105B202D0D8901200D880120056EC74
:109C4000F1F0E2C42FF1E3C430F11200400E040140
:109C50001C1B1C17880E1C13880C14981C920301E3
:109C6000C16B00011B9C1200E8CF1BF11BC1F5F07A
:109C70001200A0A8010C0401B151120005920001CC
:109C8000F85112000401E26BE36B1200CA94BB6A44
:109C90001200FFFFFFFFFFFFFFFFFFFFFFFFFFFFC0
:109CA000FFFFFFFFFFFFFFFFFFFFFFFFFFFFFFFFC4
:109CB000FFFFFFFFFFFFFFFFFFFFFFFFFFFFFFFFB4
:109CC000FFFFFFFFFFFFFFFFFFFFFFFFFFFFFFFFA4
:109CD000FFFFFFFFFFFFFFFFFFFFFFFFFFFFFFFF94
:10EAC000FFFFFFFFFFFFFFFFFFFF30352F30312F2C
:10EAD00030312C30303A30303A30300051495552D4
:10EAE000433A2022636C6F7365642200434D5320C8
:10EAF0004552524F523A2031393300434D5320454D
:10EB000052524F523A2035313500434D452045523F
:10EB1000524F523A20313300434D45204552524F17
:10EB2000523A2031310051495552433A2022726500
:10EB300063762200434F4E4E454354204641494C94
:10EB40000051534D54505055543A202D0001000AA5
:10EB5000006400E80310274353513A20302C300062
:10EB60004352494E473A2000434D54493A2000430E
:10EB70005245473A2000434C4F53454400735F6C65
:10EB80006F636B002B43504252002B43504257009F
:10EB90002B434D4752002241434B220009024300C0
:10EBA000020100C064090400000102020000052403
:10EBB00000100104240202052406000105240100BE
:10EBC000010705820308000209040100020A00008F
:10EBD00000070503024000010705830240000112FF
:10EBE00001100102000008D8040A00010000000022
:10EBF000012B514654504346473D226163636F7574
:10EC00006E74222C22636F727465787570646174FF
:10EC100065222C2242647467246664764B220D00C0
:10EC2000432F25642E466C617368696E672120440A
:10EC30006F6E277420706F776572206F6666210D86
:10EC40000A002B514654504F50454E3D227570647A
:10EC50006174652E636F727465782E6C76222C3227
:10EC6000310D002B514655504C3D22757064617436
:10EC7000652E686578222C3336353030302C350DD2
:10EC8000002B515552434346473D22757263706FC6
:10EC90007274222C227561727431220D00446F77D8
:10ECA0006E6C6F616465642073756363657373660E
:10ECB000756C6C792E0D0A002E686578222C225511
:10ECC00046533A7570646174652E686578222C30FD
:10ECD0000D00436F6D6D616E64206E6F7420617600
:10ECE00061696C61626C652E0D0A00557067726116
:10ECF00064696E672E2E2E506C6561736520776196
:10ED000069742E002B51534D54504346473D227396
:10ED10006D7470736572766572222C22002B5143DC
:10ED200046473D226E777363616E6D6F6465222C7A
:10ED3000302C310D002B514654504346473D226341
:10ED40006F6E746578746964222C320D002B514902
:10ED50004346473D227064702F7265747279222C8D
:10ED6000302C310D002B51494346473D22706470D1
:10ED70002F7265747279222C312C310D002B515376
:10ED80004D54504346473D22636F6E7465787469F5
:10ED900064222C3100465450206469726563746F9C
:10EDA0007279206572726F722E0D0A00556E706C4A
:10EDB00075672074686520555342206361626C65F5
:10EDC0000D0A002B43504D533D22534D222C22530C
:10EDD0004D222C22534D220D00555047524144459F
:10EDE0003A4845582053495A45204552523B002B3A
:10EDF00051534D54504346473D226163636F756ED6
:10EE000074222C22002B51534D54504346473D222F
:10EE100073736C74797065222C3000446F776E6C5C
:10EE20006F6164696E67206572726F722E0D0A00E1
:10EE30002B514644454C3D227570646174652E68C3
:10EE40006578220D002B4347514D494E3D312C3002
:10EE50002C302C302C302C300D002B434751524598
:10EE6000513D312C302C302C302C302C300D002BDF
:10EE700051534D54504346473D2273656E6465724D
:10EE8000222C22002B51494F50454E3D312C312C24
:10EE900022544350222C220046545020736572762F
:10EEA0006572206572726F722E0D0A0023343A303B
:10EEB000323030303030323030303046430D0A009E
:10EEC000495320414C5245414459204C4F434B45F6
:10EED000440D0A002B51494F50454E3D312C302CEA
:10EEE00022544350222C22004469726563746F726D
:10EEF00079206572726F722E0D0A002B514955529E
:10EF0000433A202272656376222C302C00514955F9
:10EF100052433A202272656376222C312C3300232F
:10EF2000343A303030303030303146460D0A0D0A38
:10EF3000004D6F64656D206572726F7220302E2EE9
:10EF40000D0A004D6F64656D206572726F7220311D
:10EF50002E2E0D0A004D6F64656D206572726F7202
:10EF600020322E2E0D0A004D6F64656D2065727281
:10EF70006F7220332E2E0D0A0055504752414445E2
:10EF80003A48455820455252313B0055504752416E
:10EF900044453A48455820455252333B0055504766
:10EFA000524144453A54494D452D4F55543B002B51
:10EFB000434744434F4E543D312C224950222C228A
:10EFC000002B434E4D493D322C312C302C302C300F
:10EFD0000D002B43434C4B3D2230302F30312F302E
:10EFE000312C0053544154453A20434F4E4E454333
:10EFF000544544005761697420666F7220686578D3
:10F000002E2E0D0A0046696E616C2076657273695A
:10F010006F6E2E0D0A002B514654504357443D222B
:10F0200047543532220D002B514654504745543D2C
:10F030002247545F46353200554E53454E545F4289
:10F0400055465F46554C4C0D0051495552433A20A8
:10F050002272656376222C300051495552433A2082
:10F060002272656376222C31004350494E3A204E7D
:10F070004F5420494E534552004350494E3A204E7A
:10F080004F542052454144590053494D5320554E49
:10F090004C4F434B45440D0A002B514654504745B5
:10F0A000543D2247545F3532005550475241444544
:10F0B0003A4353204552523B0030362C25732C38AE
:10F0C00034303939303025640030372C25732C38F2
:10F0D00034303939303025640030362C25732C38E3
:10F0E00034313939303025640030372C25732C38D1
:10F0F00034313939303025640030362C25732C38C2
:10F100003538393930302564002B51534D54504433
:10F1100053543D312C312C2200434D452045525251
:10F120004F523A20313030004845582053495A4513
:10F13000204552520D0A002B514654504E4C535408
:10F140003D222E220D005465737454696D653A207A
:10F1500025642C200030362C25732C383530393975
:10F160003030300030372C25732C38353039393079
:10F1700030300030362C25732C383031393930306E
:10F18000300030362C25732C38323139393030305C
:10F190000030362C25732C3832323939303030007B
:10F1A00030372C25732C383232393930303000303A
:10F1B000362C25732C383233393930303000303624
:10F1C0002C25732C38303439393030300030362C1F
:10F1D00025732C38323439393030300030372C2513
:10F1E000732C38303839393030300030362C2573B4
:10F1F0002C38323939393030300030372C25732CE7
:10F2000038323939393030300030362C25732C38CB
:10F21000333339393032300030372C25732C3833C2
:10F220003339393032300030362C25732C383330B6
:10F2300039393030310030372C25732C38333039A0
:10F24000393030310030362C25732C383032393992
:10F250003030310030372C25732C3830323939308A
:10F2600030310030362C25732C3835343939303074
:10F27000310030362C25732C383535393930303162
:10F280000030372C25732C38353539393030310082
:10F2900030362C25732C3833303939303032003049
:10F2A000372C25732C383330393930303200303632
:10F2B0002C25732C38303239393030320030372C2D
:10F2C00025732C38303239393030320030362C2525
:10F2D000732C38353439393030320030362C2573C0
:10F2E0002C38353539393030320030372C25732CF5
:10F2F00038353539393030320030362C25732C38DA
:10F30000333039393030330030372C25732C3833D3
:10F310003039393030330030362C25732C383534C1
:10F3200039393030330030362C25732C38333039AE
:10F33000393030340030372C25732C38333039399C
:10F340003030340030362C25732C38353439393090
:10F3500030340030362C25732C3833303939303086
:10F36000350030372C25732C38333039393030356F
:10F370000030362C25732C38333039393030360094
:10F3800030372C25732C3833303939303036003053
:10F39000362C25732C383430393930256400303719
:10F3A0002C25732C38343039393025640030362C14
:10F3B00025732C38343139393025640030372C2509
:10F3C000732C38343139393025640030362C2573AC
:10F3D0002C3835383939302564002B51464C44538C
:10F3E0003D22554653220D00514654504F50454E34
:10F3F0003A20302C300051534D54505055543A203F
:10F40000302C3000434D45204552524F523A203166
:10F4100030004350494E3A2053494D2050494E0048
:10F4200049705254696D653A25646D2C2000415530
:10F43000544F20555047524144453A002B514944BE
:10F440004E534346473D312C22002B435343533DFB
:10F4500022495241220D0051534D5450424F4459BC
:10F460003A202D0051465450434C4F53453A2030DA
:10F470000051534D5450424F44593A203100434FAC
:10F480004E4E454354204641494C00762E25645F3C
:10F490006D6F6465300D0A00762E25645F6D6F64B4
:10F4A00065310D0A00484558205752204552520DEB
:10F4B0000A005349412049503A4F46462C20004704
:10F4C0007072734174743A25642C20004F4E2C28BE
:10F4D00025642064617973290030362C253033642B
:10F4E00039393030300030372C25303364393930F9
:10F4F00030300030362C3834303939303025640023
:10F5000030372C3834303939303025640030362CDF
:10F510003834313939303025640030372C383431C3
:10F520003939303025640030362C383538393930A7
:10F5300030256400222C22382E382E382E38220D09
:10F54000002B514953454E443D302C300D002B4982
:10F5500050523D31393230300D002B434F50533D26
:10F56000342C302C22002B5149434C4F53453D3114
:10F570000D00313630302039392030303000313311
:10F5800030312039392030303000333330312039B8
:10F5900039203030300031333032203939203030AA
:10F5A00030003333303220393920303030003136BA
:10F5B000303220393920303030003133393320397E
:10F5C000392030303000313134302039392030307A
:10F5D000310033313430203939203030310031318D
:10F5E0003430203939203030320033313430203952
:10F5F0003920303032003131343020393920303048
:10F600003300333134302039392030303300514920
:10F610004F50454E3A20302C300051494F50454E06
:10F620003A20312C300051494E49535441543A202C
:10F63000320051494F50454E3A20302C3500514947
:10F640004E49535441543A2037004350494E3A20D2
:10F650005245414459004953204C4F434B45440DBA
:10F660000A002B514944454143543D320D002B5172
:10F67000465450434C4F53450D0053746179412813
:10F680002564292C20005349412049503A4F4E2CE3
:10F6900020005154696D653A2564732C20004E6F2B
:10F6A00020557067726164652E0030362C38353015
:10F6B00039393030300030372C3835303939303046
:10F6C000300030362C383031393930303000303677
:10F6D0002C38323139393030300030362C38323233
:10F6E00039393030300030372C3832323939303017
:10F6F000300030362C383233393930303000303643
:10F700002C38303439393030300030362C383234FF
:10F7100039393030300030372C38303839393030E2
:10F72000300030362C38323939393030300030370B
:10F730002C38323939393030300030362C383333C8
:10F7400039393032300030372C38333339393032B0
:10F75000300030362C3833303939303031003037E2
:10F760002C38333039393030310030362C383032A3
:10F7700039393030310030372C3830323939303087
:10F78000310030362C3835343939303031003036AC
:10F790002C38353539393030310030372C38353563
:10F7A00039393030310030362C3833303939303057
:10F7B000320030372C38333039393030320030367F
:10F7C0002C38303239393030320030372C38303242
:10F7D00039393030320030362C3835343939303020
:10F7E000320030362C383535393930303200303748
:10F7F0002C38353539393030320030362C3833300A
:10F8000039393030330030372C38333039393030F3
:10F81000330030362C383534393930303300303617
:10F820002C38333039393030340030372C383330DD
:10F8300039393030340030362C38353439393030BD
:10F84000340030362C3833303939303035003037E9
:10F850002C38333039393030350030362C383330AD
:10F8600039393030360030372C3833303939303090
:10F870003600555047524144453A4F4B3B003036D5
:10F880002C38343039393025640030372C38343056
:10F8900039393025640030362C3834313939302547
:10F8A000640030372C383431393930256400303633
:10F8B0002C383538393930256400466F7263654F0E
:10F8C00066663A2564002B514944454143543D3115
:10F8D0000D002B5149444E534346473D22002B51C6
:10F8E00049435347503D312C33002B4346554E205E
:10F8F0003D20310D002B5149435347503D310D0000
:10F900002B4356455253494F4E0D002B51494E49FA
:10F91000535441540D0051534D54505055543A20B6
:10F9200000514654504357443A20300051465450F9
:10F930004745543A20300043475245473A20312C3E
:10F94000300043475245473A20312C31004347525B
:10F9500045473A20312C320043475245473A20313F
:10F960002C330043475245473A20312C340043475B
:10F970005245473A20312C3500434F4E4E454354B3
:10F98000204F4B0048455820455252310D0A00483F
:10F99000455820455252330D0A0049532057524FC3
:10F9A0004E470D0A00434F4445204552520D0A0070
:10F9B00053544154204552520D0A000D0A4743202A
:10F9C0007625640D0A002B514654504745543D227C
:10F9D00000504F5254313A25732C2000504F52544E
:10F9E000323A25732C2000504F5254333A25732C51
:10F9F00020007374616E646172742C200064696706
:10FA000069706C65782C20002B514953454E443D5C
:10FA1000300D002B51534D5450434C520D002B517F
:10FA20004953454E443D302C002B514953454E44DB
:10FA30003D312C002B43475245473D310D002B51A2
:10FA40004E57494E464F0D002241444D2D434944E7
:10FA50002200514453494D3A20302C00514453491F
:10FA60004D3A20312C00435245473A20312C30008A
:10FA7000435245473A20312C3100435245473A2002
:10FA8000312C3200435245473A20312C3300435247
:10FA900045473A20312C3400435245473A20312C17
:10FAA0003500514654504E4C53543A00434D452076
:10FAB0004552524F5200434D53204552524F52002F
:10FAC000434F4445204F4B0D0A00484558204552AE
:10FAD000520D0A00526573746172740D0A002B5145
:10FAE000494143543D320D0047454E4552414C2C4F
:10FAF0002000554E4B4E4F574E2C20004241542073
:10FB00004C4F572C20006D6167656C616E2C200096
:10FB1000756E6B6E6F776E2C20005365637572691E
:10FB200074793A002B51504F57443D310D002B5101
:10FB3000494143543D310D002B43474154543D311D
:10FB40000D0053454E44204641494C002B4353443D
:10FB5000483D300D002B434F50533D300D002B439B
:10FB60004D45453D310D002B435245473D310D007C
:10FB70002B434C49503D310D002B43475245473FE5
:10FB80000D002B434D47463D300D002B434D47465E
:10FB90003D310D002B5149535441540D0043474111
:10FBA00054543A20300043475245473A20310043ED
:10FBB000474154543A2031004445414354204F4B6F
:10FBC000004545204552520D0A00435320455252EC
:10FBD0000D0A002B4346554E3D300D002A23736914
:10FBE0006D5F6730004546463646303846006674DD
:10FBF000705F6C6F6164004C4E723A25642C20007B
:10FC000053413A2025732C2000534D3A2025732C64
:10FC10002000534E3A2025732C200053503A2025C3
:10FC2000732C20004950313A25732C200049503262
:10FC30003A25732C20004950333A25732C2000417B
:10FC4000504E3A25732C2000444E533A25732C20F5
:10FC5000005757573A25732C2000657370726974EA
:10FC60002C20002843524547256420004347524535
:10FC700047256420004E6F5F436172642900536919
:10FC80006D4C6F636B3A0050616E537461743A004F
:10FC90006125732C25730D0A002B514453494D3FA8
:10FCA0000D002B43474154543F0D002B4352433D1D
:10FCB000310D002B435245473F0D002B434F50530E
:10FCC0003F0D002B51434349440D002B4350494EF7
:10FCD0003D22002B43434C4B3D2200302E302E3032
:10FCE0002E30003A757064617465002B43434C4BB1
:10FCF0003F0D002B434D47533D22000A303030303A
:10FD0000303000435041533A2030004346554E3A7C
:10FD1000203100434F4E4E45435400455252256416
:10FD200029200044282564292C200070616E656C10
:10FD30002C20004C3A2025732C20004F6E6C696EED
:10FD4000653A0047454E4552414C00554E4B4E4F8B
:10FD5000574E002B4350494E3F0D002B4346554E06
:10FD60003F0D00514953454E443A0053454E4420FF
:10FD70004F4B00286E756C6C29002B435355420D78
:10FD8000002B43494D490D002B4347534E0D002B8B
:10FD90005147534E0D002B43474D520D002B5147F9
:10FDA0004D520D002B435042523D002B434D4753C3
:10FDB0003D00434C49503A2000435042523A200003
:10FDC000434F50533A2000432F25640D0A00442826
:10FDD00031292C200053494D312C200064736331AC
:10FDE0002C2000647363322C200042454C4C2C20A4
:10FDF00000475052532C2000414F66662C20004D86
:10FE00004F66662C20004C3A25732C2000503A2572
:10FE1000732C2000616275732C2000563A25643BD8
:10FE20002000434D4525642000434D5325642000A8
:10FE300053494D313A280028636F64652900557392
:10FE40006572733A004143544956450030303031B1
:10FE50003030002B4353510D002B3030220D0075F4
:10FE6000706F6666002C3134352C002C3132392C01
:10FE7000002B434D474400224E414B220043535137
:10FE80003A200043434C4B3A00434D47533A00510C
:10FE9000434349440053494D31200053494D3220DA
:10FEA0000023343A3130006D6F646530006D6F644B
:10FEB0006531006D6F64653F006E636F646500724D
:10FEC000656465660073696D5F6C00736669726D69
:10FED000002825642920002F256429200047534D40
:10FEE0002C2000414F6E2C20004D4F6E2C200028FE
:10FEF000747874290053494D313A004F5554313AC2
:10FF0000004F5554323A004D6F64653A00524543F4
:10FF10004F4E0053494D455200534D534552004DED
:10FF20003A202573002B434D450075706F6E0051CC
:10FF300047534E0033344342006C74616200737463
:10FF4000616200252E3264006C636667007363662D
:10FF500067006C6C6F67006C746D70006C74787403
:10FF60000073747874006E782C200025733B200099
:10FF70002F256429004F55543A002573293B004E24
:10FF80004F4E450047505253004441595300475289
:10FF90005354004D525354003030303800524459BD
:10FFA0000045310D004F4E2F004950310020553192
:10FFB000004950320020553200205533002055347E
:10FFC00000494E3A004F4646004255460047534DC1
:10FFD0000045525200444E5300282564002F2564EA
:10FFE00000510D0A00480D005530004C3000222C05
:10FFF0000039310041310023005B007C003E0000ED
:020000040001F9
:100000000101A26B65511B6F030E66151C6F1E6B01
:100010000E0E1D6FBBEC4AF0040E1B25A66F040EDE
:100020001C21A76F6651A56FA541E8423F0B070B46
:10003000A56FA6C125F1A7C126F1A7EC38F001E212
:10004000000C14A803D00101A5051FE01FAA04D0CD
:100050000101A551030A19E00101A55160ECE0F08E
:10006000EFE330C5A2F1AA6B0BD084EC8EF06B0EDF
:10007000AA25E16EE26A010EE222DFCFE7FFAA2B9A
:10008000050130510101AA5DF0E3BB054EE166AF09
:1000900034D0050130EC8EF015EC8EF0310EDF6EB1
:1000A000AA2B310EF0EC8DF0D1EC8DF0676F673933
:1000B0000F0B5BEC4CF0DF6EAA2BD1EC8DF00F0B2D
:1000C0005BEC4CF05CEC8EF0A965EED7310EE6EC03
:1000D0008DF0310EAA25FBEC8DF05BEC4CF002ECC0
:1000E0008EF05BEC4CF0DF6EAA2BAA514FEC06F0C1
:1000F00060EC8EF019EC2AF015D00501E68118A409
:1001000009D0010E0101246F000E23EC13F09AECCC
:100110008EF002D00101AA6BAA5167ECEAF002E26C
:100120000101A56B0101A5511200BB51020A4FE16B
:1001300066AF3AD0050130EC8EF015EC8EF0320E41
:10014000DF6EAA2B310EF0EC8DF0D1EC8DF0676FE5
:1001500067390F0B5BEC4CF0DF6EAA2BD1EC8DF006
:100160000F0B5BEC4CF05CEC8EF0A965EED7310E1A
:10017000E6EC8DF0030EA96FD1EC8DF0676F673957
:100180000F0B5BEC4CF0DF6EAA2BD1EC8DF00F0B5C
:100190005BEC4CF0DF6EAA2BA92B040EA965ECD703
:1001A000AA514FEC06F0A4D70501E68118A409D0A6
:1001B000010E0101246F000E23EC13F09AEC8EF077
:1001C00002D00101AA6BAA5167ECEAF0A8D7BB5193
:1001D000030A4FE166AF3AD0050130EC8EF015EC22
:1001E0008EF0330EDF6EAA2B310EF0EC8DF0D1ECD9
:1001F0008DF0676F67390F0B5BEC4CF0DF6EAA2B4D
:10020000D1EC8DF00F0B5BEC4CF05CEC8EF0A96543
:10021000EED7310EE6EC8DF0030EA96FD1EC8DF028
:10022000676F67390F0B5BEC4CF0DF6EAA2BD1ECDC
:100230008DF00F0B5BEC4CF0DF6EAA2BA92B050E9B
:10024000A965ECD7AA514FEC06F052D70501E6811B
:1002500018A409D0010E0101246F000E23EC13F045
:100260009AEC8EF002D00101AA6BAA5167ECEAF079
:1002700056D7BB51060A03E0BB51070A5CE166AFE3
:1002800047D00501E66B0101AA6BBB390F0B5BEC94
:100290004CF00501316F010115EC8EF0BB510F0BD5
:1002A0005BEC4CF0DF6EAA2B310EE6EC8DF0010E0C
:1002B000A96FD1EC8DF0676F67390F0B5BEC4CF0D9
:1002C000DF6EAA2BD1EC8DF00F0B5BEC4CF05CECED
:1002D0008EF0A965EED7310EE6EC8DF0030EA96F16
:1002E000D1EC8DF0676F67390F0B5BEC4CF0DF6E74
:1002F000AA2BD1EC8DF00F0B5BEC4CF0DF6EAA2B30
:10030000A92B060EA965ECD7AA514FEC06F0F0D642
:100310000501E68118A409D0010E0101246F000E29
:1003200023EC13F09AEC8EF002D00101AA6BAA51D3
:1003300067ECEAF0F4D6BB51080A01E083D066AF5F
:100340006ED00501E66B0101AA6BBB390F0B5BECAC
:100350004CF00501316F010115EC8EF0BB510F0B14
:100360005BEC4CF0DF6EAA2B310EE6EC8DF0010E4B
:10037000A96FD1EC8DF0676F67390F0B5BEC4CF018
:10038000DF6EAA2BD1EC8DF00F0B5BEC4CF05CEC2C
:100390008EF0A965EED7BE290DE0310E0101AA2528
:1003A000FBEC8DF05BEC4CF002EC8EF05BEC4CF077
:1003B000DF6EAA2B310EE6EC8DF01DEC8EF04E0EAA
:1003C000DF6EAA2BBF517C6FC0517B6FA36BA35113
:1003D0007B25A06F000E7C21A16F000EA05D800E1A
:1003E000A15902E3D50EA127A0C11EF1A1C11FF1A1
:1003F000F6EC37F09F6F9F6701D00DD0310E0101F1
:10040000AA25D96EDA6A050EDA229FC1DFFFAA2B70
:10041000A32BA329DCE1AA514FEC06F069D6050114
:10042000E68118A409D0010E0101246F000E23EC0F
:1004300013F09AEC8EF002D00101AA6BAA5167EC7E
:10044000EAF06DD6BB2901E0FBD5BEC1D7F1BE51A4
:10045000190A09E0BE51200A06E0BE51210A03E054
:10046000BE51220A2CE10501E66B010E0101A96FC4
:10047000BE51200A02E1020EA96FBE51210A02E11B
:10048000030EA96FBE51220A02E1040EA96FA95101
:1004900060ECE0F001E2D4D5AA6B07D084EC8EF0DA
:1004A000310EAA2522EC15F0AA2B050130510101CD
:1004B000AA5DF4E31DEC8EF0DF6AAFEF8DF0BE5164
:1004C000810A0AE1050138EC8EF0EC0E2A6FEB0E82
:1004D000296F66ECD5F00CD0BE51820A0DE1050102
:1004E00038EC8EF0F60E2A6F9E0E296F66ECD5F072
:1004F0002751A96FAFEF8DF0BE518A0A01E00DD1EF
:100500000501E66B050E010124EC8EF066ECD5F0DA
:100510002751A96FA9C1AAF11EBE23D00101A86B62
:100520000EEC8EF0CD0EA8251E6F1F6B000E1F2344
:10053000F6EC37F0DF6E0EEC8EF0DF5004E0A82B07
:100540000F0EA865EDD7310ECAEC8DF0FC0E2A6FA8
:10055000240E296F010E2C6F7F0E2B6F66ECD5F0E9
:100560001ED0310ECAEC8DF0FC0E2A6F510E296F91
:10057000080E2C6FD20E2B6F66ECD5F02751A96FA9
:10058000A951AA27310ECAEC8DF0FC0E2A6F480E35
:10059000296F070E2C6FA60E2B6F66ECD5F0E0ECE2
:1005A0008DF00EEC8EF0C80EA8251E6F1F6B000E8E
:1005B0001F23F6EC37F0DF6E0EEC8EF0DF5004E018
:1005C000A82B040EA865EDD7310ECAEC8DF0F90EFC
:1005D0002A6FD10E296F010E2C6F7F0E2B6F66ECE8
:1005E000D5F0E0EC8DF00EEC8EF08A0EA8251E6F93
:1005F0001F6B010E1F23F6EC37F0DF6E0EEC8EF052
:10060000DF5004E0A82B0F0EA865EDD7310ECAEC21
:100610008DF0FC0E2A6F2D0E296F010E2C6F7F0EB0
:100620002B6F66ECD5F0E0EC8DF00EEC8EF0850EC5
:10063000A8251E6F1F6B010E1F23F6EC37F0DF6E2F
:100640000EEC8EF0DF5004E0A82B040EA865EDD769
:10065000310ECAEC8DF0F90E2A6FDC0E296F010EF7
:100660002C6F7F0E2B6F66ECD5F0E0EC8DF00EEC6E
:100670008EF093EC8EF0F6EC37F0DF6E0EEC8EF031
:10068000DF5004E0A82B0F0EA865F1D7310ECAEC9D
:100690008DF0FC0E2A6F360E296F010E2C6F7F0E27
:1006A0002B6F66ECD5F0E0EC8DF00EEC8EF08CEC60
:1006B0008EF0F6EC37F0DF6E0EEC8EF0DF5004E0DB
:1006C000A82B040EA865F1D7310ECAEC8DF0F90EF7
:1006D0002A6FE70E296F010E2C6F7F0E2B6F66ECD1
:1006E000D5F02751A96FA951AA271F6B750E1E6F50
:1006F000F6EC37F0A96FD890A933030EA917310E85
:10070000CAEC8DF0F80E2A6FBA0E296FA9C12BF131
:100710002C6B66ECD5F0AFEF8DF0BE518B0A01E08B
:1007200011D10501E66B0101AA6B050E24EC8EF0D8
:1007300066ECD5F02751A96FA951AA27310ECAEC52
:100740008DF0F10E2A6F460E296FF2C22BF12C6B41
:1007500066ECD5F02751A96FA951AA27310ECAEC32
:100760008DF0F60E2A6F920E296FE1C22BF12C6BE1
:1007700066ECD5F02751A96FA951AA27310ECAEC12
:100780008DF0F40E2A6F220E296FE2C22BF12C6B32
:1007900066ECD5F02751A96FA951AA27310ECAECF2
:1007A0008DF0F40E2A6F200E296FDEC22BF12C6B18
:1007B00066ECD5F02751A96FA951AA27310ECAECD2
:1007C0008DF0F40E2A6FBF0E296FCBC32BF12C6B6B
:1007D00066ECD5F02751A96FA951AA271FA60AD008
:1007E000310ECAEC8DF0F60E2A6F860E296F66EC7C
:1007F000D5F009D0310ECAEC8DF0F40E2A6FB20E8E
:10080000296F66ECD5F02751A96FA951AA27310E9F
:10081000CAEC8DF0FB0E2A6FF70E296FD8C12BF1B1
:100820002C6B66ECD5F02751A96FA951AA27310E80
:10083000CAEC8DF0FE0E2A6FFB0E296F66ECD5F028
:100840002751A96FA951AA270DA60ED0310ECAECC7
:100850008DF0FA0E2A6FE80E296F66ECD5F027515D
:10086000A96FA951AA272ED00EAA0AD0310ECAEC20
:100870008DF0FE0E2A6FDD0E296F66ECD5F0EFD7F6
:100880000EA00AD0310ECAEC8DF0FD0E2A6FF10ECB
:10089000296F66ECD5F0E3D708AE0AD0310ECAEC6A
:1008A0008DF0FD0E2A6FEA0E296F66ECD5F0D7D7D2
:1008B000310ECAEC8DF0FA0E2A6FF20E296F66EC3B
:1008C000D5F0CDD7310ECAEC8DF0FF0E2A6F010E98
:1008D000296F66ECD5F02751A96FA951AA270DA859
:1008E0000FD0310ECAEC8DF0FD0E2A6F430E296F2A
:1008F00066ECD5F02751A96FA951AA27AFEF8DF06B
:100900000EAC0AD0310ECAEC8DF0FF0E2A6FCD0E60
:10091000296F66ECD5F0EED70EA20AD0310ECAECE4
:100920008DF0FF0E2A6F840E296F66ECD5F0E2D7AA
:10093000310ECAEC8DF0FD0E2A6F4B0E296F66EC5E
:10094000D5F0D8D7BE518C0A01E06AD10501E66B1B
:10095000050E010124EC8EF066ECD5F02751A96F4D
:10096000A9C1AAF1500E1F6FEA0E1E6FF6EC37F008
:10097000550A17E1310ECAEC8DF0F80E2A6F720E8F
:10098000296F66ECD5F02751A96F500E1E6FEA0E45
:100990001D6F000E1F6BE2EC3DF00101A951AA276B
:1009A0005AD0500E1F6FEA0E1E6FF6EC37F0430A56
:1009B0000AE1310ECAEC8DF0F00E2A6FA90E296FF4
:1009C00066ECD5F0E0D7500E1F6FEA0E1E6FF6EC06
:1009D00037F0470A0AE1310ECAEC8DF0EF0E2A6FAC
:1009E000790E296F66ECD5F0CED7500E1F6FEA0E48
:1009F0001E6FF6EC37F0410A0AE1310ECAEC8DF0B9
:100A0000EF0E2A6F8B0E296F66ECD5F0BCD7500E17
:100A10001F6FEA0E1E6FF6EC37F0530A0AE1310E33
:100A2000CAEC8DF0ED0E2A6FD90E296F66ECD5F069
:100A3000AAD7500E1F6FEA0E1E6FF6EC37F0540A5D
:100A40000AE1310ECAEC8DF0EF0E2A6F9D0E296F70
:100A500066ECD5F098D7310ECAEC8DF0FF0E2A6FF8
:100A60006B0E296F070E2C6F960E2B6F66ECD5F070
:100A70002751A96FA951AA27310ECAEC8DF0FF0E9C
:100A80002A6F6B0E296F090E2C6FB40E2B6F66EC5C
:100A9000D5F02751A96FA951AA27310ECAEC8DF0C4
:100AA000FF0E2A6F6B0E296F070E2C6F860E2B6FB1
:100AB00066ECD5F02751A96FA951AA27310ECAECCF
:100AC0008DF0FE0E2A6F300E296F66ECD5F0E0EC4B
:100AD0008DF00EEC8EF0ED0EA8251E6F1F6B000E34
:100AE0001F23F6EC37F0DF6E0EEC8EF0DF5004E0E3
:100AF000A82B080EA865EDD7310ECAEC8DF0FE0EBE
:100B00002A6F060E296F010E2C6F7F0E2B6F66EC7D
:100B1000D5F0E0EC8DF00EEC8EF0F60EA8251E6FF1
:100B20001F6B000E1F23F6EC37F0DF6E0EEC8EF01D
:100B3000DF5004E0A82B080EA865EDD7310ECAECF3
:100B40008DF0FE0E2A6F0D0E296F010E2C6F7F0E99
:100B50002B6F66ECD5F0E0EC8DF00EEC8EF0980E7D
:100B6000A8251E6F1F6B000E1F23F6EC37F0DF6EFB
:100B70000EEC8EF0DF5004E0A82B1A0EA865EDD71E
:100B8000310ECAEC8DF0FC0E2A6F3F0E296F010E5C
:100B90002C6F7F0E2B6F66ECD5F0E0EC8DF0370EEE
:100BA0000101A825D96EDA6A070EDA227F0EA82580
:100BB000E16EE26A010EE222DFCFE7FF0EEC8EF07B
:100BC000DF5004E0A82B130EA865E9D7310ECAEC5C
:100BD0008DF0FF0E2A6F7A0E296F010E2C6F7F0E9B
:100BE0002B6F66ECD5F02751A96F010E226F7F0E97
:100BF000216FFA0E246FB00E236F266B050E256F42
:100C0000EBEC2FF02251211101E076D6310ECAEC27
:100C10008DF0FC0E2A6F750E296F66ECD5F06AD642
:100C2000BE518D0A01E0C1D30501E66B050E01013D
:100C300024EC8EF066ECD5F02751A96FA9C1AAF17A
:100C4000310ECAEC8DF0FF0E2A6F070E296F66EC8D
:100C5000D5F02751A96FA951AA27DE670AD0310E16
:100C6000CAEC8DF0F90E2A6FF20E296F66ECD5F002
:100C700070D0DE51080A0AE1310ECAEC8DF0FE0E8A
:100C80002A6F140E296F66ECD5F063D0DE51040A8A
:100C90000AE1310ECAEC8DF0FC0E2A6F5A0E296F54
:100CA00066ECD5F056D0DE51060A0AE1310ECAECE8
:100CB0008DF0FB0E2A6F060E296F66ECD5F049D039
:100CC000DE510C0A0AE1310ECAEC8DF0FD0E2A6FDE
:100CD000DC0E296F66ECD5F03CD0DE51020A0AE149
:100CE000310ECAEC8DF0FD0E2A6F2B0E296F66ECCB
:100CF000D5F02FD0DE510A0A0AE1310ECAEC8DF090
:100D0000FD0E2A6FE30E296F66ECD5F022D0DE517E
:100D10000E0A0AE1310ECAEC8DF0F90E2A6FFD0EB3
:100D2000296F66ECD5F015D0DE050AE1310ECAEC6C
:100D30008DF0FF0E2A6F660E296F66ECD5F009D094
:100D4000310ECAEC8DF0FB0E2A6F100E296F66EC87
:100D5000D5F02751A96FA951AA27310ECAEC8DF001
:100D6000FE0E2A6FF50E296F66ECD5F02751A96F9C
:100D7000A951AA2713A80ED0310ECAEC8DF0FF0E90
:100D80002A6F7F0E296F66ECD5F02751A96FA95104
:100D9000AA2716D019A60AD0310ECAEC8DF0FF0E84
:100DA0002A6FD10E296F66ECD5F0EFD7310ECAEC61
:100DB0008DF0FE0E2A6F450E296F66ECD5F0E5D753
:100DC000310ECAEC8DF0FD0E2A6FD20E296F66EC43
:100DD000D5F02751A96FA951AA27310ECAEC8DF081
:100DE000F40E2A6F2E0E296F66ECD5F02751A96FED
:100DF000A951AA2707A435D00301AC510101676F9F
:100E00000301AD510101686F696B6A6B6751C008DE
:100E10001B6FA80E68551C6F000E69551D6F000EE4
:100E20006A551E6FA00E1F6F050E206F000E216BFE
:100E3000226BD2EC23F01BC17DF11CC17EF1310E7F
:100E4000CAEC8DF0F40E2A6FCC0E296F7DC12BF108
:100E50007EC12CF166ECD5F02751A96FA951AA27C4
:100E60000AD0310ECAEC8DF0FF0E2A6FC50E296F25
:100E700066ECD5F0F1D7310ECAEC8DF0FD0E2A6F7D
:100E8000D20E296F66ECD5F02751A96FA951AA2778
:100E9000310ECAEC8DF0FF0E2A6FC10E296F66EC81
:100EA000D5F02751A96FA951AA27E1A10DD0310E84
:100EB000CAEC8DF0FB0E2A6FAD0E296F66ECD5F0F3
:100EC0002751A96FA951AA27E1A30DD0310ECAEC71
:100ED0008DF0F60E2A6F300E296F66ECD5F0275193
:100EE000A96FA951AA27E1A50DD0310ECAEC8DF04A
:100EF000FA0E2A6F8C0E296F66ECD5F02751A96F78
:100F0000A951AA27E1A70DD0310ECAEC8DF0FA0E37
:100F10002A6F960E296F66ECD5F02751A96FA9515B
:100F2000AA27E1A90DD0310ECAEC8DF0F60E2A6F7A
:100F30003C0E296F66ECD5F02751A96FA951AA275D
:100F4000310ECAEC8DF0FD0E2A6FD20E296F66ECC1
:100F5000D5F02751A96FA951AA2707AC0DD0310EA2
:100F6000CAEC8DF0FA0E2A6FFC0E296F66ECD5F0F4
:100F70002751A96FA951AA27310ECAEC8DF0FF0E97
:100F80002A6F750E296F66ECD5F02751A96FA9510C
:100F9000AA278AAE0DD0310ECAEC8DF0F60E2A6F5C
:100FA000300E296F66ECD5F02751A96FA951AA27F9
:100FB0008AAC0DD0310ECAEC8DF0FB0E2A6FAD0E4F
:100FC000296F66ECD5F02751A96FA951AA27310ED8
:100FD000CAEC8DF0FD0E2A6FD20E296F66ECD5F0AB
:100FE0002751A96FA951AA2715A06BD0310ECAECC1
:100FF0008DF0FC0E2A6F870E296F66ECD5F0275115
:10100000A96FA951AA2709A00DD0310ECAEC8DF005
:10101000FD0E2A6FEA0E296F66ECD5F02751A96FF5
:10102000A951AA2701011F6B540E1E6FF6EC37F071
:10103000A46FA451F00B0BE1310ECAEC8DF0FD0E44
:101040002A6F230E3FEC8EF066ECD5F036D0A4511B
:10105000F00B100A0BE1310ECAEC8DF0F60E2A6F80
:101060007E0E3FEC8EF066ECD5F027D0A451F00B4D
:10107000200A0BE1310ECAEC8DF0FD0E2A6F230E13
:101080003FEC8EF066ECD5F018D0A451F00B300A8E
:101090000BE1310ECAEC8DF0F60E2A6F7A0E3FECA2
:1010A0008EF066ECD5F009D0310ECAEC8DF0FD0E55
:1010B0002A6FCE0E296F66ECD5F02751A96FA95182
:1010C000AA27310ECAEC8DF0FE0E2A6F3E0E296F54
:1010D00066ECD5F02751A96FA951AA27010E60EC43
:1010E000E0F029E3310ECAEC8DF0FF0E2A6FAD0E51
:1010F000296F66ECD5F02751A96FA951AA27010ED7
:1011000085EC46F000090AE1310ECAEC8DF0FE0EC6
:101110002A6FEF0E296F66ECD5F009D0310ECAECBC
:101120008DF0FE0E2A6F370E296F66ECD5F0275131
:10113000A96FA951AA27020E60ECE0F029E3310E55
:10114000CAEC8DF0FF0E2A6FB50E296F66ECD5F054
:101150002751A96FA951AA27020E85EC46F0000974
:101160000AE1310ECAEC8DF0FE0E2A6FEF0E296FE8
:1011700066ECD5F009D0310ECAEC8DF0FE0E2A6F68
:10118000370E296F66ECD5F02751A96FA951AA2710
:10119000030E60ECE0F029E3310ECAEC8DF0FF0E97
:1011A0002A6FB90E296F66ECD5F02751A96FA951A6
:1011B000AA27030E85EC46F000090AE1310ECAECBD
:1011C0008DF0FE0E2A6FEF0E296F66ECD5F009D078
:1011D000310ECAEC8DF0FE0E2A6F370E296F66ECC9
:1011E000D5F02751A96FA951AA27040E60ECE0F0B1
:1011F00029E3310ECAEC8DF0FF0E2A6FBD0E296F68
:1012000066ECD5F02751A96FA951AA27040E85ECE9
:1012100046F000090AE1310ECAEC8DF0FE0E2A6F8D
:10122000EF0E296F66ECD5F009D0310ECAEC8DF0C7
:10123000FE0E2A6F370E296F66ECD5F02751A96F85
:10124000A951AA27310ECAEC8DF0FD0E2A6FD20EDD
:10125000296F66ECD5F02751A96FA951AA27310E45
:10126000CAEC8DF0FB0E2A6F1A0E296F66ECD5F0D2
:101270002751A96FA951AA274F0E1F6FD30E1E6FBA
:10128000F6EC37F0676F67AD0AD0310ECAEC8DF01F
:10129000F60E2A6F8D0E296F66ECD5F009D0310E4F
:1012A000CAEC8DF0F40E2A6FB90E296F66ECD5F0FA
:1012B000E0EC8DF0310ECAEC8DF0FC0E2A6F7E0E44
:1012C000296F66ECD5F02751A96FA951AA27000E06
:1012D00017EC0FF000090FE0310ECAEC8DF0FD0E97
:1012E0002A6FD50E296F66ECD5F02751A96F010E34
:1012F000A86FA951AA270101A86710D0310EAA250D
:10130000276F286B050E2823F40E2A6FB90E296F5C
:1013100066ECD5F02751A96FA951AA27310ECAEC66
:101320008DF0FD0E2A6F3B0E296F66ECD5F027512C
:10133000A96FA951AA2714A823D0310ECAEC8DF0A9
:10134000FF0E2A6FA50E296F66ECD5F02751A96F05
:10135000A951AA270AA20AD0310ECAEC8DF0FF0EBD
:101360002A6FB10E296F66ECD5F0F9D3310ECAECB5
:101370008DF0FF0E2A6FA90E296F66ECD5F0EFD322
:1013800017A00AD0310ECAEC8DF0FF0E2A6F0D0E99
:10139000296F66ECD5F0E3D3310EFCDBFF0E2A6F2C
:1013A000C50E296F66ECD5F0DAD3BE518E0A01E086
:1013B000E4D00501E66B1FAA0CD0050E0101286FD1
:1013C000310E276FFE0E2A6FE90E296F66ECD5F0FD
:1013D0000BD0050E0101286F310E276FFD0E2A6F0D
:1013E000FF0E296F66ECD5F02751A96FA9C1AAF1AC
:1013F000A86B0EEC8EF093EC8EF0F6EC37F0DF6E0F
:101400000EEC8EF0DF5004E0A82B1F0EA865F1D77C
:10141000310EC0DBFC0E2A6F000E296F010E2C6FFF
:101420007F0E2B6F66ECD5F0CBDBF8DB8CEC8EF00F
:10143000F6EC37F0DF6EF2DBDF5004E0A82B050E90
:10144000A865F3D7310EA6DBFC0E2A6F1B0E296FA1
:10145000010E2C6F7F0E2B6F66ECD5F0B1DBDEDB5F
:10146000C00EA8251E6F1F6B010E1F23F6EC37F070
:10147000DF6ED4DBDF5004E0A82B1F0EA865EFD78A
:10148000310E88DBFD0E2A6F330E296F010E2C6F93
:101490007F0E2B6F66ECD5F02751A96FA951AA27B3
:1014A0001FA809D0310E76DBFE0E2A6FE30E296FDE
:1014B00066ECD5F008D0310E6DDBFD0E2A6FF80E0C
:1014C000296F66ECD5F07CDBA9DBF10EA8251E6F39
:1014D0001F6B010E1F23F6EC37F0DF6E9FDBDF5032
:1014E00004E0A82B0F0EA865EFD7310E53DBFC0EDE
:1014F0002A6F120E296F010E2C6F7F0E2B6F66EC78
:10150000D5F05EDB8BDBA8291E6F1F6B020E1F233D
:10151000F6EC37F0DF6E82DBDF5004E0A82B1F0E05
:10152000A865F0D7310E36DBFC0E2A6F090E296F45
:10153000010E2C6F7F0E2B6F66ECD5F041DB6EDB5E
:10154000210EA8251E6F1F6B020E1F23F6EC37F02D
:10155000DF6E64DBDF5004E0A82B1F0EA865EFD719
:10156000310E18DBFF0E2A6F1F0E296F010E2C6F34
:101570007F0E2B6F66ECD5F0F2D2BE518F0A01E0E0
:1015800069D20501E66B0101AA6B050E286F310EC9
:10159000276FFF0E2A6F890E296F66ECD5F0275151
:1015A000A96FA951AA27500E1F6FBF0E1E6FF6EC30
:1015B00037F0676F500E1F6FBE0E1E6FF6EC37F0E0
:1015C000A76F6751A66F310EE5DA64DB66ECD5F0E4
:1015D0002751A96FA951AA27500E1F6FC10E1E6F68
:1015E000F6EC37F0676F500E1F6FC00E1E6FF6ECF3
:1015F00037F0A76F6751A66F310ECCDA54DB66EC7B
:10160000D5F02751A96FA951AA27310EC3DAFF0ED1
:101610002A6FA90E296F66ECD5F02751A96FA95141
:10162000AA27500E1F6FC50E1E6FF6EC37F0676FBE
:10163000500E1F6FC40E1E6FF6EC37F0A76F675188
:10164000A66F310EA7DA26DB66ECD5F02751A96F1D
:10165000A951AA27500E1F6FC30E1E6FF6EC37F06C
:10166000676F500E1F6FC20E1E6FF6EC37F0A76F3C
:101670006751A66F310E8EDA2DDB66ECD5F027515F
:10168000A96FA951AA27500E1F6FCB0E1E6FF6EC43
:1016900037F0676F500E1F6FCA0E1E6FF6EC37F0F3
:1016A000A76F6751A66F310E75DAFDDA66ECD5F0DB
:1016B0002751A96FA951AA27310E6CDAFF0E2A6FA4
:1016C000B10E296F66ECD5F02751A96FA951AA2751
:1016D000500E1F6FC90E1E6FF6EC37F0676F500E7D
:1016E0001F6FC80E1E6FF6EC37F0A76F6751A66F1D
:1016F000310E50DACFDA66ECD5F02751A96FA95137
:10170000AA27500E1F6FC70E1E6FF6EC37F0676FDB
:10171000500E1F6FC60E1E6FF6EC37F0A76F6751A5
:10172000A66F310E37DAD6DA66ECD5F02751A96FFD
:10173000A951AA27500E1F6FCD0E1E6FF6EC37F081
:10174000676F500E1F6FCC0E1E6FF6EC37F0A76F51
:101750006751A66F310E1EDAA6DA66ECD5F0275176
:10176000A96FA951AA27310E15DAFF0E2A6F130EA1
:10177000296F66ECD5F02751A96FA951AA27500E01
:101780001F6FCF0E1E6FF6EC37F0676F500E1F6F96
:10179000CE0E1E6FF6EC37F0A76F6751A66F310EB5
:1017A000F9D978DA66ECD5F02751A96FA951AA27A3
:1017B000500E1F6FD10E1E6FF6EC37F0676F500E94
:1017C0001F6FD00E1E6FF6EC37F0A76F6751A66F34
:1017D000310EE0D968DA66ECD5F02751A96FA9512E
:1017E000AA27310ED7D9FF0E2A6F190E296F66EC82
:1017F000D5F02751A96FA951AA27500E1F6FE30EEC
:101800001E6FF6EC37F0676F500E1F6FE20E1E6F03
:10181000F6EC37F0A76F6751A66F310EBBD963DACC
:1018200066ECD5F02751A96FA951AA27310EB2D97C
:10183000FF0E2A6FC90E296F66ECD5F02751A96FEC
:10184000A951AA27500E1F6FE10E1E6FF6EC37F05C
:10185000676F500E1F6FE00E1E6FF6EC37F0A76F2C
:101860006751A66F310E96D93EDA66ECD5F0275156
:10187000A96FA951AA27310E8DD9FF0E2A6F8E0E9E
:10188000296F66ECD5F02751A96FA951AA27500EF0
:101890001F6FDB0E1E6FF6EC37F0676F500E1F6F79
:1018A000DA0E1E6FF6EC37F0A76F6751A66F310E98
:1018B00071D9FC0E2A6F630E296FA6C12BF1A7C147
:1018C0002CF166ECD5F02751A96FA951AA27500E2B
:1018D0001F6FDD0E1E6FF6EC37F0676F500E1F6F37
:1018E000DC0E1E6FF6EC37F0A76F6751A66F310E56
:1018F00051D9FC0E2A6F6C0E296FA6C12BF1A7C11E
:101900002CF166ECD5F02751A96FA951AA27500EEA
:101910001F6FD70E1E6FF6EC37F0676F500E1F6FFC
:10192000D60E1E6FF6EC37F0A76F6751A66F310E1B
:1019300031D9FE0E2A6F220E296FA6C12BF1A7C145
:101940002CF166ECD5F02751A96FA951AA27500EAA
:101950001F6FD90E1E6FF6EC37F0676F500E1F6FBA
:10196000D80E1E6FF6EC37F0A76F6751A66F310ED9
:1019700011D9FE0E2A6F290E296FA6C12BF1A7C11E
:101980002CF166ECD5F02751A96FA951AA27500E6A
:101990001F6FDF0E1E6FF6EC37F0676F500E1F6F74
:1019A000DE0E1E6FF6EC37F0A76F6751A66F310E93
:1019B000F1D8FD0E2A6F1B0E296FA6C12BF1A7C10E
:1019C0002CF166ECD5F02751A96FA951AA27310E49
:1019D000E1D8FF0E2A6F930E296F66ECD5F02751E0
:1019E000A96FA951AA27500E1F6FD30E1E6FF6ECD8
:1019F00037F0676F500E1F6FD20E1E6FF6EC37F088
:101A0000A76F6751A66F310EC5D844D966ECD5F0E3
:101A10002751A96FA951AA27500E1F6FD50E1E6F0F
:101A2000F6EC37F0676F500E1F6FD40E1E6FF6EC9A
:101A300037F0A76F6751A66F310EACD8FF0E2A6F33
:101A4000700E296FA6C12BF1A7C12CF166ECD5F061
:101A50007AEF84F00201F55127E00101BE51260A18
:101A600009E0BE51270A06E0BE51280A03E0BE5134
:101A7000290A75E10201F50506E1050E01013CD9CF
:101A800066ECD5F00ED0F551020A0BE1050E01010E
:101A9000286F310E276FFA0E2A6FB00E296F66EC91
:101AA000D5F00201F56B5BD00101BE51300AD8B40C
:101AB00066BF05D0050E20D966ECD5F050D066AFD4
:101AC00037D00501E66B00011FA62ED00101AA6BDD
:101AD000660E0501316F0101A8D8660EDF6EAA2BD4
:101AE000310E7ED85ED8676F67390F0B5BEC4CF018
:101AF000DF6EAA2B56D80F0B5BEC4CF0DDD8A96536
:101B0000F1D7310E63D8310EAA2575D85BEC4CF0B5
:101B100079D85BEC4CF0DF6EAA2BAA514FEC06F0A3
:101B2000CFD819EC2AF01BD0000E49ECC1F017D029
:101B30000501E68118A408D0010E0101246F000EF2
:101B400023EC13F0F7D802D00101AA6BAA5149EC9B
:101B5000C1F0AA5167ECEAF002E20101A56BA2C153
:101B600030F50101AA6B10D06B0EAA25D96EDA6A86
:101B7000010EDA22200E0101AA25E16EE26A050EAD
:101B8000E222DFCFE7FFAA2BA251AA5D02E392EF88
:101B900080F0EAD70101AA25276F286B050E2823BC
:101BA0001200310E0101AA25D96EDA6A050EDA2279
:101BB000BB0EA925E16EE26A010EE222E750120097
:101BC0002751A96FA951AA27A86B12000101AA25C4
:101BD000D96EDA6A050EDA222C0EDF6EAA2B2C0CD7
:101BE000AA25D96EDA6A050EDA222C0EDF6EAA2B30
:101BF000010EA96F010CD96EDA6A050EDA22BE3920
:101C00000F0B1200DF6EAA2B310E0101AA25D96E2F
:101C1000DA6A050EDA22BE510F0B12007F0EA825DC
:101C2000D96EDA6A010EDA221200AA2B310EAA2529
:101C3000D96EDA6A050EDA221200310EAA25D96EA3
:101C4000DA6A050EDA221200286F310E276FFE0EB7
:101C50002A6F1B0E296F140E2C6F550E2B6F550C0F
:101C6000E66B0101AA6B300E0501316F0101300CEA
:101C7000E66B050E0101286F310E276F1200296FE8
:101C8000A4C167F10F0E671767292B6F2C6B000E2D
:101C90002C23000CFF0E2A6FD90E296FA6C12BF141
:101CA000A7C12CF11200FE0E2A6FD70E296FA6C114
:101CB0002BF1A7C12CF11200DF6EAA2BA92B020C6D
:101CC0003F0E0101AA25D96EDA6A0501050EDA2256
:101CD000DF6A000CFF0E2A6FDD0E296FA6C12BF103
:101CE000A7C12CF11200FE0E2A6FD10E296FA6C1DA
:101CF0002BF1A7C12CF11200286F310E276FFD0EBA
:101D00002A6F700E296F1200200E0101AA25D96ECC
:101D1000DA6A050EDA221200BA0EA8251E6F1F6BB2
:101D2000010E1F23010C9A0EA8251E6F1F6B010EBA
:101D30001F23010C090E0101AA6F090C340E0501C5
:101D4000FE6F4086FC69408240804084060EFD6F35
:101D50002BEC18F0E36B1AD083500F0BDE6F270EBD
:101D6000CC6F100ECB6F01D004000101CB07D8A0BF
:101D7000CC07CB29D8B4CC29F7E183500F0BDE195F
:101D800004E0E35103E0E30701D0E32BE3510A0A47
:101D9000E3E1DE6BDE6705D01880949C829C94841E
:101DA00050D0DE51040A10E10B8E949C9484AD94C3
:101DB0007E86090E7F6EC20EB06EAC8EAC88AD8A88
:101DC0009E9A9F9A9D8A3DD0DE51060A02E11282B8
:101DD0002DD0DE510E0A08E10A86949C9484AD94BD
:101DE0007E867F6A340EE8D7DE0508E1138EF1881F
:101DF000F092F08EF088060E766E23D0DE510A0A3D
:101E000003E0DE510C0A0AE1108A0101DE510A0AE0
:101E100001E1108CF19CF292F28813D0DE51080A95
:101E20000DE10001058A3BEC49F09896949C94845E
:101E3000AD947E86010E7F6E370EBED7DE51020A4C
:101E4000ABE0080E0101E36F8D968D948A988A9617
:101E50008D9C8D9A8D8C8D8A8D868D848A888A86BC
:101E60008F808F808C8AEA0ECC6F600ECB6F01D092
:101E700004000101CB07D8A0CC07CB29D8B4CC29CA
:101E8000F7E18D9C8D9A8D968D948A988A968F9085
:101E90008F908C9AEA0ECC6F600ECB6F01D004004D
:101EA0000101CB07D8A0CC07CB29D8B4CC29F7E1C6
:101EB000E32FD0D7D08EF28EF28C1F6BFF0E1E69EF
:101EC000F6EC37F00501FE1916E001011F6BFF0E5D
:101ED0001E69F6EC37F00501FE190DE03BECE5F06C
:101EE00001011E6BFF0E1D69FEC51FF1E2EC3DF006
:101EF000010E0101E36F64ECB1F0130E01011F6FDD
:101F0000890E1E6FF6EC37F00701E66FE629D8B4AC
:101F10008F800601C55113E0060E0101226FC50E28
:101F2000216FFC0E246FDB0E236F266B070E256FCF
:101F3000EBEC2FF02251211102E01FA60F880701C0
:101F4000A65102E01FA60F88F4C4CBF1F5C4CCF172
:101F50000401F56B020EF46F0001409442EC4EF068
:101F60001FEC4EF03D0E01012F5D000E3059F8E3DD
:101F7000CBC1F4F4CCC1F5F413EC36F0D66B158E6E
:101F80001680048E00010580F9EC43F086CFE2F163
:101F9000E2A916D0270ECC6F100ECB6FCB07D8A0BE
:101FA000CC070101CB29D8B4CC29F8E186CFE2F1E6
:101FB000E2A906D000010F8E000E82EC45F04CD055
:101FC000AEECCAF013BC48D01B8C179E1684500E82
:101FD00001011E6FC00E1D6F000E1F6BE2EC3DF085
:101FE000500E01011E6FC10E1D6F000E1F6BE2EC43
:101FF0003DF044ECECF019A822D08D8C8D8AEA0ECD
:102000000101CC6F600ECB6F01D000F00101CB0756
:10201000D8A0CC07CB29D8B4CC29F7E18D9C8D9AD8
:10202000EA0ECC6F600ECB6F01D000F00101CB0740
:10203000D8A0CC07CB29D8B4CC29DFE0F6D78A8248
:10204000020E0101D46F099A099EF19CF292F28866
:1020500000011AA084ECBDF012BC15AA01D00F82B9
:1020600012AC05D000010FA202D0FF00FFD7000183
:1020700012AC05D08D8C8D9A010EB5ECB5F012BC6A
:102080000FAE15D086CFE2F10101E2B910D0270ED4
:10209000CC6F100ECB6FCB07D8A0CC070101CB299A
:1020A000D8B4CC29F8E186CFE2F1E2A9FF0012BC56
:1020B0001BD086CFE2F10101E2A916D0270ECC6F2A
:1020C000100ECB6FCB07D8A0CC070101CB29D8B419
:1020D000CC29F8E186CFE2F1E2A906D000010F8E0B
:1020E000010E82EC45F0B8D704B016A40BD01694BC
:1020F0008D9C168A18A006D0040EBB6E9E949F94E9
:102100009D84948C000112BC09D045EC0DF00301B4
:10211000E66FE65103E0E651FFECCCF014AA06D0DE
:102120000301D56703D0DBEC33F0149A040E0301EE
:10213000C9650AD0C96B500E0101266FDE0E256FEE
:10214000A3EC40F0AEECCAF003A403D00394030167
:10215000BF2B040E0301BF650AD0BF6B500E0101F7
:10216000266FDE0E256FA3EC40F0AEECCAF002AA9B
:1021700009D0500E0101266FD60E256FA3EC40F05A
:10218000AEECCAF002A809D0500E0101266FD60E9F
:10219000256FA3EC40F0AEECCAF002AC10D0029C6C
:1021A0000301BD2B010EBD650AD0BD6B500E0101B0
:1021B000266FD80E256FA3EC40F0AEECCAF002AE4D
:1021C00010D0029E0301BE2B010EBE650AD0BE6B6D
:1021D000500E0101266FD80E256FA3EC40F0AEEC37
:1021E000CAF003AC04D00001039C5BECE6F00AA447
:1021F0000FD00A94500E0101266FBE0E256FA3EC7E
:1022000040F0500E0101266FC00E256FA3EC40F088
:1022100012AC0FA071D017BE6FD00BAE17D0030E4B
:1022200001011D6FF40E1C6FBEEC48F0030E01019E
:102230002D6FF40E2C6F05ECDDF05EE2030E010154
:102240001C6FF40E1B6F44EC37F054D012A20FD069
:10225000030E01011D6FF40E1C6F56EC48F0030EC7
:102260000101266FF40E256F3EECDBF0E7D70AA6DE
:102270000FD0030E01011D6FF40E1C6F56EC48F0D9
:10228000030E0101306FF40E2F6FB3ECDEF0D5D7E3
:1022900010AA0FD0030E01011D6FF40E1C6FFBEC92
:1022A00040F0030E01012D6FF40E2C6F1CECC8F0F2
:1022B000C4D713AE0FD0030E01011D6FF40E1C6FB7
:1022C0008AEC48F0030E0101256FF40E246FE2EC56
:1022D0000DF010D005BA05B60FD0030E01011D6F29
:1022E000F40E1C6FEAEC47F00301F451080A02E116
:1022F000058602D0178E178C12AC10AA3FD00101B0
:10230000D051080A25E110BC06D00301EA51EB0ABE
:102310001FE10D801DD00101CFB51AD0CFA30FD082
:102320000301EA51A50A14E0020E0101CF170301CF
:10233000EA51EB0A0DE1040E0101CF6F09D0030150
:10234000EA51A50A05E10101CFB1E3D7CF81CF83DF
:102350001BB60BD01BA403D01B940301E46B030139
:10236000E4A70CD01B86158609D00D801BA406D0CF
:102370001B940301E46B1B9611A2158812AC05AAED
:1023800091D017BA29D00101D3678CD005A611D0FE
:102390000588F7C31CF1F5C31DF1010E1E6F030183
:1023A000F651BDEC1BF0178A059CF00E0101D36FAE
:1023B00079D00301B12B450E01011C6FB1C31DF192
:1023C0001E6B540EBDEC1BF00301B1510F0AEBE183
:1023D000B16B8F801484E7D70101D3670AD0179AB5
:1023E000000105B803D001EC26F05CD005980596F5
:1023F00059D005AC57D005A802D005980596059C84
:10240000179A0301EA51240A06E0EA515E0A03E042
:10241000EA51260A30E1EA51240A02E1199E04D069
:10242000EA515E0A03E1198E059E02D0199E058EBF
:102430000301B25123EEEBF0DF621DD00101CE515A
:10244000120A03E0CE51060A16E1CE51D5EC35F062
:1024500012E30301EB5138EC4CF0D16FCE51120A6C
:102460001EE109A20BD0150E01011C6FB1C31DF1B5
:102470001E6BBDEC1BF001EC26F097D7060E010198
:102480001C6FB1C31DF11E6BBDEC1BF008EC1DF001
:10249000030E01011D6FEA0E1C6F0BEC4AF044ECB9
:1024A00044F083D712AC13AE13D014A208D0149208
:1024B0000301E46B1BA60CD01B96158809D0030101
:1024C000E4A306D0E46B1BB603D01B8615860D80F3
:1024D00012BC04D0000115B056ECF1F012AC1CBCDB
:1024E00000D119AAFED0199A19A618AE78D013BA3D
:1024F00076D0000114A808D02DEC4EF0DBEC33F0C0
:102500001782010E0101E36F310EADEC13F0E26FA3
:10251000E251DDEC1AF00DE2000119B223D019826C
:102520001980500E0101266FD00E256FA3EC40F0EC
:1025300019D00001049042EC4EF009D0000104A033
:1025400006D019A20CD0199219840E9E08D01FEC47
:102550004EF0410E01012F5D9C0E3059EFE300015A
:1025600004A0DAD7300EADEC13F0E26FE46BE25169
:10257000DDEC1AF00EE2010E0101E46F18BA21D071
:10258000188A1888500E266FCE0E256FA3EC40F0E7
:1025900018D00001049042EC4EF009D0000104A0D4
:1025A00006D018AA0CD0189A188C0E9E08D01FECD2
:1025B0004EF0410E01012F5D9C0E3059EFE304A057
:1025C000DAD70101E45103E0AEECCAF002D01AEC14
:1025D00039F00101E35101E184D01C8282D019B6A7
:1025E00013B87FD0000114A808D02DEC4EF0DBEC1E
:1025F00033F01782010E0101E36F300EADEC13F0E2
:10260000E26FE46BE251DDEC1AF00EE2010E010123
:10261000E46F18BA28D0188A1888500E266FCE0E8C
:10262000256FA3EC40F01FD00001049042EC4EF067
:1026300009D0000104A006D018AA0CD0189A188C52
:102640000E9E08D01FEC4EF0410E01012F5D9C0E36
:102650003059EFE304B007D0010E0101E46F18BA5E
:1026600002D0188A18880101E45137E0310EADEC30
:1026700013F0E26FE46BE251DDEC1AF00EE2010EB2
:102680000101E46F19B221D019821980500E266F12
:10269000D00E256FA3EC40F018D00001049042EC5E
:1026A0004EF009D0000104A006D019A20CD0199256
:1026B00019840E9E08D01FEC4EF0410E01012F5DD3
:1026C0009C0E3059EFE304A0DAD70101E45103E096
:1026D000AEECCAF002D01AEC39F00101E35101E08E
:1026E0007CD712AC1BACCED11B9CF10E01011D6F2F
:1026F000440E1C6F010E13EC3CF0130E0101306F01
:10270000880E2F6F77EC40F00101E36B19A602D021
:10271000010EE36F0101E35117EC0FF0020A07E12C
:102720000301E22BE251020A04E1FF0002D003019F
:10273000E26BFA0E01011D6F3E0E1C6F010E13ECD1
:102740003CF0880E01012F6F130E306F000E316BBD
:10275000326B336B7CECA0F00101E26FF80E1D6F61
:10276000F50E1C6F010E13EC3CF0880E01012F6F6B
:10277000130E306F000E316B326B336B7CECA0F0BC
:102780000101E26F030EE36F0301C32B18D0FE0EAD
:102790001D6F530E1C6F010E13EC3CF0880E0101EF
:1027A0002F6F130E306F000E316B326B336B7CEC7E
:1027B000A0F00101E26FE251230A04E0E307010106
:1027C000E367E5D7E3512BE00301C36B0101E46B41
:1027D000750E0101E425D96EDA6A060EDA22960E2C
:1027E000E425E16EE26A070EE222DFCFE7FF750E15
:1027F000E425D96EDA6A060EDA22DF5004E0E42B13
:102800000F0EE465E5D7880E01012F6F130E306FB0
:10281000316B326B010E336F7CECA0F007D0020EEF
:102820000301C36503D0C36BAEECCAF0030E010114
:10283000E36F0301C02B69D0FC0E1D6FBB0E1C6F34
:10284000010E13EC3CF0880E01012F6F130E306F58
:10285000000E316B326B336B7CECA0F00101E26F48
:10286000BA6BE46B750E0101E425D96EDA6A060EC7
:10287000DA22B40EE425E16EE26A090EE222DFCF2D
:10288000E7FFBA51030A0BE1750EE425D96EDA6A47
:10289000060EDA22370EDF6202D08C8A0ED00101DA
:1028A000BA51030A0AE1750EE425D96EDA6A060EFA
:1028B000DA22300EDF6201D08C9A750E0101E42518
:1028C000D96EDA6A060EDA222C0EDF6201D0BA2B3C
:1028D000750E0101E425D96EDA6A060EDA22DF50A0
:1028E00004E0E42B1F0EE465BDD7880E01012F6FB5
:1028F000130E306F316B326B010E336F7CECA0F036
:102900000101E251130A04E0E3070101E36794D7F0
:10291000E35103E00301C06B07D0020E0301C06561
:1029200003D0C06BAEECCAF03CEC17F017E2500ECF
:102930000101266FDA0E256FA3EC40F0AEECCAF071
:1029400018BA13AA01D00E8E19B213A801D00E8E98
:1029500018BA19A201D00E8E17B01C82030E010105
:10296000E36F0301BC2B4FD0FB0E1D6F790E1C6F64
:10297000010E13EC3CF0880E01012F6F130E306F27
:10298000000E316B326B336B7CECA0F00101E26F17
:10299000E46B750E0101E425D96EDA6A060EDA22BF
:1029A000860EE425E16EE26A070EE222DFCFE7FF42
:1029B000750EE425D96EDA6A060EDA22DF5004E0DD
:1029C000E42B0F0EE465E5D7880E01012F6F130E7F
:1029D000306F316B326B010E336F7CECA0F0010174
:1029E000E2511C0A13E0E2511D0A10E0E2511E0AF6
:1029F0000DE0E2511F0A0AE0E251200A07E0E2512D
:102A0000210A04E0E3070101E367AED7E3510CE0DC
:102A1000E251200A09E0E2511E0A06E0E2511F0AD3
:102A200003E00301BC6B0ED0040E0301BC650AD0A9
:102A3000BC6B500E0101266FDC0E256FA3EC40F03D
:102A4000AEECCAF09B0E0701E66F070EE76FE6C714
:102A500021F1E7C722F1C8EC20F02151E26FE251E9
:102A6000630A03E10301CC6B0DD00B0EE26102D0CF
:102A7000010E06D0100EE26102D0020E01D0030E4C
:102A80000301CC6F12BCA1D21BB215AC01D01682CF
:102A900015BC1BA216921BB007AC01D0088A07BC5C
:102AA0001BA0089A14B807A609D0050E0101596F9A
:102AB000310E586F000E5A6BBFECA6F013A005D074
:102AC0000401F951F811D8B4FF0013A204D0000199
:102AD0001392AEECCAF014B803AE1DD0039EF80EEC
:102AE00001011D6FC60E1C6F010E13EC3CF02DECA6
:102AF0004EF017820AB208D0500E0101266FC20EA6
:102B0000256FA3EC40F007D0500E0101266FC60ED2
:102B1000256FA3EC40F01CA00ED01C9014A80BD085
:102B200000010AA208D02DEC4EF0DBEC33F0069841
:102B30000A921C820C841CA2F3D014A817A0EBD01C
:102B400004B008BAE8D016B2E6D017B28AD006B8F8
:102B500043D00101E36BC50E0101E325D96EDA6AAA
:102B6000060EDA22CD0EE3251E6F1F6B000E1F230B
:102B7000F6EC37F0DF6EC50E0101E325D96EDA6A97
:102B8000060EDA22DF5004E0E32B0F0EE365E3D7F5
:102B90000101E36BF70E0101E325D96EDA6A050E38
:102BA000DA22C80EE3251E6F1F6B000E1F23F6EC02
:102BB00037F0DF6EF70E0101E325D96EDA6A050EF4
:102BC000DA22DF5004E0E32B040EE365E3D710B410
:102BD000068800010A9247D0000110A444D00101E8
:102BE000E36BC50E0101E325D96EDA6A060EDA221F
:102BF0008A0EE3251E6F1F6B010E1F23F6EC37F0C4
:102C0000DF6EC50E0101E325D96EDA6A060EDA22FF
:102C1000DF5004E0E32B0F0EE365E3D70101E36B24
:102C2000F70E0101E325D96EDA6A050EDA22850E68
:102C3000E3251E6F1F6B010E1F23F6EC37F0DF6ECE
:102C4000F70E0101E325D96EDA6A050EDA22DF50AC
:102C500004E0E32B040EE365E3D7069800010A8243
:102C600002D0000117923CEC17F016AE0AD0020E0B
:102C700002019E6F000E8BEC39F00101E36F169E8E
:102C800008D0010E02019E6F000E8BEC39F001019D
:102C9000E36F0101E30506E0E351020A03E0E351BB
:102CA000040A20E10AB208D0500E0101266FCA0EB4
:102CB000256FA3EC40F007D0500E0101266FCC0E1B
:102CC000256FA3EC40F010A40BD00AB203D003018F
:102CD000CF8102D00301CF83CF51030A19E1CF6B1B
:102CE0000E8616D0E36714D00301CF6B0E960AB29E
:102CF00008D0500E0101266FC40E256FA3EC40F0E2
:102D000007D0500E0101266FC80E256FA3EC40F0CE
:102D10000301D06B1C900CA402D00C9401D01C9227
:102D200014B816A654D00001169627EC4BF00101FA
:102D3000E36F0301E65104E0E66BE651FFECCCF0F3
:102D40000101E36701D0178203AE17D00AB208D0A1
:102D5000500E0101266FC20E256FA3EC40F007D084
:102D6000500E0101266FC60E256FA3EC40F0000146
:102D7000039E2DEC4EF017822AD00101E35103E0AF
:102D8000E351050A16E10AB208D0500E0101266F80
:102D9000C20E256FA3EC40F007D0500E0101266F44
:102DA000C60E256FA3EC40F02DEC4EF0DBEC33F0BB
:102DB0000ED0E351030A04E1010EFFECCCF007D082
:102DC000E351040A04E1010EFFECCCF016860FA6D5
:102DD0000BD014980F960F9817900301C16B000148
:102DE0001B9CDBEC33F0F1D00FA8EFD00F9814B898
:102DF000ECD017800101E36BC50E0101E325D96E0C
:102E0000DA6A060EDA22CD0EE3251E6F1F6B000E66
:102E10001F23F6EC37F0DF6EC50E0101E325D96EF6
:102E2000DA6A060EDA22DF5004E0E32B0F0EE365C8
:102E3000E3D70101E36BF70E0101E325D96EDA6AEE
:102E4000050EDA22C80EE3251E6F1F6B000E1F232E
:102E5000F6EC37F0DF6EF70E0101E325D96EDA6A82
:102E6000050EDA22DF5004E0E32B040EE365E3D71E
:102E70000A920698000110A402D0000106883CECDA
:102E800017F0CBC39EF2000E8BEC39F00101E36F1B
:102E9000169EE30505E119B602D00E8401D00D8E11
:102EA0000101E351020A03E0E351040A55E10F8CEA
:102EB00010A452D00101E36BC50E0101E325D96EC8
:102EC000DA6A060EDA228A0EE3251E6F1F6B010EE8
:102ED0001F23F6EC37F0DF6EC50E0101E325D96E36
:102EE000DA6A060EDA22DF5004E0E32B0F0EE36508
:102EF000E3D70101E36BF70E0101E325D96EDA6A2E
:102F0000050EDA22850EE3251E6F1F6B010E1F23AF
:102F1000F6EC37F0DF6EF70E0101E325D96EDA6AC1
:102F2000050EDA22DF5004E0E32B040EE365E3D75D
:102F30000A82000106983CEC17F0CBC39EF2000E0B
:102F40008BEC39F00101E36F169EE351020A03E0B6
:102F5000E351040A01E10F8A0101E351050A01E18D
:102F6000088C0101E30506E0E351020A03E0E351A6
:102F7000040A13E10AB208D0500E0101266FCA0EEE
:102F8000256FA3EC40F007D0500E0101266FCC0E48
:102F9000256FA3EC40F00E8614D0E36712D00E9696
:102FA0000AB208D0500E0101266FC40E256FA3ECA3
:102FB00040F007D0500E0101266FC80E256FA3EC1C
:102FC00040F01C920301D06B1C9012BC23D010A0C7
:102FD00002D010901C8E40840101D6511AE045ECBD
:102FE00016F00101E36B11D0E351020D000EF32442
:102FF000D96EDA6A060EDA220101DECF54F1DDCF96
:1030000055F18AEC05F004E3E32BD651E35DECE3E4
:10301000D66B409412BCF7D004A0F4D00401EF5159
:10302000EE1101E0EFD0010E26EC41F01BC1D9FFFB
:103030001CC1DAFFDF50E26F020E26EC41F01BC12B
:10304000D9FF1CC1DAFFDF50E22700011ABC09D00A
:10305000030E26EC41F01BC1D9FF1CC1DAFFDF5083
:10306000E227040E26EC41F01BC1D9FF1CC1DAFF98
:10307000DF50E227050E26EC41F01BC1D9FF1CC131
:10308000DAFFDF50E227E26711D00301E96B0FA4FA
:1030900005D000010F94DBEC33F0FF0000011CAE03
:1030A000B1D0010E82EC45F01C9EACD00301E92B9F
:1030B000050EE96502D0010EE96FE95126EC41F0F9
:1030C0001BC1D9FF1CC1DAFFDF50E26FE26701D0FC
:1030D00099D0E9C31EF1000E21EC4AF01EC1CBF1DC
:1030E0001FC1CCF1E9C3E7F3CBC1E6F7CCC1E7F7E9
:1030F0000D0E0701E86FD890E733E633E82FFBD7D2
:10310000E651030B0301B46FE7050DE1000114A8BC
:103110000AD0000E0101CB11656F800ECC11666FD5
:1031200000EC80F006D0CBC165F1CCC166F100ECBB
:1031300080F0E36F030E0401EF6FE80EEE6F010104
:10314000E36706D0E7C31EF1000E7DEC30F05AD0E5
:1031500014A804D0010E0301E76506D00301E7516E
:10316000030AD8A43CEC17F014A804D0010E030104
:10317000E76536D00301CE6745D000010C8C65ECC5
:10318000D3F019E2500E0101266FE20E256FA3EC79
:1031900040F00301E751030A0AE11FAA08D0C82B37
:1031A000038CC851050A03E11A8CC86B049E030105
:1031B000E729C76F13D00301BD6BBE6BE7C31EF1D8
:1031C000000E7DEC30F00301E751030A04E11FAA71
:1031D00002D0C86B048E060E0301CE6F0C9C12D079
:1031E00000010C8C89EC19F005E2020E0301C76F97
:1031F000C92BF4D70301C96BE7C31EF1000E7DECA8
:1032000030F0ECD700F012BC28EF90F0000103A0E2
:1032100003D0000E6DEC1AF0000103A228EF90F02D
:10322000010E6DEC1AF028EF90F0E8CF64F16DC656
:103230001BF1010164516BEC49F002E2D8901200DD
:1032400005013451740A03E03451540A4FE13551F9
:10325000720A03E03551520A16E1E551050AEEE122
:103260000101676BC20E67251D6F1E6B500E1E237A
:10327000000E1F6BE2EC3DF00101672B250E676528
:10328000F1D714EFA0F0050EE56101D0D7D725EEF8
:10329000E5F0070EDF6401D0D1D7310EE525D96EF8
:1032A000DA6A050EDA22DF6A350E0101626F050E59
:1032B000636F62C121F163C122F1C8EC20F021C12A
:1032C00065F122C166F1000E655D010E6659B6E238
:1032D00066516511B3E065C1F2F21E6B550E1D6FAC
:1032E000F2C21FF1E2EC3DF014EFA0F034516E0A8F
:1032F00003E034514E0A31E1050EE56101D09ED75D
:1033000025EEE5F0060EDF6401D098D7310EE525F5
:10331000D96EDA6A050EDA22DF6A350E0101626FB4
:10332000050E636F62C121F163C122F1C8EC20F088
:1033300021C165F122C166F1110E655D000E66596D
:1033400001E37CD765C1D8F11E6B760E1D6FD8C125
:103350001FF1E2EC3DF014EFA0F03451690A04E0F3
:103360003451490A01E0AED03551690A03E03551C4
:10337000490A5CE10C0EE56101D060D725EEE5F06D
:10338000140EDF6401D05AD7050E0101676F21D0FA
:10339000310E01016725D96EDA6A050EDA22C00EF8
:1033A0006725E16EE26A060EE222DFCFE7FF850EB7
:1033B00067251D6F1E6B010E1E23310E6725D96E0A
:1033C000DA6A050EDA22DF501F6FE2EC3DF00101F0
:1033D000672B0501E5510101675DDAE3C10E672541
:1033E000D96EDA6A060EDA22DF6A850E67251D6F4E
:1033F0001E6B010E1E23000E1F6BE2EC3DF01094BD
:103400000601C55157E0060E0101226FC50E216F5E
:10341000FC0E246FDB0E236F266B070E256FEBEC83
:103420002FF02251211146E0108444D00B0EE561AB
:1034300001D004D725EEE5F0130EDF6401D0FED6EF
:10344000040E0101676F21D0310E01016725D96E8D
:10345000DA6A050EDA22C10E6725E16EE26A060E0F
:10346000E222DFCFE7FFC90E67251D6F1E6B000E3E
:103470001E23310E6725D96EDA6A050EDA22DF5077
:103480001F6FE2EC3DF00101672B0501E5510101E1
:10349000675DDAE3C10E6725D96EDA6A060EDA22B5
:1034A000DF6AC90E67251D6F1E6B000E1E231F6B82
:1034B000E2EC3DF006980A92000114B8FCEC4CF0E6
:1034C00014EFA0F03451610A04E03451410A01E0E4
:1034D000BED03551610A03E03551410A4CE1060E78
:1034E000E56101D0ABD625EEE5F01F0EDF6401D01B
:1034F000A5D6050E0101676F24D019A60FD0310E95
:1035000001016725D96EDA6A050EDA22660E672593
:10351000E16EE26A070EE222DFCFE7FF1B0E010138
:1035200067251D6F1E6B030E1E23310E6725D96E96
:10353000DA6A050EDA22DF501F6FE2EC3DF001017E
:10354000672B0501E5510101675DD7E319A607D097
:10355000660E6725D96EDA6A070EDA22DF6A1B0E5D
:10356000010167251D6F1E6B030E1E23000E1F6BCE
:10357000E2EC3DF04AD0050EE56101D05FD625EEC4
:10358000E5F01E0EDF6401D059D6040E0101676F0D
:1035900024D019B60FD0310E01016725D96EDA6A31
:1035A000050EDA22670E6725E16EE26A070EE22257
:1035B000DFCFE7FF940E010167251D6F1E6B000E24
:1035C0001E23310E6725D96EDA6A050EDA22DF5026
:1035D0001F6FE2EC3DF00101672B0501E551010190
:1035E000675DD7E319B607D0670E6725D96EDA6A2B
:1035F000070EDA22DF6A940E010167251D6F1E6B2C
:10360000000E1E231F6BE2EC3DF014B855D7EF0EF1
:1036100001011D6FAF0E1C6F010E13EC3CF0070E85
:1036200001011D6F6B0E1C6F000E13EC3CF0220E9F
:1036300000EC4CF00D0E00EC4CF0130E0101306F5D
:10364000880E2F6F77EC40F049EC25F035D73451D8
:10365000700A03E03451500A7CE13551700A03E0EE
:103660003551500A31E1060EE56101D0E7D525EE6E
:10367000E5F0090EDF6401D0E1D5050E0101676FA9
:1036800013D0800E67251D6F1E6B010E1E23310E99
:1036900001016725D96EDA6A050EDA22DF501F6F45
:1036A000E2EC3DF00101672B0501E5510101675D89
:1036B000E8E3800E67251D6F1E6B010E1E23000EB2
:1036C0001F6BE2EC3DF0F6D6050EE56101D0B6D5F4
:1036D00025EEE5F0080EDF6401D0B0D5040E01013F
:1036E000676F21D0310E01016725D96EDA6A050EA8
:1036F000DA22F30E6725E16EE26A050EE222DFCFE1
:10370000E7FFC40E67251D6F1E6B000E1E23310ED2
:103710006725D96EDA6A050EDA22DF501F6FE2ECF8
:103720003DF00101672B0501E5510101675DDAE319
:10373000F30E6725D96EDA6A050EDA22DF6AC40E47
:1037400067251D6F1E6B000E1E231F6BE2EC3DF004
:10375000B1D63451640A03E03451440A57E135517B
:10376000690A03E03551490A51E125EEE5F0140EEE
:10377000DF6401D063D5E551050A0CE1010E0101BA
:103780001E6F750E1D6F000E1F6BE2EC3DF0070102
:10379000A66B92D6050E0101676F21D0310E010193
:1037A0006725D96EDA6A050EDA22A10E6725E16E69
:1037B000E26A070EE222DFCFE7FF700E67251D6F7A
:1037C0001E6B010E1E23310E6725D96EDA6A050EB7
:1037D000DA22DF501F6FE2EC3DF00101672B05019B
:1037E000E5510101675DDAE3A10E6725D96EDA6A5A
:1037F000070EDA22DF6A700E67251D6F1E6B010E41
:103800001E23000E1F6BE2EC3DF056D63451640AC5
:1038100003E03451440A4CE13551640A03E0355168
:10382000440A46E125EEE5F0250EDF6401D006D519
:10383000060EE56101D002D5050E0101676F21D0AA
:10384000310E01016725D96EDA6A050EDA22CD0E36
:103850006725E16EE26A080EE222DFCFE7FF500E35
:1038600067251D6F1E6B010E1E23310E6725D96E55
:10387000DA6A050EDA22DF501F6FE2EC3DF001013B
:10388000672B0501E5510101675DDAE3CD0E672580
:10389000D96EDA6A080EDA22DF6A500E67251D6FCC
:1038A0001E6B010E1E23000E1F6BE2EC3DF004D6D2
:1038B0003451770A03E03451570A69E125EEE5F007
:1038C000130EDF6401D0BAD4050EE56101D0B6D481
:1038D000040E0101676F1CD0310E01016725D96EFE
:1038E000DA6A0501050EDA22DF50800A500F01E284
:1038F000A5D4310E01016725D96EDA6A0501050EDE
:10390000DA22DF50800A460F01E398D40101672BC9
:103910000501E5510101675DDFE3040E676F21D00A
:10392000310E01016725D96EDA6A050EDA22B20E70
:103930006725E16EE26A070EE222DFCFE7FFAF0EF6
:1039400067251D6F1E6B000E1E23310E6725D96E75
:10395000DA6A050EDA22DF501F6FE2EC3DF001015A
:10396000672B0501E5510101675DDAE3B20E6725BA
:10397000D96EDA6A070EDA22DF6AAF0E67251D6F8D
:103980001E6B000E1E231F6BE2EC3DF095D53451EB
:10399000720A03E03451520A34E1050EE56101D0A8
:1039A0004DD425EEE5F0070EDF6401D047D4310E8B
:1039B000E525D96EDA6A050EDA22DF6A350E0101D5
:1039C000626F050E636F62C121F163C122F1C8EC21
:1039D00020F021C165F122C166F1000E655D010E86
:1039E000665901E32BD46651651101E127D465C105
:1039F000DEF21E6B730E1D6FDEC21FF1E2EC3DF0B6
:103A000013D334516F0A03E034514F0A36E1050EE7
:103A1000E56101D013D425EEE5F0070EDF6401D097
:103A20000DD4310EE525D96EDA6A050EDA22DF6A89
:103A3000350E0101626F050E636F62C121F163C132
:103A400022F1C8EC20F021C165F122C166F1000E1F
:103A5000655D010E665902E31EEF99F0665165112E
:103A600002E11EEF99F065C1E1F21E6B700E1D6F51
:103A7000E1C21FF1E2EC3DF0D7D234516D0A03E010
:103A800034514D0A38E1050EE56102D01EEF99F080
:103A900025EEE5F0070EDF6402D01EEF99F0310E3F
:103AA000E525D96EDA6A050EDA22DF6A350E0101E4
:103AB000626F050E636F62C121F163C122F1C8EC30
:103AC00020F021C165F122C166F1000E655D010E95
:103AD000665902E31EEF99F06651651102E11EEF8F
:103AE00099F065C1E2F21E6B720E1D6FE2C21FF10A
:103AF000E2EC3DF099D23451660A03E03451460AB3
:103B000039E1E551050A02E01EEF99F001011F6B52
:103B1000750E1E6FF6EC37F0676F05013551300AF0
:103B200006E11B901B92F90E010167171AD035515F
:103B3000310A06E11B801B9201016783679511D052
:103B40003551320A06E11B901B820101678567939C
:103B500008D03551330A05E11B801B82060E010196
:103B6000671301011E6B750E1D6F67C11FF1E2EC3B
:103B70003DF05AD23451650A03E03451450A25E13B
:103B8000E551050A02E01EEF99F001011F6B4F0E8F
:103B90001E6FF6EC37F0676F05013551300A04E10E
:103BA0001F9A0101679908D03551310A05E11F8A32
:103BB000010167895BECE6F001011E6B4F0E1D6F82
:103BC00067C11FF1E2EC3DF02FD23451730A03E0DC
:103BD0003451530A0FE1E551050A02E01EEF99F056
:103BE0003551300A01E120D23551310A01E11CD2B0
:103BF0001EEF99F03451630A04E03451430A01E0A6
:103C0000D3D0E551050A20E13551310A03E1000125
:103C10000A8E0AD23551320A03E100010B8004D228
:103C20003551330A03E100010A8AFED13551340AC5
:103C300003E100010A88F8D13551360A02E01EEF8F
:103C400099F000010B82F0D1E5510A0A44E1EF0E30
:103C500001011D6FD20E1C6F010E13EC3CF005012B
:103C6000355100EC4CF00501365100EC4CF03A0EA9
:103C700000EC4CF00501375100EC4CF005013851D7
:103C800000EC4CF03A0E00EC4CF00501395100EC20
:103C90004CF005013A5100EC4CF0FE0E01011D6F95
:103CA000590E1C6F000E13EC3CF0130E0101306F27
:103CB000880E2F6F77EC40F002E30001188442EC8D
:103CC0004EF01FEC4EF0E90E01012F5D030E30594E
:103CD00001E3AAD1F6D7E551100A01E0A5D1FC0E07
:103CE00001011D6FD30E1C6F010E13EC3CF005019A
:103CF000395100EC4CF005013A5100EC4CF02F0E1C
:103D000000EC4CF00501375100EC4CF00501385146
:103D100000EC4CF02F0E00EC4CF00501355100EC9E
:103D20004CF00501365100EC4CF02C0E00EC4CF040
:103D300005013B5100EC4CF005013C5100EC4CF00E
:103D40003A0E00EC4CF005013D5100EC4CF0050141
:103D50003E5100EC4CF03A0E00EC4CF005013F51A6
:103D600000EC4CF00501405100EC4CF0FE0E01015E
:103D70001D6F590E1C6F000E13EC3CF0130E010169
:103D8000306F880E2F6F77EC40F002E3000118844B
:103D900042EC4EF01FEC4EF0E90E01012F5D030ED8
:103DA000305901E341D1F6D73451790A05E0345155
:103DB000590A02E01EEF99F03551790A04E03551B5
:103DC000590A01E098D0060EE56102D01EEF99F085
:103DD00025EEE5F00E0EDF6402D01EEF99F03651AD
:103DE000310A42E1060E0101676F24D019A60FD0F7
:103DF000310E01016725D96EDA6A050EDA22D90E75
:103E00006725E16EE26A060EE222DFCFE7FF350E9C
:103E1000010167251D6F1E6B030E1E23310E6725E2
:103E2000D96EDA6A050EDA22DF501F6FE2EC3DF040
:103E30000101672B0501E5510101675DD7E319A673
:103E400007D0D90E6725D96EDA6A060EDA22DF6A44
:103E5000350E010167251D6F1E6B030E1E23000E1C
:103E60001F6BE2EC3DF0DCD03651320A02E01EEF6F
:103E700099F0060E0101676F24D019A60FD0310EFC
:103E800001016725D96EDA6A050EDA22E20E67258E
:103E9000E16EE26A060EE222DFCFE7FF3E0E01018D
:103EA00067251D6F1E6B030E1E23310E6725D96E0D
:103EB000DA6A050EDA22DF501F6FE2EC3DF00101F5
:103EC000672B0501E5510101675DD7E319A607D00E
:103ED000E20E6725D96EDA6A060EDA22DF6A3E0E36
:103EE000010167251D6F1E6B030E1E23000E1F6B45
:103EF000E2EC3DF095D0050EE56102D01EEF99F0A1
:103F000025EEE5F00D0EDF6402D01EEF99F035517D
:103F1000310A41E1050E0101676F24D019B60FD0B7
:103F2000310E01016725D96EDA6A050EDA22DA0E42
:103F30006725E16EE26A060EE222DFCFE7FFE80EB8
:103F4000010167251D6F1E6B000E1E23310E6725B4
:103F5000D96EDA6A050EDA22DF501F6FE2EC3DF00F
:103F60000101672B0501E5510101675DD7E319B632
:103F700007D0DA0E6725D96EDA6A060EDA22DF6A12
:103F8000E80E010167251D6F1E6B000E1E231F6BBF
:103F9000E2EC3DF045D03551320A02E01EEF99F0D7
:103FA000050E0101676F24D019B60FD0310E010143
:103FB0006725D96EDA6A050EDA22E30E6725E16E0F
:103FC000E26A060EE222DFCFE7FFF10E010167256C
:103FD0001D6F1E6B000E1E23310E6725D96EDA6A27
:103FE000050EDA22DF501F6FE2EC3DF00101672B76
:103FF0000501E5510101675DD7E319B607D0E30E6E
:104000006725D96EDA6A060EDA22DF6AF10E01013F
:1040100067251D6F1E6B000E1E231F6BE2EC3DF02B
:10402000000114A849EC25F045EC16F001016439B3
:10403000F00B676F0AAE07D00A9E8A0E466F675173
:1040400010EC07F038D00BA008D00B908B0E0101BC
:10405000466F675110EC07F02ED00AAA08D00A9AD2
:104060008C0E0101466F675110EC07F024D00AA8AE
:1040700008D00A988D0E0101466F675110EC07F0C9
:104080001AD00AAC08D00A9C8E0E0101466F675107
:1040900010EC07F010D00BA208D00B928F0E01018C
:1040A000466F675110EC07F006D0830E0101466F92
:1040B000675110EC07F046C165F147C166F11AA4DB
:1040C00004D000011A94D880120006016D51B6EC9C
:1040D0004DF0F9E3645185EC46F00101676F65C16D
:1040E0003FF166C140F164C141F167C142F1030E85
:1040F000436F16EC3DF0E7D733671BD005010A6B21
:104100000B6B0C6B0D6B0294029604D056ECF1F025
:1041100002B40FD005010D51800A800F08E1000E96
:104120000C5D05E1EA0E0B5D02E1610E0A5DEEE356
:104130000C0C05010A6B0B6B0C6B0D6B02A6029449
:1041400008D056ECF1F002A404D002940201CF672B
:1041500017D001013251800A346F05010A51010163
:104160002F5D05010B510101305905010C51010171
:10417000315905010D51800A01013459D9E3E1D7C4
:1041800002960101356BA00E01013525D96EDA6A60
:10419000080EDA22750E3525E16EE26A060EE2227D
:1041A000DFCFE7FF750E3525D96EDA6A060EDA2203
:1041B000DF5004E0352B310E3565E5D7060E0101E1
:1041C000226F750E216FF90E246F790E236F266B07
:1041D0000A0E256FEBEC2FF02251211106E10001B0
:1041E00002A4020C00010286020C060E0101226FDD
:1041F000750E216FF40E246F7E0E236F266B0C0E4E
:10420000256FEBEC2FF02251211106E1000102A4F1
:104210002F0C000102862F0C060E0101226F750E75
:10422000216FFD0E246F130E236F266B070E256F73
:10423000EBEC2FF022512111D2E0060E0101226F8A
:10424000750E216FEF0E246FE30E236F266B100E99
:10425000256FEBEC2FF02251211106E1000102A4A1
:10426000060C00010286060C060E0101226F750E77
:10427000216FFB0E246FB80E236F266B080E256F7F
:10428000EBEC2FF02251211106E1000102A4240CD5
:1042900000010286240C060E0101226F750E216FAB
:1042A000FD0E246F700E236F266B020E256FEBEC54
:1042B0002FF02251211106E1000102A4080C000197
:1042C0000286080C060E0101296F750E286F070E75
:1042D0002B6FD60E2A6F57EC2FF02951281106E0CC
:1042E000000102A4030C00010286030C060E01016A
:1042F000226F750E216FF90E246F2A0E236F266B25
:10430000010E256FEBEC2FF02251211106E1000187
:1043100002A40D0C000102860D0C060E0101226F95
:10432000750E216FFB0E246FAD0E236F266B010EF1
:10433000256FEBEC2FF02251211106E1000102A4C0
:10434000100C00010286100C060E0101226F750E82
:10435000216FF60E246F300E236F266B010E256F32
:10436000EBEC2FF02251211106E1000102A4110C07
:1043700000010286110C060E0101226F750E216FDD
:10438000EF0E246FF20E236F266B010E256FEBEC00
:104390002FF02251211106E1000102A40F0C0001AF
:1043A00002860F0C060E0101226F750E216FFE0EA4
:1043B000246F8F0E236F266B050E256FEBEC2FF00D
:1043C0002251211106E1000102A43A0C00010286EB
:1043D0003A0C060E0101226F750E216FFF0E246F3D
:1043E0002F0E236F266B040E256FEBEC2FF022515E
:1043F000211106E1000102A43B0C000102863B0CE6
:10440000060E0101226F750E216FF60E246F0E0E3F
:10441000236F266B0B0E256FEBEC2FF02251211131
:1044200001E1DDD6060E0101226F750E216FF60E39
:10443000246F320E236F266B0B0E256FEBEC2FF0E3
:104440002251211101E1E2D6060E0101226F750E03
:10445000216FF60E246F1A0E236F266B0B0E256F3D
:10446000EBEC2FF02251211106E1000102A4430CD4
:1044700000010286430C060E0101226F750E216FAA
:10448000F00E246F590E236F266B0F0E256FEBEC89
:104490002FF02251211106E1000102A4440C000179
:1044A0000286440C060E0101226F750E216FEF0E7D
:1044B000246F0D0E236F266B110E256FEBEC2FF082
:1044C0002251211106E1000102A4450C00010286DF
:1044D000450C060E0101226F750E216FF00E246F40
:1044E000490E236F266B0F0E256FEBEC2FF0225138
:1044F000211106E1000102A4390C00010286390CE9
:10450000060E0101226F750E216FFA0E246FA20EA6
:10451000236F266B090E256FEBEC2FF02251211132
:1045200006E1000102A43E0C000102863E0C060ECC
:104530000101226F750E216FF30E246FE80E236FB9
:10454000266B0D0E256FEBEC2FF02251211106E1A9
:10455000000102A4400C00010286400C060E01017D
:10456000226F750E216FF90E246F210E236F266BBB
:104570000A0E256FEBEC2FF02251211106E100010C
:1045800002A4420C00010286420C060E0101226FB9
:10459000750E216FF90E246F2C0E236F266B0A0EF9
:1045A000256FEBEC2FF02251211106E1000102A44E
:1045B0003F0C000102863F0C060E0101226F750EB2
:1045C000216FF40E246F640E236F266B0C0E256F83
:1045D000EBEC2FF02251211106E1000102A4410C65
:1045E00000010286410C060E0101226F750E216F3B
:1045F000F10E246F190E236F266B0E0E256FEBEC58
:104600002FF02251211106E1000102A4090C000142
:104610000286090C060E0101226F750E216FF40E41
:10462000246F040E236F266B0D0E256FEBEC2FF01D
:104630002251211106E1000102A42C0C0001028686
:104640002C0C060E0101226F750E216FFA0E246FDD
:10465000AC0E236F266B090E256FEBEC2FF0225169
:104660002111D2E0060E0101226F750E216FFA0EA4
:10467000246FB00E236F266B050E256FEBEC2FF029
:1046800022512111C1E0060E0101226F750E216F2A
:10469000FA0E246FB60E236F266B090E256FEBEC16
:1046A0002FF02251211106E1000102A4320C000179
:1046B0000286320C060E0101226F750E216FF90E73
:1046C000246F370E236F266B0A0E256FEBEC2FF04D
:1046D0002251211106E1000102A41C0C00010286F6
:1046E0001C0C060E0101226F750E216FF90E246F4E
:1046F000420E236F266B0A0E256FEBEC2FF0225132
:10470000211106E1000102A41D0C000102861D0C0E
:10471000060E0101226F750E216FF90E246F4D0EEA
:10472000236F266B0A0E256FEBEC2FF0225121111F
:1047300006E1000102A41E0C000102861E0C060EFA
:104740000101226F750E216FF90E246F580E236F31
:10475000266B0A0E256FEBEC2FF02251211106E19A
:10476000000102A41F0C000102861F0C060E0101AD
:10477000226F750E216FF90E246F630E236F266B67
:104780000A0E256FEBEC2FF02251211106E10001FA
:1047900002A4200C00010286200C060E0101226FEB
:1047A000750E216FF90E246F6E0E236F266B0A0EA5
:1047B000256FEBEC2FF02251211106E1000102A43C
:1047C000210C00010286210C060E0101226F750EDC
:1047D000216FFF0E246FFD0E236F266B010E256FD8
:1047E000EBEC2FF02251211106E1000102A4250C6F
:1047F00000010286250C060E0101226F750E216F45
:10480000FD0E246F6B0E236F266B070E256FEBECEE
:104810002FF02251211106E1000102A4260C000113
:104820000286260C060E0101226F750E216FFE0E08
:10483000246F890E236F266B050E256FEBEC2FF08E
:104840002251211106E1000102A42B0C0001028675
:104850002B0C060E0101226F750E216FFB0E246FCB
:10486000A60E236F266B080E256FEBEC2FF022515E
:10487000211106E1000102A4040C00010286040CCF
:10488000060E0101226F750E216FFB0E246F9D0E27
:10489000236F266B080E256FEBEC2FF022512111B0
:1048A00006E1000102A40B0C000102860B0C060EAF
:1048B0000101226F750E216FFB0E246FAF0E236F67
:1048C000266B080E256FEBEC2FF02251211106E12B
:1048D000000102A40A0C000102860A0C060E010166
:1048E000226F750E216FFD0E246FB90E236F266B9C
:1048F000060E256FEBEC2FF02251211106E100018D
:1049000002A4150C00010286150C060E0101226F8F
:10491000750E216FFE0E246F7D0E236F266B050E24
:10492000256FEBEC2FF02251211106E1000102A4CA
:10493000230C00010286230C060E0101226F750E66
:10494000216FFD0E246FC00E236F266B060E256FA0
:10495000EBEC2FF02251211106E1000102A4130C0F
:1049600000010286130C060E0101226F750E216FE5
:10497000FD0E246F030E236F266B070E256FEBECE5
:104980002FF02251211106E1000102A4140C0001B4
:104990000286140C060E0101226F750E216FFD0EAA
:1049A000246FB90E236F266B060E256FEBEC2FF0EC
:1049B00022512111A4E0060E0101226F750E216F14
:1049C000FA0E246F660E236F266B090E256FEBEC33
:1049D0002FF02251211106E1000102A4180C000160
:1049E0000286180C060E0101226F750E216FFA0E59
:1049F000246F700E236F266B090E256FEBEC2FF0E2
:104A00002251211106E1000102A4160C00010286C8
:104A1000160C060E0101226F750E216FFA0E246F1F
:104A20007A0E236F266B090E256FEBEC2FF02251C7
:104A3000211106E1000102A4190C00010286190CE3
:104A4000060E0101226F750E216FFA0E246F840E7F
:104A5000236F266B090E256FEBEC2FF022512111ED
:104A600006E1000102A41A0C000102861A0C060ECF
:104A70000101226F750E216FFA0E246F8E0E236FC7
:104A8000266B090E256FEBEC2FF02251211106E168
:104A9000000102A41B0C000102861B0C060E010182
:104AA000226F750E216FFA0E246F980E236F266BFE
:104AB000090E256FEBEC2FF02251211106E10001C8
:104AC00002A4170C00010286170C060E0101226FCA
:104AD000750E216FFE0E246F830E236F266B050E5D
:104AE000256FEBEC2FF02251211106E1000102A409
:104AF000270C00010286270C060E0101226F750E9D
:104B0000216FF60E246F4A0E236F266B0B0E256F56
:104B1000EBEC2FF02251211106E1000102A4280C38
:104B200000010286280C060E0101226F750E216F0E
:104B3000F00E246F790E236F266B0F0E256FEBECB2
:104B40002FF02251211106E1000102A4350C0001D1
:104B50000286350C060E0101226F750E216FF40ED0
:104B6000246F120E236F266B0D0E256FEBEC2FF0CA
:104B70002251211106E1000102A4290C0001028644
:104B8000290C060E0101226F750E216FF00E246FA5
:104B9000690E236F266B0F0E256FEBEC2FF0225161
:104BA000211106E1000102A4360C00010286360C38
:104BB000060E0101226F750E216FF60E246F3E0E58
:104BC000236F266B0B0E256FEBEC2FF0225121117A
:104BD00006E1000102A42D0C000102862D0C060E38
:104BE0000101226F750E216FF60E246F260E236FC2
:104BF000266B0B0E256FEBEC2FF02251211106E1F5
:104C0000000102A42E0C000102862E0C060E0101EA
:104C1000226F750E216FF40E246F570E236F266BD3
:104C20000C0E256FEBEC2FF02251211106E1000153
:104C300002A4300C00010286300C060E0101226F26
:104C4000750E216FF40E246F710E236F266B0C0E00
:104C5000256FEBEC2FF02251211106E1000102A497
:104C60003C0C000102863C0C060E0101226F750E01
:104C7000216FF30E246FF60E236F266B0D0E256F3A
:104C8000EBEC2FF02251211106E1000102A4310CBE
:104C900000010286310C060E0101226F750E216F94
:104CA000F90E246F160E236F266B0A0E256FEBECA0
:104CB0002FF02251211106E1000102A43D0C000158
:104CC00002863D0C060E0101226F750E216FFA0E51
:104CD000246F520E236F266B090E256FEBEC2FF01D
:104CE0002251211106E1000102A4330C00010286C9
:104CF000330C060E0101226F750E216FFA0E246F20
:104D00005C0E236F266B090E256FEBEC2FF0225102
:104D1000211106E1000102A4340C00010286340CCA
:104D2000060E0101226F750E216FFD0E246FB20E6B
:104D3000236F266B060E256FEBEC2FF0225121110D
:104D400006E1000102A4370C00010286370C060EB2
:104D50000101226F750E216FFD0E246F0B0E236F64
:104D6000266B070E256FEBEC2FF02251211106E187
:104D7000000102A4380C00010286380C000C0496D5
:104D800004980101D56B0201D56BF76B0101A26B91
:104D9000A36B5A0501E0B4D000010C869C9EA88448
:104DA0007C867D6A670EAB6E9C8E9C88A88AA49ACE
:104DB000A59AA38A8E9C8D9842EC4EF01FEC4EF083
:104DC000590E01012F5D020E3059F8E38D8842EC37
:104DD0004EF01FEC4EF0650E01012F5D000E3059B4
:104DE000F8E38E8C270E0201B36F100EB26FE46BE6
:104DF0000FD0B351B2110CE1EF0E01011C6F310E57
:104E00001B6F100E1D6FEEEC4CF08E9C8D981200F7
:104E1000E451030AEEE1030EB36FE80EB26FE46BE8
:104E2000FF0E01011D6FA10E1C6F010E13EC3CF073
:104E30000DD0B351B2110AE1EF0E01011C6F430E08
:104E40001B6F100E1D6FEEEC4CF0DFD70201E40576
:104E5000F0E1170EB36F700EB26FE46BFB0E010141
:104E60001D6FD30E1C6F010E13EC3CF00DD0B3512F
:104E7000B2110AE1EF0E01011C6F550E1B6F100EEF
:104E80001D6FEEEC4CF0C1D70201E405F0E1EE0E2F
:104E900001011D6F300E1C6F010E13EC3CF0010E72
:104EA0000101306FF40E2F6F77EC40F0170E020106
:104EB000B36F700EB26FE46BEC0E01011D6F630EE9
:104EC0001C6F010E13EC3CF00DD0B351B2110AE18E
:104ED000EF0E01011C6F670E1B6F100E1D6FEEECC5
:104EE0004CF093D70201E451020AEFE1EF0E010109
:104EF0001C6FF40E1B6F100E1D6FEEEC4CF09DD26C
:104F000007961A8EFA0E01011D6FDE0E1C6F010E40
:104F100013EC3CF04C0E0101306F080E2F6F77EC54
:104F200040F0ED0E01011D6F350E1C6F010E13ECEC
:104F30003CF0130E0101306F880E2F6F77EC40F0BC
:104F4000EB0E01011D6FF10E1C6F010E13EC3CF016
:104F5000130E0101306F880E2F6F77EC40F0EC0ECE
:104F600001011D6F420E1C6F010E13EC3CF0070E89
:104F70000101306FD00E2F6F77EC40F0880E0101E9
:104F80002F6F130E306F000E316B326B336B7CEC76
:104F9000A0F00101B06FB051400A19E0F60E1D6F8C
:104FA000620E1C6F010E13EC3CF0030E0101306F1A
:104FB000E80E2F6F77EC40F0EE0E0101326F980E85
:104FC000316F346B130E336F9EEC0CF0C2D0F00EC9
:104FD0001D6F160E1C6F010E13EC3CF0070E010145
:104FE000306FD00E2F6F77EC40F0880E01012F6FDD
:104FF000130E306F000E316B326B336B7CECA0F014
:105000000101B06FB051420A0DE075EC42F0EE0EB6
:105010000101326FE80E316F346B120E336F9EEC6C
:105020000CF097D0EE0E1D6F300E1C6F010E13ECBE
:105030003CF0010E0101306FF40E2F6F77EC40F061
:1050400012A833D00101AC6BAC5158255B6F000E38
:1050500059215C6F0E0E5B25D96E000E5C21DA6E55
:10506000D50E0101AC25E16EE26A060EE222DFCF29
:10507000E7FFAC2B060EAC65E7D7F90E1D6FC60E29
:105080001C6F010E13EC3CF0060E01011D6FD50ED6
:105090001C6F000E13EC3CF0EC0E01011D6FB80EFE
:1050A0001C6F000E13EC3CF042D1F10E01011D6F9C
:1050B000370E1C6F010E13EC3CF0E80E01012F6F50
:1050C000030E306F000E316B326B336B7CECA0F053
:1050D0000101B06FB051020A0DE075EC42F0ED0E27
:1050E0000101326F950E316F346B130E336F9EECEE
:1050F0000CF02FD00D8A0201DD6B130E0101306F11
:10510000880E2F6F77EC40F0600E0201DD25D96E1E
:10511000DA6A080EDA22DF6A0D9AE80E01012F6FB3
:10512000030E306F000E316B326B336B7CECA0F0F2
:105130000101B06FB0513E0A0EE075EC42F0ED0E89
:105140000101326F950E316F346B130E336F9EEC8D
:105150000CF01A9E5ED0AD6BAE6BAF6B37D0640EA9
:105160000101AD25D96EDA6A080EDA222E0EDF6251
:105170002BD0620E5B6F080E5C6FAD515B27000E8B
:105180005C235BC121F15CC122F1C8EC20F021C19C
:10519000A4F122C1A5F15F0E0101AD25D96EDA6A35
:1051A000080EDA22460EDF6205D00D84A4C19FF1FD
:1051B000A5C1A0F10101A451AE5DA551AF5904E212
:1051C000A4C1AEF1A5C1AFF10101AD2B640E010187
:1051D000AD25D96EDA6A080EDA22DF50C0E10DA4DF
:1051E00053D0060EAE5D000EAF5919E275EC42F0D9
:1051F0001A9EA80E0301AD6FC00EAC6FF00E010138
:10520000326F050E316F346B100E336F9EEC0CF065
:1052100057D000011AA21200000ED7EF3EF0080E80
:105220000101286F640E276FFF0E2A6F430E296F4E
:10523000AEC12BF1AFC12CF166ECD5F0AF51A01986
:1052400002E1AE519F1908E1F00E1D6F270E1C6F91
:10525000010E13EC3CF007D0F00E1D6F990E1C6F81
:10526000010E13EC3CF0080E01011D6F640E1C6F63
:10527000000E13EC3CF0EC0E01011D6FB80E1C6F1C
:10528000000E13EC3CF053D007B402D012A441D06E
:10529000060E0101AE5D000EAF5914E275EC42F04E
:1052A0001A9EA80E0301AD6FC00EAC6FF00E010187
:1052B000326F050E316F346B100E336F9EEC0CF0B5
:1052C0001294A7D7080E0101286F640E276FFF0EF6
:1052D0002A6F430E296FAEC12BF1AFC12CF166ECE2
:1052E000D5F0F00E1D6F990E1C6F010E13EC3CF003
:1052F000080E01011D6F640E1C6F000E13EC3CF0D4
:10530000EC0E01011D6FB80E1C6F000E13EC3CF08B
:105310000ED007B40CD0000112B409D075EC42F0E5
:105320001A9EA80E0301AD6FC00EAC6FC00C129494
:10533000030E0101306FE80E2F6F77EC40F0880EFE
:1053400001012F6F130E306F000E316B326B336B18
:105350007CECA0F00101B06FB0513F0A15E075EC94
:1053600042F0EE0E0101326F1B0E316F346B140EE2
:10537000336F9EEC0CF000011AA203D0000ED7ECA4
:105380003EF000011A9E120075EC42F0030E01017E
:10539000306FE80E2F6F77EC40F0500E01011E6F5A
:1053A000E70E1D6F460E1F6FE2EC3DF0500E01013F
:1053B0001E6FE80E1D6F4C0E1F6FE2EC3DF0500E9D
:1053C00001011E6FE90E1D6F530E1F6FE2EC3DF0E1
:1053D000500E01011E6FEA0E1D6F310E1F6FE2ECC1
:1053E0003DF0EC0E0101326F9D0E316F346B1A0EE1
:1053F000336F9EEC0CF0030E0101306FE80E2F6F3F
:1054000077EC40F0F80E01011D6FC60E1C6F010E07
:1054100013EC3CF0030E0101306FE80E2F6F77ECB8
:1054200040F01380070E0401F96FD00EF86F0001F1
:105430001AA2D00C010ED7EF3EF00E9810D0010149
:105440005A0506E1FA0E1C6FD40E1B6F090E0CD123
:10545000FA0E326FD40E316F346B090E0CD158C175
:1054600023F159C124F13C0E0101256F5AC126F1E7
:1054700007EC3FF00101B16FB1C1A9FFA8A2FED7AF
:105480001CBADDD70101B1513A0AE9E1A24BA32BC5
:1054900058C12DF159C12EF10A0E2F6F5AC130F1AA
:1054A000C3EC46F0B16F1CBACAD7B1C1A7F1A7C10E
:1054B000D0F258C12DF159C12EF10A0E01012F6F02
:1054C0005AC130F1C3EC46F0B16F1CBAB8D7010134
:1054D000B1515C6F5B6B5D6B5C515E6F5DC1A8F140
:1054E0005EC1A9F1AA6BAB6B58C12DF159C12EF168
:1054F0000A0E2F6F5AC130F1C3EC46F0B16F1CBADF
:105500009ED70101B151A81358C12DF159C12EF1F7
:105510000A0E2F6F5AC130F1C3EC46F0A16F1CBACE
:105520008ED704A892D10101D890AA2B000EAB23EC
:105530008CD158C12DF159C12EF10A0E2F6F5AC1CD
:1055400030F1C3EC46F0A66F1CBA79D70101AB511C
:10555000A811A911AA1117E10B0E58255B6F000EB7
:1055600059215C6F5BC121F15CC122F1FB0E246FFC
:10557000E50E236F266B080E256FEBEC2FF0225102
:10558000211101E00D8C0101A951040A600ED8B46B
:10559000A819AA11AB1117E1090E58255B6F000E6F
:1055A00059215C6F5BC121F15CC122F1FF0E246FB8
:1055B000340E236F266B040E256FEBEC2FF0225177
:1055C000211101E007820101AB51800A800F08E13F
:1055D000010EAA5D05E1EC0EA95D02E1010EA85DD8
:1055E00001E3198C0101A82B000EA923AA23AB23E8
:1055F000A7070101A7299DE158C133F159C134F131
:105600000A0E356F5AC136F1A6EC3EF001E304866E
:105610001CBA15D724D758C133F159C134F10A0E39
:10562000356F5AC136F1A6EC3EF001E304861CBA90
:1056300006D704A610D001015A0506E1FB0E1C6F27
:10564000CA0E1B6F080E10D0FB0E326FCA0E316FE0
:10565000346B080E10D00DAC11D001015A0507E1D2
:10566000F90E1C6F840E12D01D6FEEEF4CF0F90E88
:10567000326F840E11D0336F9EEF0CF007A210D062
:1056800001015A0506E1F90E1C6F8F0E1B6F0A0E01
:10569000EBD7F90E326F8F0E316F346B0A0EEBD7EA
:1056A00019AC10D001015A0506E1F10E1C6F280E4D
:1056B0001B6F0E0ED9D7F10E326F280E316F346B7F
:1056C0000E0ED9D70101010E286F5F0E276FEC0E69
:1056D0002A6F200E296FA2C12BF1A3C12CF166EC19
:1056E000D5F02751B16F5A0515E1010E1C6F5F0E01
:1056F0001B6FB1C11DF1EEEC4CF0270E0101A36F41
:10570000100EA26FA207D8A0A3070101A351A211F6
:105710001CE0F8D7010E326F5F0E316FB1C133F16B
:10572000346B9EEC0CF0EC0E0101326F250E316FE4
:10573000346B1C0E336F9EEC0CF0F80E01011D6FE4
:10574000C60E1C6F010E13EC3CF00B0E0101306F06
:10575000B80E2F6F77EC40F0500E01011E6FE70E70
:105760001D6F460E1F6FE2EC3DF0500E01011E6FE3
:10577000E80E1D6F4C0E1F6FE2EC3DF0500E010164
:105780001E6FE90E1D6F530E1F6FE2EC3DF0500EC1
:1057900001011E6FEA0E1D6F300E1F6FE2EC3DF02F
:1057A000130E0101306F880E2F6F77EC40F0FF0071
:1057B0001200A66B0DD058C12DF159C12EF10A0E61
:1057C0002F6F5AC130F1C3EC46F0A6131CBA37D67E
:1057D0000101A707A729EFE1A651F00B100A02E18A
:1057E000048801D0049858C133F159C134F10A0E2C
:1057F0000101356F5AC136F1A6EC3EF007D758C10A
:105800002DF159C12EF10A0E2F6F5AC130F1C3ECA0
:1058100046F0A66F1CBA13D60101A707A729EFE12E
:10582000A6C15BF10F0E5B175B0502E1048801D096
:10583000049858C133F159C134F10A0E0101356F92
:105840005AC136F1A6EC3EF0E1D60101A15101E1C9
:10585000CFD6010A01E1DFD6030AABE0060ADCE09D
:10586000FED50201B551B41103E0B407D8A0B507C5
:105870000401EB51EA1103E0EA07D8A0EB07F95164
:10588000F81103E0F807D8A0F9070201B351B211EB
:1058900003E0B207D8A0B30704009E90D10ECF6EEC
:1058A000200ECE260401E24BE32BEC4BED2B050141
:1058B0000A2B000E0B230C230D230301AA4BAB2B49
:1058C00014A009D01490030E226EEA0E216EA8ECEB
:1058D0002CF08F8014860401F751F61108E0F607CA
:1058E000D8A0F707F751F61102E10201E86B0401B5
:1058F000EF51EE1103E0EE07D8A0EF070301A84B2C
:10590000A92BA951800A296EA651A85DA751800A2A
:10591000295801E31E8C0401D607D8A0D707D75118
:10592000D61102E111A6119A15A00AD00301D72BB6
:10593000040ED76505D0D76B00011582D6EC44F074
:105940000301C7670AD00CAC07BC07D016BA12BC5B
:1059500004D013B402D08D8A8D9C0301C75117E087
:10596000E35102E0E3073DD00CBA06D08D9A8D9C3E
:105970000301E3690C8A35D08D9A8D8C0301E369AC
:105980000C9AC707C7672DD08D8A8D9C2AD013A487
:1059900012D00201EE2B270EEE6523D0EE6B8D8C1C
:1059A0008D8A0301CA2BCA51050A1BE18D9C8D9A71
:1059B000CA6B139416D00CAC07D00201EE2B310E3B
:1059C000EE6502D0EE6B0CD007AC0BD005011C4B82
:1059D0001D2BE80E1C5D030E1D5903E31C6B1D6B94
:1059E0008D7A14A408D00301D22B310ED26503D0D6
:1059F000D26B14948F900CAE0FD00201E52B310EB8
:105A0000E5650AD0E56B8F700301DA2B3B0EDA6592
:105A100003D0DA6B0C9E8F9009AC07D00201E52B06
:105A2000C70EE56502D0E56B8F700DA010D00301A5
:105A3000DD2B310EDD650BD0DD6B8F70DC2B3B0E6B
:105A4000DC6505D0DC6B8F900D901BB60D8014A625
:105A500008D00301D32B310ED36503D0D36B14963A
:105A60008F900301E02B1D0EE06504D0E06BDF6B2F
:105A70000201EB6B40B494D20301DB2B180EDB6503
:105A80008FD2DB6B0101E06BF4C424F0F5C425F088
:105A90002CEC1CF00201FE6F15B416D0DC51010194
:105AA000D95DD8B0D9C1CDF30201DC510101D96172
:105AB0002FD0D9510201DC5D2A6E0F0E2A6428D046
:105AC0001584949C829C24D015A422D00101D45129
:105AD000050A0EE1D9510301CD5D2A6E230E0101A5
:105AE000D96503D0240E2A6002D0098C01D0099C0C
:105AF0000101D9510201DC610BD0DC510101D95DFA
:105B00002A6E0A0E2A6404D01594050E0201EA6F6B
:105B1000D9C1DCF215B00BAA05D00201FD51E00B92
:105B2000FE1903D00201FE51FD190101E06FE8C327
:105B300020F0E05180EC37F02B6E2B5001E18DD03E
:105B400015AE8AD02BA015D015A005D00101E051CB
:105B50008FEC31F00ED00101E0A106D0216A220EB7
:105B6000206E74EC23F005D0216A240E206E74ECB4
:105B700023F02BA215D015A005D00101E0512AEC8D
:105B80002EF00ED00101E0A306D0216A260E206E71
:105B900074EC23F005D0216A280E206E74EC23F0FB
:105BA0002BA415D015A005D00101E05113EC32F063
:105BB0000ED00101E0A506D0216A2A0E206E74ECF9
:105BC00023F005D0216A2C0E206E74EC23F02BA656
:105BD00015D015A005D00101E051D1EC31F00ED067
:105BE0000101E0A706D0216A2E0E206E74EC23F08E
:105BF00005D0216A300E206E74EC23F02BA815D04E
:105C000015A005D00101E0514DEC31F00ED001019D
:105C1000E0A906D0216A360E206E74EC23F005D080
:105C2000216A380E206E74EC23F02BAA15D015A033
:105C300005D00101E05166EC4DF00ED00101E0AB62
:105C400006D0216A900E206E74EC23F005D0216AF4
:105C5000920E206E74EC23F0158EE0C1E8F3E0C1E3
:105C6000E1F116A007D000011690216A400E206EC7
:105C700074EC23F007AE07D00001079E216A320EB4
:105C8000206E74EC23F008A007D000010890216A70
:105C9000340E206E74EC23F01CA80CD000011C986C
:105CA000216A440E206E74EC23F014B803D010A2C5
:105CB00010B4138212A607D000011296216A3E0E7C
:105CC000206E74EC23F017AC07D00001179C216AFA
:105CD000460E206E74EC23F00EA407D000010E9443
:105CE000216A880E206E74EC23F00DAE08D00001FE
:105CF0000D9E020E216EB40E206E74EC23F00FACDC
:105D000007D000010F9C216A8E0E206E74EC23F0E8
:105D10000FAA08D000010F9A020E216EB60E206E57
:105D200074EC23F008AC07D00001089C216A960EA1
:105D3000206E74EC23F015A607D000011596216A99
:105D40003A0E206E74EC23F015A807D000011598C8
:105D5000216A3C0E206E74EC23F018A807D00001D5
:105D60001898216A8A0E206E74EC23F019A007D0CF
:105D700000011990216A8C0E206E74EC23F018AC8F
:105D800008D00001189C020E216EB80E206E74EC33
:105D900023F019A408D000011994020E216EBA0E46
:105DA000206E74EC23F00201CD510AE0DE0ECD2509
:105DB000206E216A020E212274EC23F00201CD6BC9
:105DC0000BA407D000010B94216A200E206E74EC06
:105DD00023F00CA207D000010C92216A860E206EDF
:105DE00074EC23F00BAC07D000010B9C216A940EDD
:105DF000206E74EC23F0010E05A0000E296E010E3A
:105E000004AE000E291A15E0060E04BE070E0301AB
:105E1000F46F990EF56FF66F850EF76F490EF86FF8
:105E2000900EF96F050EFA6F178E178C059004BE51
:105E3000058007BC42D0010E09AE000E296E010E8E
:105E400009AA000E291A19E009AA04D0060E0301B6
:105E5000F46F04D0070E0301F46F8F90990EF56F65
:105E6000F66F850EF76F190EF86F900EF96FFA6BDB
:105E7000178E178C099E09BA098E010E0AA0000E12
:105E8000296E010E09AC000E291A1DE009AC04D0E0
:105E9000060E0301F46F04D0070E0301F46F8F9018
:105EA000990EF56FF66F850EF76F190EF86F900E5D
:105EB000F96FFA6B178E178C03D0099E09BA098EF9
:105EC0000A9009BC0A800201C86722D015BE0DB62F
:105ED0001FD006A003D006B451D052D006AC03D0D8
:105EE00007B04CD04DD00EAA03D00EBE47D048D03C
:105EF0000EA003D00EB642D043D008A403D008B8F9
:105F00003DD03ED01BA804D00201F35137E138D078
:105F100000F00201C96741D0000115AE3ED000017A
:105F20000DB83BD006A204D0000106B42FD030D06B
:105F300006AE04D0000107B029D02AD00EAC04D0A0
:105F400000010EBE23D024D00EB215A004D0000153
:105F500006BA1CD01DD00EA204D000010EB616D079
:105F600017D008A604D0000108B810D011D0000145
:105F70001BAA13D00201F45109E10AD08A8C02D085
:105F80008A9CC6D7030E0201C86FC2D78A8E02D080
:105F90008A9E03D0030E0201C96F00F08EEC44F01C
:105FA00013B802D013AA03D00201DA6B03D0010E9A
:105FB0000201DA6F0501124B132B1051125D1151C2
:105FC000135934E3126B136B0201DA6708D019B668
:105FD00003D08A988A962AD08D968D9427D0DA0598
:105FE00025E11FA016D01F9019B608D019B203D012
:105FF0008A988A860AD08A888A9607D018BA03D0E7
:106000008D968D8402D08D868D940501116B640E62
:106010000CD01F8019B603D08A988A9602D08D962C
:106020008D941F0E0501116F400E106F0501164B68
:10603000172B1451165D1551175960E3166B176B2A
:1060400004B002D00301CC6B0301CC6723D01FA2A4
:106050000CD01F9219B603D08D868D9402D08A88F9
:106060008A960501156B640E13D01F8219B603D0F2
:106070008D968D9402D08A988A9604B005D0010E30
:106080000501156F900E04D0090E0501156FC40EA1
:10609000146F34D0CC0512E11FA22AD01F9219B67A
:1060A00003D08D868D9402D08A888A9614B8ECD756
:1060B000D8D78A988A9614B8D4D7E6D7CC51020A92
:1060C0000AE11FA215D01F9219B602D08D860CD0FE
:1060D0008A888A86EBD7CC51030A10E11FA208D028
:1060E0001F9219B603D08D968D84E0D78A98F1D788
:1060F0001F8219B6DED78D968D94DDD712AC04D0F1
:106100008D968D948A988A960401F04BF12BE80EB7
:10611000F05D030EF15971E30201EA51D8A4EA07D8
:10612000EA0502E1EB6B948CF351D8A4F307F45128
:10613000D8A4F4070401F06BF16BE84BE92B0001E4
:1061400012ACFBEC19F00301D50715A006D0020133
:10615000CE5103E0CE2F01D01C840501FD51D8A4FF
:10616000FD070201F851D8A4F8071ABE0ED0E1517C
:106170000301D42BD45D02E3D46B16860301C12B3B
:106180001D0EC16502D0C16B1B8C1BAE08D0580E12
:106190000401DA5D020EDB5902E2DA4BDB2B06A6C4
:1061A0000AD00401D951D81103E18A9C069603D084
:1061B000D807D8A0D9071CAC09D005011F511E1162
:1061C00002E11C9C03D01E07D8A01F0714AC0AD004
:1061D0000401F351F21103E18A9E149C03D0F207EB
:1061E000D8A0F3070201C851D8A4C807C951D8A440
:1061F000C9070301CE51D8A4CE0705011A4B1B2BAA
:10620000600E1A5DEA0E1B59D8A012001A6B1B6BA8
:106210000301AD51AC1103E0AC07D8A0AD07AC054C
:10622000AD1104E107860301AC6BAD6BE42B15A047
:1062300008D00201CA5105E0CA2F03D0099008BE58
:106240008A9C0201E2510301D92BD95D02E3D96B8B
:106250001C820201DE510301D02BD05D02E3D06B22
:106260001C800301B32B020EB36501D0B36B050193
:10627000184B192B0A0E185D000E19591CE3186BE8
:10628000196B0301C42B8F0EC46502D0C46B0A8442
:106290000201F2510301E52BE55D0DE3E56B1C887E
:1062A000198A1BA803D0140E0201F36F1BAA03D096
:1062B000140E0201F46F0301D82B020ED865020CF4
:1062C000D86B0001158A12000101306B500E0101DC
:1062D0003025D96EDA6A060EDA2230511E6F1F6B36
:1062E0001EBF1F07F6EC37F0DF6E302B3051800AEF
:1062F000610FECE3306B000E01013025D96EDA6AD4
:10630000050EDA22800EC4DBF6EC37F0DF6E302BA0
:106310003051800A7A0FEFE31F6B550E1E6FF6ECBB
:1063200037F00201F26F01011F6B4B0E1E6FF6EC8E
:1063300037F0296F286B1F6B4A0E1E6FF6EC37F093
:1063400028110401F46F010129510401F56F0101C5
:106350001F6B520E1E6FF6EC37F00201FD6F01014C
:106360001F6B560E1E6FF6EC37F00201D16F010164
:106370001F6B570E1E6FF6EC37F00301B86F01016B
:106380001F6B760E1E6FF6EC37F0D86F1F6B590E31
:106390001E6FF6EC37F0296F286B1F6B5A0E1E6FBD
:1063A000F6EC37F02811C96F2951CA6F1F6B4F0ED9
:1063B0001E6FF6EC37F0306F1F96010130B51F8667
:1063C0001F9830B71F88306BB2DB9A0E55DBF6ECA6
:1063D00037F0DF6EACDBDF5005E0302B3051800A48
:1063E000700FF2E30101306B8ADBBA0E45DBF6EC8D
:1063F00037F0DF6E84DBDF5005E0302B3051800A50
:106400007B0FF2E31F9A0701C65104E00601F15128
:1064100001E01F8A01011F6B750E1E6FF6EC37F04D
:10642000306F189E010130B1188E1B9030B31B8065
:10643000119C30B7118C079430BF0784129E30BD79
:10644000128E1B9230B51B820D960690069C0E9AFA
:106450000E9008941B980D980692069E0E9C0E9224
:1064600008961B9A1F6B4C0E1E6FF6EC37F0306FC0
:10647000306702D00D8618D030B1FCD730A302D0DF
:10648000068012D030A502D0068C0ED030A702D0E4
:106490000E8A0AD030A902D00E8006D030AB02D0CE
:1064A000088402D030BD1B8801011F6B4D0E1E6F8A
:1064B000F6EC37F0306F306702D00D8818D030B16D
:1064C000FCD730A302D0068212D030A502D0068EAF
:1064D0000ED030A702D00E8C0AD030A902D00E8286
:1064E00006D030AB02D0088602D030BD1B8A030E26
:1064F00001011F6F500E1E6FF6EC37F0296F286BED
:10650000030E1F6F510E1E6FF6EC37F028110201BB
:10651000BA6F010129510201BB6F030E01011F6F08
:10652000520E1E6FF6EC37F0296F286B030E1F6FAB
:10653000530E1E6FF6EC37F028110201BC6F0101FB
:1065400029510201BD6F030E01011F6F540E1E6F12
:10655000F6EC37F0296F286B030E1F6F550E1E6F78
:10656000F6EC37F028110201BE6F0101295102013A
:10657000BF6F030E01011F6F560E1E6FF6EC37F052
:10658000296F286B030E1F6F570E1E6FF6EC37F046
:1065900028110201C06F010129510201C16F030ED0
:1065A00001011F6F580E1E6FF6EC37F0296F286B34
:1065B000030E1F6F590E1E6FF6EC37F02811020103
:1065C000C26F010129510201C36FE80EBA5D030ECB
:1065D000BB5917E3030E01011E6F500E1D6F030E12
:1065E0001F6FE2EC3DF0030E01011E6F510E1D6F97
:1065F0003E0E1F6FE2EC3DF0030E0201BB6F3E0E3C
:10660000BA6FE80EBC5D030EBD5917E3030E01011E
:106610001E6F520E1D6F030E1F6FE2EC3DF0030E56
:1066200001011E6F530E1D6F3E0E1F6FE2EC3DF019
:10663000030E0201BD6F3E0EBC6FE80EBE5D030E81
:10664000BF5917E3030E01011E6F540E1D6F030E99
:106650001F6FE2EC3DF0030E01011E6F550E1D6F22
:106660003E0E1F6FE2EC3DF0030E0201BF6F3E0EC7
:10667000BE6FE80EC05D030EC15917E3030E0101A2
:106680001E6F560E1D6F030E1F6FE2EC3DF0030EE2
:1066900001011E6F570E1D6F3E0E1F6FE2EC3DF0A5
:1066A000030E0201C16F3E0EC06FE80EC25D030E05
:1066B000C35917E3030E01011E6F580E1D6F030E21
:1066C0001F6FE2EC3DF0030E01011E6F590E1D6FAE
:1066D0003E0E1F6FE2EC3DF0030E0201C36F3E0E53
:1066E000C26F01011F6B6C0E1E6FF6EC37F00201DA
:1066F000F96F1D94F9B71D84070EF91701011F6B7F
:10670000680E1E6FF6EC37F00201FA6F1D9EFAB7A5
:106710001D8E070EFA1701011F6B690E1E6FF6EC36
:1067200037F00201FB6F1E94FBB71E84070EFB17A8
:1067300001011F6B6A0E1E6FF6EC37F00201FC6F51
:106740001E9AFCB71E8A070EFC1701011F6B540E20
:106750001E6FF6EC37F0306F3051F00B09E1069AFE
:106760001A9630C128F10F0E01012817282925D0CB
:106770003051F00B100A0FE1068A1A9630C128F149
:106780000F0E0101281728290001FA6F0401E16B9F
:10679000010EE06F14D03051F00B200A03E1069A8D
:1067A0001A86DFD73051F00B300A03E1068A1A86C9
:1067B000E5D7069A07981A96010E0201CC6F1DA420
:1067C0001DBE04D01EB402D01EAA02D01A8801D069
:1067D0001A9801011F6B640E1E6FF6EC37F003016F
:1067E000C56F01011F6B650E1E6FF6EC37F00301DC
:1067F000C66F01011F6B660E1E6FF6EC37F00201CB
:10680000D86F01011F6B670E1E6FF6EC37F00201A7
:10681000D36F01011F6B6B0E1E6FF6EC37F0306FFC
:106820001196010130B111860B9A30B50B8A089E82
:1068300015A007D0088E0D960690069C0E9A0E9015
:10684000089401011F6B700E1E6FF6EC37F0020109
:10685000E16F01011F6B720E1E6FF6EC37F0020143
:10686000E26F01011F6B710E1E6FF6EC37F0030132
:10687000CB6F01011F6B730E1E6FF6EC37F0020138
:10688000DE6F0101306B0DD98A0EF6D8F6EC37F0C9
:10689000DF6E07D9DF5005E0302B3051800A700FD2
:1068A000F2E310940601C55107E00DD9EBEC2FF08F
:1068B0002251211101E010840101306BF2D8CD0E7C
:1068C000E7D8F6EC37F0DF6EECD8DF5005E0302B80
:1068D0003051800A700FF2E310920601C55107E0B3
:1068E000F2D8EBEC2FF02251211101E010820101CE
:1068F000306BF6D8B30ECCD8F6EC37F0DF6EF0D8AC
:10690000DF5005E0302B3051800A700FF2E30101B7
:10691000306B15D9DD0EBCD8F6EC37F0DF6E0FD931
:10692000DF5005E0302B3051800A700FF2E3010197
:106930002F6B980E2E6F19A604D0030E2F6F200E0A
:106940002E6F0101306B0AD9B4D8F6EC37F0DF6E48
:1069500005D9DA22DF5005E0302B3051800A650F6F
:10696000F2E301012F6BED0E2E6F19A604D0030E7A
:106970002F6F3B0E2E6F0101306BBAD89AD8F6EC10
:1069800037F0DF6EB5D8DA22DF5005E0302B30511A
:10699000800A770FF2E301012F6BF60E2E6F19A616
:1069A00004D0030E2F6F440E2E6F0101306BCFD831
:1069B00080D8F6EC37F0DF6ECAD8DA22DF5005E077
:1069C000302B3051800A770FF2E30101306B9FD8F2
:1069D000550E52D8F6EC37F0DF6E99D8DF5005E04F
:1069E000302B3051800A600FF2E30101306B97D8F1
:1069F000750E42D8F6EC37F0DF6E91D8DF5005E027
:106A0000302B3051800A700FF2E3420E01011F6FEC
:106A10003A0E1E6FF6EC37F00201F66F500E0101D0
:106A20001F6FE50E1E6FF6EC37F02A6F500E1F6FCA
:106A3000E60E1E6FF6EC37F02B6F2A512D6F2B519F
:106A40002C6F000E2C5D550E2D5906E3000E2C5DAB
:106A5000800E2D59D8A01200500E1E6FE50E1D6F2E
:106A6000550E1F6FE2EC3DF0500E01011E6FE60E59
:106A70001D6F1F6BE2EF3DF0286F010E296F28514B
:106A800030251E6F000E30BFFF0E29211F6F120030
:106A900030251E6FE86AD8B0E82A30BFE8061F6FBD
:106AA0001200C50E01013025D96EDA6A060EDA220F
:106AB0001200DA222E5130251E6F000E30BFFF0E5D
:106AC0002F211F6F1200060E0101226FC50E216FCC
:106AD000FC0E246FDB0E236F266B070E256F070C51
:106AE000B60E01013025D96EDA6A070EDA221200DD
:106AF000DF0E01013025D96EDA6A060E1200F10EA2
:106B000001013025D96EDA6A060EDA221200D20EA1
:106B100001013025D96EDA6A080EDA221200A60EBB
:106B200001013025D96EDA6A070EDA221200C60E8C
:106B300001013025D96EDA6A070EDA221200D60E6C
:106B400001013025D96EDA6A070EDA221200E80E4A
:106B500001013025D96EDA6A060E12006B0E0101B2
:106B60003025D96EDA6A070E1200E8CF97F20201DB
:106B7000970510E1020E01011C6F500E1B6FA4EC73
:106B800048F00201966F966701D012000301D86B9E
:106B9000159A28D0966B14D002019651800A400FA6
:106BA00021E2310E9625D96EDA6A050EDA22500EF0
:106BB0009625E16EE26A020EE222DFCFE7FF962B16
:106BC000E5C5B2F10101B36B96C2B4F1B56BB4BFC8
:106BD000B507B551800AB66FB251B45DB351800AA2
:106BE000B659DAE30301D86B159A0201970567E1FC
:106BF000020E0101226F500E216FFE0E246FC50E92
:106C0000236F266B050E256FEBEC2FF0225121111F
:106C100018E1130E636F6A0E626F656B1E0E646F70
:106C2000020E0101676F500E666F97C268F1A1EC0A
:106C3000B9F001016351621104E102019751A5EC21
:106C40004AF0020E0101226F500E216FFB0E246FDD
:106C5000DC0E236F266B080E256FEBEC2FF0225114
:106C600021112DE1130E1E6F6A0E1D6F000E1F6B9A
